:020000040801F1
:100000000000022001F40108A92E0108B12E010808
:10001000B92E0108C12E0108C92E010800000000F8
:10002000000000000000000000000000D12E0108C8
:10003000DF2E010800000000ED2E0108FB2E010854
:1000400051F4010851F4010851F4010851F4010878
:1000500051F4010851F4010851F4010851F4010868
:1000600051F4010851F4010851F40108092F010865
:100070001D2F010851F4010851F4010851F4010841
:1000800051F4010851F4010851F4010851F4010838
:10009000312F010851F4010851F4010851F401080D
:1000A00051F4010851F4010851F4010851F4010818
:1000B00051F4010851F4010851F4010851F4010808
:1000C00051F4010851F4010851F4010851F40108F8
:1000D00051F4010851F4010851F4010851F40108E8
:1000E00051F4010851F4010851F4010851F40108D8
:1000F00051F4010851F4010851F4010851F40108C8
:1001000051F4010851F4010851F4010851F40108B7
:1001100051F4010851F4010851F4010851F40108A7
:1001200051F4010851F4010851F4010851F4010897
:1001300051F4010851F4010851F4010851F4010887
:1001400051F4010851F4010851F4010800000000C5
:10015000000000000000000000000000000000009F
:1001600000000000000000000000000051F4010841
:1001700051F4010851F4010851F4010851F4010847
:1001800051F4010851F4010851F4010851F4010837
:1001900051F401080000000051F4010851F4010875
:1001A00051F4010851F4010851F4010851F4010817
:1001B00051F4010851F4010851F4010851F4010807
:1001C00051F4010851F4010851F4010851F40108F7
:0801D00051F4010851F401088B
:1001E00010B5054C237833B9044B13B10448AFF371
:1001F00000800123237010BD0002002000000000D9
:10020000500A020808B5034B1BB103490348AFF37A
:10021000008008BD0000000004020020500A02080F
:1002200053B94AB9002908BF00281CBF4FF0FF315D
:100230004FF0FF3000F06AB9ADF1080C6DE904CE63
:1002400000F006F8DDF804E0DDE9022304B07047B1
:100250002DE9F047089D0C46002B4ED194468C4565
:100260008646B2FA82F262D94AB1C2F120039140C5
:1002700020FA03F30CFA02FC194300FA02FE4FEADB
:100280001C471FFA8CF6B1FBF7F44FEA1E4307FB3D
:10029000141143EA014304FB06F199420AD91CEB0D
:1002A000030304F1FF3080F01281994240F20F8184
:1002B000023C6344591A1FFA8EF3B1FBF7F007FBB7
:1002C000101143EA014300FB06F69E420AD91CEBDB
:1002D000030300F1FF3180F0FC809E4240F2F98080
:1002E000634402389B1B40EA044000211DB1D34007
:1002F0000022C5E90032BDE8F0878B4205D90DB177
:10030000C5E9000100210846F5E7B3FA83F10029A9
:1003100046D1A34202D39042C0F0F080861A64EB2B
:1003200003030120002DE6D0C5E90063E3E7002ABE
:1003300040F09080A1EB0C044FEA1C481FFA8CF7A8
:100340000121B4FBF8F64FEA1E4308FB164443EACA
:10035000044307FB06F0984208D91CEB030306F19F
:10036000FF3402D2984200F2CD8026461C1A1FFAB2
:100370008EF3B4FBF8F008FB104443EA044300FB9F
:1003800007F79F4208D91CEB030300F1FF3402D2A8
:100390009F4200F2B0802046DB1B40EA0640A5E702
:1003A000C1F120068B4022FA06F71F4320FA06FC13
:1003B00004FA01F343EA0C03F44000FA01F8380CA4
:1003C0004FEA1349B4FBF0FE1FFA87FC00FB1E4402
:1003D00049EA04440EFB0CF9A14502FA01F20AD9DC
:1003E0003C190EF1FF3A80F08480A14540F28180F3
:1003F000AEF1020E3C44A4EB09041FFA83F9B4FBEE
:10040000F0F300FB134449EA044403FB0CFCA4454D
:1004100007D93C1903F1FF3067D2A44565D9023BE7
:100420003C4443EA0E40A0FB0293A4EB0C049C4224
:10043000CE469C4651D34ED055B1B8EB0E0364EB7B
:100440000C0404FA06F6CB401E43CC40C5E9006418
:10045000002150E7C2F1200320FA03F10CFA02FC5C
:1004600024FA03F394400C434FEA1C4800FA02FEBE
:100470001FFA8CF7B3FBF8F008FB1031230C43EAAA
:10048000014300FB07F1994208D91CEB030300F17B
:10049000FF362CD299422AD9023863445B1AA4B29F
:1004A000B3FBF8F108FB113344EA034401FB07F303
:1004B000A34208D91CEB040401F1FF3613D2A34276
:1004C00011D902396444E41A41EA004139E704468B
:1004D000F0E6084606E7C845AED2B9EB020E63EB7C
:1004E000070C0138A8E73146EDE7034699E73046A7
:1004F000D4E7D6467FE7634402384DE706462346F5
:1005000008460FE7023E634430E700BF704700BF74
:10051000034613F8012B002AFBD1181A0138704743
:1005200001F0FF01102A2BDB10F0070F08D010F8A4
:10053000013B013A8B422DD010F0070F42B3F6D1A8
:10054000F0B441EA012141EA014122F007047FF0C1
:1005500000070023F0E80256083C85EA010586EA18
:10056000010685FA47F5A3FA87F586FA47F6A5FA54
:1005700087F68EB9EED1F0BC01F0FF0102F0070260
:1005800032B110F8013B013A83EA010313B1F8D10B
:100590000020704701387047002D06BF35460338EC
:1005A000073815F0010F07D1013015F4807F02BF25
:1005B000013015F4C03F0130F0BC0138704700BF76
:1005C000002310B50446C0E90033C0E9043383605A
:1005D00081814366C2818361194608225C3000F044
:1005E000F6F80D4B63620D4BA3620D4BE3620D4BAE
:1005F00023630D4B24629C4206D003F168029442AF
:1006000002D0D0339C4205D104F15800BDE810401F
:1006100000F050B910BD00BF450701086B07010885
:10062000A3070108C70701081C020020024A03496A
:10063000034800F069B800BF00000020B50B0108B6
:100640001000002041680C4B994210B5044601D0BF
:1006500000F0B0FAA168094B994202D0204600F0A0
:10066000A9FAE168064B994204D02046BDE8104043
:1006700000F0A0BA10BD00BF1C02002084020020C0
:10068000EC02002010B50B4B0B4C0C4A1A602046B4
:1006900000220421FFF794FF04F1680001220921E0
:1006A000FFF78EFF04F1D0000222BDE810401221B6
:1006B000FFF786BF540300201C0200202D0601080E
:1006C000014800F0F8B800BF5D030020014800F0C9
:1006D000F3B800BF5D03002010B50446FFF7F0FF3C
:1006E000236A1BB1BDE81040FFF7F0BF044B236243
:1006F000044B1B68002BF5D1FFF7C4FFF2E700BFE6
:1007000045060108540300202DE9F84307468846B2
:1007100014460026D4E90195B9F1010905D52468EC
:10072000002CF7D13046BDE8F883AB89012B07D9FF
:10073000B5F90E30013303D029463846C047064389
:100740006835E9E710B50C46B1F90E1000F06AF80B
:100750000028ABBF636DA3891B1823F48053ACBF83
:100760006365A38110BD002070472DE9F0411F464D
:100770008B89DB0505460C46164605D5B1F90E10EA
:100780000223002200F03CF8A389B4F90E1023F4F0
:100790008053A38132463B462846BDE8F04100F035
:1007A00053B810B50C46B1F90E1000F029F8431CEF
:1007B000A38915BF606523F4805343F48053A3815C
:1007C00018BFA38110BDB1F90E1000F009B80244A2
:1007D0000346934200D1704703F8011BF9E700007C
:1007E00038B5064D0023044608462B600EF0D4FDB4
:1007F000431C02D12B6803B1236038BD580300208D
:1008000038B5074D04460846114600222A601A46AC
:100810000EF0E9FD431C02D12B6803B1236038BD03
:100820005803002038B5074D0446084611460022FB
:100830002A601A460EF077FD431C02D12B6803B1E3
:10084000236038BD5803002038B5074D04460846DC
:10085000114600222A601A460EF082FD431C02D186
:100860002B6803B1236038BD5803002070B50D4DCF
:100870000D4C641BA4100026A64209D10B4D0C4C54
:1008800010F0E6F8641BA4100026A64205D170BD46
:1008900055F8043B98470136EEE755F8043B984776
:1008A0000136F2E7C00E0208C00E0208C00E0208B0
:1008B000C40E0208704770477047000038B50546FF
:1008C000002941D051F8043C0C1F002BB8BFE4189C
:1008D00000F0E0F81D4A136833B9636014602846DD
:1008E000BDE8384000F0DCB8A34208D920682118E0
:1008F0008B4201BF19685B6809182160EDE71A4651
:100900005B680BB1A342FAD911685018A0420BD111
:1009100020680144501883421160E0D118685B6878
:10092000536008441060DAE702D90C232B60D6E745
:10093000206821188B4204BF19685B68636004BF9C
:10094000091821605460CAE738BD00BF6403002065
:1009500070B50F4E0C463168054611B900F052F9DA
:1009600030602146284600F04DF9431C03D14FF07A
:10097000FF34204670BDC41C24F00304A042F8D00C
:10098000211A284600F03EF90130F2D1EFE700BF0E
:10099000600300202DE9F843CD1C25F00305083540
:1009A0000C2D38BF0C25002D064601DBA94204D9C9
:1009B0000C2333600020BDE8F883DFF8D48000F01A
:1009C00069F8D8F800301C4644BB29463046FFF78A
:1009D000BFFF431C044658D1D8F800402746002FDB
:1009E00043D1002C4BD023683946304604EB030931
:1009F00000F008F9814542D121686D1A2946304638
:100A0000FFF7A6FF01303AD023682B442360D8F8C3
:100A100000305A6862BBC8F800700FE02268521BB1
:100A200020D40B2A17D96119A342256018BF596039
:100A3000636808BFC8F8001062514B60304600F090
:100A40002FF804F10B00231D20F00700C21A1CBF71
:100A50001B1AA350AFE76268A3420CBFC8F800207E
:100A60005A60EBE723466468AEE73C467F68B6E72A
:100A70001A465B68A342FBD100235360DEE70C23D8
:100A80003360304600F00CF894E70560D6E700BF0D
:100A9000640300200148FFF70EBF00BF5C03002085
:100AA0000148FFF709BF00BF5C030020B1F90C202B
:100AB0002DE9F041160705460C4654D44B68002B2F
:100AC00002DC0B6C002B48DDE66A002E45D00023CB
:100AD00012F480522F68216A2B6030D0626DA38996
:100AE000590705D56368D21A636B0BB1236CD21A10
:100AF0000023E66A216A2846B047431CA38906D131
:100B000029681D292BD82A4A0A41D60727D4002252
:100B10006260D9042269226004D5421C01D12B688D
:100B200003B96065616B2F60B9B104F14403994268
:100B300002D02846FFF7C2FE002363630DE00123C5
:100B40002846B0470246501CC9D12B68002BC6D09E
:100B50001D2B01D0162B1ED12F60002022E043F068
:100B600040031BB21BE00F69002FF6D093070E68FD
:100B700008BF4B690F6018BF0023A6EB07088B6006
:100B8000B8F1000FE9DD216AA66A43463A462846D5
:100B9000B047002808DCB4F90C3043F04003A381CF
:100BA0004FF0FF30BDE8F0810744A8EB0008E7E70D
:100BB000FEFFBFDF38B50B6905460C4613B90025AB
:100BC000284638BD18B1036A0BB9FFF785FDB4F9A3
:100BD0000C30002BF3D0626ED00704D4990502D4F8
:100BE000A06DFFF768FE28462146FFF75FFF636EA2
:100BF000DA070546E4D4A3899B05E1D4A06DFFF78D
:100C00005BFEDDE738B5064D0023044608462B6041
:100C10000EF030FB431C02D12B6803B1236038BDBA
:100C20005803002090B585B000AF6423FB6006F048
:100C300075FF00F0C1F900F00DFC00F08FFE00F030
:100C4000BFFE00F057FF01F01DF801F0A7F800F01B
:100C50005FFC00F007FD01F0AFF902F09BFC01F032
:100C600023FF142200214E4801F094FF4C4801F06C
:100C7000F7FB0023BB6016E04A49BA6813465B00E5
:100C800013449B000B44043300221A604549BA68A0
:100C900013465B0013449B000B440833424A1A601E
:100CA000BB680133BB60BB68052BE5D97F213F489A
:100CB0000AF0CAFA7F213E480AF0C6FA04223D49EA
:100CC0003A4809F0BDFB02223B49394809F0B8FB1C
:100CD0003A4B1B6800225A63384B1B6800229A6308
:100CE000364B1B680022DA63354B1B6800225A63BF
:100CF000334B1B6800229A63314B1B680022DA6376
:100D000000212E480AF066FE04212C480AF062FEFB
:100D100008212A480AF05EFE002129480AF05AFEFE
:100D2000042127480AF056FE082125480AF052FE01
:100D300024480AF07DFD01F0B9FB01F0D7FE224BFB
:100D40001B78002B77D0214B1B78002B73D000230E
:100D50007B601FE013497A6813465B0013449B00D5
:100D60000B44D3ED007A9FED1A2ADFED1A1A9FED9E
:100D70001A1ADFED170AB0EE670A00F009FBF0EE71
:100D8000407A164A7B689B001344C3ED007A7B6867
:100D900001337B607B68052BDCD901233B603FE09E
:100DA000DC030020780300209A99993EF00300208C
:100DB0005C0400206803002070030020E005002090
:100DC0002C06002078060020740300207503002004
:100DD0000000C8420000000000C07345C0030020AE
:100DE0006D4A3B689B001344D3ED007A6A4B93ED48
:100DF000007AB0EE472ADFED691A9FED691ADFED40
:100E0000670AB0EE670A00F0C3FAF0EE407A624A71
:100E10003B689B001344C3ED007A3B6801333B60A1
:100E20003B68052BDCD900F0FBF95E4B00221A7001
:100E30005D4B00221A7006F0D5FE0246FB68D31AFD
:100E4000632B7FF678AF06F0CDFEF860574B1B782A
:100E500023F001044FF40061554808F0A3FA03465B
:100E600023435AB2514B1B785BB213435BB2DAB2E5
:100E70004E4B1A704D4B1B7823F002044FF48051F7
:100E80004B4808F08FFA03465B0023435AB2474BA6
:100E90001B785BB213435BB2DAB2444B1A70434B1C
:100EA0001B7823F004044FF40051414808F07AFA0B
:100EB00003469B0023435AB23C4B1B785BB213435F
:100EC0005BB2DAB2394B1A70384B1B7823F0080446
:100ED0004FF48041364808F065FA0346DB002343AF
:100EE0005AB2324B1B785BB213435BB2DAB22F4B70
:100EF0001A702E4B1B7823F010044FF400412C483D
:100F000008F050FA03461B0123435AB2274B1B78C3
:100F10005BB213435BB2DAB2244B1A70234B1B78DB
:100F200023F020044021234808F03CFA03465B01EB
:100F300023435AB21D4B1B785BB213435BB2DAB248
:100F40001A4B1A70194B1B7823F0400420211848C3
:100F500008F028FA03469B0123435AB2134B1B782F
:100F60005BB213435BB2DAB2104B1A700F4B1B78B3
:100F700023F0800410210E4808F014FA0346DB0128
:100F800023435AB2094B1B785BB213435BB2DAB20C
:100F9000064B1A70CFE600BFC0030020000000001F
:100FA0000000C8427403002075030020D80300200D
:100FB000000400480008004880B594B000AF07F175
:100FC0001803382200211846FFF701FC3B1D0022C0
:100FD0001A605A609A60DA601A61002008F06CFCAE
:100FE0002123BB614FF48033FB6101233B63022368
:100FF0007B630323BB630423FB6355233B6402230E
:101000007B640423BB640223FB6407F118031846C6
:1010100006F016FE0346002B01D000F015FA0F2350
:101020007B600323BB600023FB6000233B61002344
:101030007B613B1D0421184607F014F90346002B81
:1010400001D000F001FA00BF5037BD4680BD00005E
:1010500080B582B000AF78607B681B68B3F1A04FA9
:1010600002D100F00FF806E07B681B68044A934247
:1010700001D100F06DF800BF0837BD4680BD00BF4C
:101080000001005080B483B000AF00237B604FE0CC
:101090002C4A7B6832F8133007EE903AB8EEE77AC4
:1010A00029497A6813465B0013449B000B440833BC
:1010B000D3ED007A27EE277A23497A6813465B003E
:1010C00013449B000B440833D3ED007AF7EE006A1B
:1010D00076EEE76A1C497A6813465B0013449B006E
:1010E0000B4404331B6807EE903AF8EE677A66EE1D
:1010F000A77A77EE277A14497A6813465B0013447F
:101100009B000B44C3ED007A0E4A7B6832F8133023
:1011100018460D497A6813465B0013449B000B4444
:1011200004331860094B01221A707B6801337B601D
:101130007B68032BACD900BF00BF0C37BD465DF800
:10114000047B7047680300207803002074030020AC
:1011500080B483B000AF04237B6051E07B68043B24
:101160002C4A32F8133007EE903AB8EEE77A2A4963
:101170007A6813465B0013449B000B440833D3ED9D
:10118000007A27EE277A24497A6813465B001344D5
:101190009B000B440833D3ED007AF7EE006A76EE3D
:1011A000E76A1D497A6813465B0013449B000B44B1
:1011B00004331B6807EE903AF8EE677A66EEA77A7A
:1011C00077EE277A14497A6813465B0013449B0034
:1011D0000B44C3ED007A7B68043B0E4A32F81330AF
:1011E00018460D497A6813465B0013449B000B4474
:1011F00004331860094B01221A707B6801337B604D
:101200007B68052BAAD900BF00BF0C37BD465DF82F
:10121000047B7047700300207803002075030020D2
:1012200080B584B000AF544B93ED017A534B1B68EB
:101230001A4642F2107302FB03F307EE903AF8EEFF
:10124000677A9FED4F6AC7EE866AB0EE662ADFEDD9
:101250004D1A9FED4B1ADFED4B0AB0EE470A00F036
:1012600097F887ED030A444B93ED027A434B5B6892
:101270001A4642F2107302FB03F307EE903AF8EEBF
:10128000677A9FED3F6AC7EE866AB0EE662ADFEDA9
:101290003D1A9FED3B1ADFED3B0AB0EE470A00F026
:1012A00077F887ED020A344B93ED037A334B9B6852
:1012B0001A4642F2107302FB03F307EE903AF8EE7F
:1012C000677A9FED2F6AC7EE866AB0EE662ADFED79
:1012D0002D1A9FED2B1ADFED2B0AB0EE470A00F016
:1012E00057F887ED010A244B93ED047A234BDB6812
:1012F0001A4642F2107302FB03F307EE903AF8EE3F
:10130000677A9FED1F6AC7EE866AB0EE662ADFED48
:101310001D1A9FED1B1ADFED1B0AB0EE470A00F005
:1013200037F887ED000A184B1B68D7ED037AFCEEFF
:10133000E77A17EE902A5A63134B1B68D7ED027AAF
:10134000FCEEE77A17EE902A9A630F4B1B68D7EDF5
:10135000017AFCEEE77A17EE902ADA630B4B1B68F2
:10136000D7ED007AFCEEE77A17EE902A5A6300BFB9
:101370001037BD4680BD00BFC0030020DC03002045
:101380000000C84200000000E00500202C060020FC
:1013900080B489B000AF87ED050AC7ED040A87ED78
:1013A000031AC7ED021A87ED012A97ED057AD7EDEA
:1013B000047A37EE677AD7ED016AD7ED027A76EED6
:1013C000E77A67EE276A97ED037AD7ED047A37EE6E
:1013D000677AC6EE877A97ED027A77EE277AC7EDBD
:1013E000077A97ED027AD7ED077AB4EEE77AF1EE55
:1013F00010FA02DDBB68FB610AE097ED017AD7EDD8
:10140000077AB4EEE77AF1EE10FA01D57B68FB615A
:10141000FB6907EE903AB0EE670A2437BD465DF8E7
:10142000047B704780B582B000AF7860391D4FF6FD
:10143000FF73012203480BF019FC7B68184608373C
:10144000BD4680BDC406002080B400AF72B600BFA8
:1014500000BFFDE780B58AB000AF07F1140300229A
:101460001A605A609A60DA601A61264BDB6C254A72
:1014700043F02003D364234BDB6C03F020033B6178
:101480003B69204BDB6C1F4A43F00103D3641D4BC7
:10149000DB6C03F00103FB60FB681A4BDB6C194A41
:1014A00043F00203D364174BDB6C03F00203BB6011
:1014B000BB68144BDB6C134A43F00403D364114B39
:1014C000DB6C03F004037B607B684FF630037B61C9
:1014D0000023BB610223FB6107F1140319460A488C
:1014E00007F0DEFD40237B610023BB610223FB612B
:1014F00007F114031946054807F0D2FD00BF28374D
:10150000BD4680BD001002400004004800080048AD
:1015100080B58CB000AF07F1240300221A605A6036
:101520009A603B1D202200211846FFF750F9484BD6
:101530004FF0A0421A60464B4FF440325A60444B81
:1015400000229A60424B0022DA60414B00221A616D
:101550003F4B01225A613E4B04229A613C4B0022D0
:101560001A773B4B00225A77394B04221A62384BC8
:10157000002283F82420364B4FF49062DA62344B19
:101580004FF480621A63324B012283F83820304BCB
:101590000022DA632E4B002283F840202C4808F00A
:1015A00093FD0346002B01D0FFF74EFF00237B6223
:1015B00007F124031946264809F0A8FE0346002B2C
:1015C00001D0FFF741FF234B7B600623BB60022362
:1015D000FB607F233B6104237B610023BB613B1DD8
:1015E00019461B4809F014F80346002B01D0FFF7F9
:1015F0002BFF194B7B600C23BB603B1D1946144825
:1016000009F006F80346002B01D0FFF71DFF134B2E
:101610007B601223BB603B1D19460D4808F0F8FFA4
:101620000346002B01D0FFF70FFF0D4B7B60182303
:10163000BB603B1D1946064808F0EAFF0346002B35
:1016400001D0FFF701FF00BF3037BD4680BD00BFAE
:10165000F003002002003004040060080800900C31
:101660001000C01080B588B000AF3B46202200219A
:101670001846FFF7ACF8334B334A1A60314B4FF43E
:1016800040325A602F4B00229A602E4B0022DA60C3
:101690002C4B00221A612B4B01225A61294B042248
:1016A0009A61284B00221A77264B00225A77254B45
:1016B00002221A62234B002283F82420214B4FF48C
:1016C0009062DA621F4B4FF480621A631D4B012255
:1016D00083F838201B4B0022DA631A4B002283F870
:1016E0004020184808F0F0FC0346002B01D0FFF71B
:1016F000ABFE164B3B6006237B600223BB607F235F
:10170000FB6004233B6100237B613B4619460D4887
:1017100008F07EFF0346002B01D0FFF795FE0C4B2F
:101720003B600C237B603B461946064808F070FF7F
:101730000346002B01D0FFF787FE00BF2037BD46D0
:1017400080BD00BF5C040020000100500000524733
:101750000020903680B5A0B000AF786007F16C0330
:1017600000221A605A609A60DA601A6107F1180361
:10177000542200211846FFF72AF87B681B68B3F152
:10178000A04F6AD14FF40043BB614FF00053FB659B
:1017900007F11803184606F07DFF0346002B01D021
:1017A000FFF752FE664B1B680133654A1360644BBA
:1017B0001B68012B0BD1634BDB6C624A43F4005373
:1017C000D364604BDB6C03F400537B617B695D4B3E
:1017D000DB6C5C4A43F00103D3645A4BDB6C03F0CF
:1017E00001033B613B690F23FB6603233B67002337
:1017F0007B6707F16C0319464FF0904007F050FCEF
:10180000514B524A1A60504B05225A604E4B0022EF
:101810009A604D4B0022DA604B4B80221A614A4B92
:101820004FF480725A61484B4FF480629A61464B84
:101830002022DA61444B4FF480521A62424807F08A
:10184000C9FD0346002B01D0FFF7FEFD7B683E4A31
:101850005A653D4A7B6893626EE07B681B683C4A30
:10186000934269D14FF40043BB614FF00053FB65D5
:1018700007F11803184606F00DFF0346002B01D0B0
:10188000FFF7E2FD2E4B1B6801332D4A13602C4BF2
:101890001B68012B0BD12B4BDB6C2A4A43F4005302
:1018A000D364284BDB6C03F40053FB60FB68254BCF
:1018B000DB6C244A43F00103D364224BDB6C03F05E
:1018C0000103BB60BB683023FB6603233B67002337
:1018D0007B6707F16C0319464FF0904007F0E0FB7F
:1018E0001C4B1D4A1A601B4B24225A60194B0022C4
:1018F0009A60184B0022DA60164B80221A61154B51
:101900004FF480725A61134B4FF480629A61114B0D
:101910002022DA610F4B4FF480521A620D4807F013
:1019200059FD0346002B01D0FFF78EFD7B68094A65
:101930005A65084A7B68936200BF8037BD4680BD08
:101940008805002000100240C80400200800024062
:1019500000010050280500201C00024080B582B024
:1019600000AF164B9B6C154A43F004039364134B72
:101970009B6C03F004037B607B68104B9B6C0F4AED
:1019800043F0010393640D4B9B6C03F001033B6038
:101990003B68002200210B2008F01DF90B2008F005
:1019A00034F9002200210C2008F015F90C2008F071
:1019B0002CF900BF0837BD4680BD00BF00100240B3
:1019C00080B500AF1B4B1C4A1A601A4B1B4A5A6069
:1019D000184B00229A60174B0122DA60154B002247
:1019E0001A61144B00225A61124B00229A61114B6A
:1019F0000022DA610F4B00221A620E4809F08EFDB8
:101A00000346002B01D0FFF71FFD0021094809F014
:101A100020FE0346002B01D0FFF716FD00210548EC
:101A200009F062FE0346002B01D0FFF70DFD00BF59
:101A300080BD00BF8C05002000540040FBA7A030F3
:101A400080B59EB000AF786007F1640300221A6091
:101A50005A609A60DA601A6107F11003542200217B
:101A60001846FEF7B4FE7B681B681F4A934236D1C6
:101A700040233B610023FB6207F11003184606F088
:101A800009FE0346002B01D0FFF7DEFC174BDB6C91
:101A9000164A43F00203D364144BDB6C03F00203D9
:101AA000FB60FB684FF440737B661223BB66002328
:101AB000FB6600233B6704237B6707F16403194639
:101AC0000B4807F0EDFA094B9B6D084A43F40013ED
:101AD0009365064B9B6D03F40013BB60BB6800BFAE
:101AE0007837BD4680BD00BF005400400010024062
:101AF0000004004880B59CB000AF07F160030022ED
:101B00001A605A609A60DA6007F1540300221A6082
:101B10005A609A6007F1380300221A605A609A608E
:101B2000DA601A615A619A613B1D3422002118461D
:101B3000FEF74DFE514B524A1A60504B10225A602C
:101B40004E4B00229A604D4B42F20F72DA604B4BC3
:101B500000221A61494B00225A61484B80229A6147
:101B6000464809F00DFE0346002B01D0FFF76CFC40
:101B70004FF480533B6607F1600319463F480AF073
:101B80004FF90346002B01D0FFF75EFC3B4809F0FC
:101B9000BFFE0346002B01D0FFF756FC00237B65F8
:101BA0000023BB650023FB6507F154031946334846
:101BB0000AF0E2FE0346002B01D0FFF745FC60234C
:101BC000BB630023FB6300233B6400237B6400238F
:101BD000BB640023FB6400233B6507F1380300224C
:101BE000194626480AF008F80346002B01D0FFF7F3
:101BF0002BFC07F1380304221946204809F0FCFFAA
:101C00000346002B01D0FFF71FFC07F13803082221
:101C100019461A4809F0F0FF0346002B01D0FFF7E0
:101C200013FC00237B600023BB600023FB600023C8
:101C30003B6100237B614FF40053BB610023FB61D8
:101C400000233B6200237B624FF00073BB620023E2
:101C5000FB6200233B6300237B633B1D194607485F
:101C60000AF020FF0346002B01D0FFF7EDFB0348ED
:101C700000F028F900BF7037BD4680BDE0050020A8
:101C8000002C014080B58EB000AF07F12803002280
:101C90001A605A609A60DA6007F11C0300221A6029
:101CA0005A609A603B4600221A605A609A60DA6075
:101CB0001A615A619A61384B4FF080421A60364B74
:101CC00010225A60344B00229A60334B42F20F725A
:101CD000DA60314B00221A612F4B80229A612E4824
:101CE00009F04EFD0346002B01D0FFF7ADFB4FF48A
:101CF0008053BB6207F12803194627480AF090F881
:101D00000346002B01D0FFF79FFB234809F000FE9C
:101D10000346002B01D0FFF797FB0023FB61002354
:101D20007B6207F11C0319461B480AF025FE034697
:101D3000002B01D0FFF788FB60233B6000237B6012
:101D40000023BB6000233B613B460022194612483A
:101D500009F052FF0346002B01D0FFF775FB3B460D
:101D6000042219460C4809F047FF0346002B01D016
:101D7000FFF76AFB3B4608221946074809F03CFF7B
:101D80000346002B01D0FFF75FFB034800F09AF8F1
:101D900000BF3837BD4680BD2C06002080B588B016
:101DA00000AF07F1100300221A605A609A60DA60EF
:101DB0003B1D00221A605A609A601D4B1D4A1A6032
:101DC0001B4BA9225A601A4B00229A60184B40F212
:101DD000E732DA60164B00221A61154B80229A61B5
:101DE000134809F0CDFC0346002B01D0FFF72CFB74
:101DF0004FF480533B6107F1100319460C480AF079
:101E00000FF80346002B01D0FFF71EFB20237B6059
:101E10000023FB603B1D194605480AF0ADFD034653
:101E2000002B01D0FFF710FB00BF2037BD4680BD5F
:101E3000780600200004004080B487B000AF7860CE
:101E40007B681B681C4A93420CD11C4B1B6E1B4ABF
:101E500043F400631366194B1B6E03F400637B614C
:101E60007B6922E07B681B68B3F1804F0CD1134B78
:101E70009B6D124A43F001039365104B9B6D03F079
:101E800001033B613B6910E07B681B680C4A93428D
:101E90000BD10A4B9B6D094A43F002039365074B34
:101EA0009B6D03F00203FB60FB6800BF1C37BD465F
:101EB0005DF8047B704700BF002C01400010024019
:101EC0000004004080B58AB000AF786007F11403C9
:101ED00000221A605A609A60DA601A617B681B6897
:101EE000324A93421ED1324BDB6C314A43F001033C
:101EF000D3642F4BDB6C03F001033B613B694FF470
:101F0000E0637B610223BB610023FB6100233B6232
:101F100006237B6207F1140319464FF0904007F047
:101F2000BFF83FE07B681B68B3F1804F3AD1204B8C
:101F3000DB6C1F4A43F00203D3641D4BDB6C03F0E0
:101F40000203FB60FB681A4BDB6C194A43F0010388
:101F5000D364174BDB6C03F00103BB60BB684FF429
:101F600081637B610223BB610023FB6100233B6231
:101F700001237B6207F1140319460E4807F090F81D
:101F80004FF400437B610223BB610023FB6100230C
:101F90003B6201237B6207F1140319464FF0904026
:101FA00007F07EF800BF2837BD4680BD002C0140F9
:101FB000001002400004004880B500AF224B234AC5
:101FC0001A60214B4FF4E1325A601F4B00229A6095
:101FD0001D4B0022DA601C4B00221A611A4B0C22A6
:101FE0005A61194B00229A61174B0022DA61164B95
:101FF00000221A62144B00225A62134B00229A628A
:1020000011480AF0E3FD0346002B01D0FFF71CFA4C
:1020100000210D480BF00CFC0346002B01D0FFF70C
:1020200013FA002108480BF041FC0346002B01D0B5
:10203000FFF70AFA04480BF0C2FB0346002B01D05D
:10204000FFF702FA00BF80BDC4060020003801403F
:1020500080B59EB000AF786007F1640300221A607B
:102060005A609A60DA601A6107F110035422002165
:102070001846FEF7ACFB7B681B681E4A934235D1BD
:1020800001233B6100237B6107F11003184606F032
:1020900001FB0346002B01D0FFF7D6F9164B1B6E50
:1020A000154A43F480431366134B1B6E03F48043BD
:1020B000FB60FB68104BDB6C0F4A43F00203D364F8
:1020C0000D4BDB6C03F00203BB60BB68C0237B6677
:1020D0000223BB660023FB6600233B6707237B6765
:1020E00007F164031946054806F0DAFF00BF7837A8
:1020F000BD4680BD00380140001002400004004889
:1021000080B483B000AF786039607B6801333A688F
:10211000B3FBF2F2396801FB02F29B1A18460C3746
:10212000BD465DF8047B704780B582B000AF786033
:102130007B68002B05D1184B184A292118480DF04F
:1021400089F9786800F072F90346002B0AD07B68A1
:102150009A687B68DB6819461046FFF7D1FF024694
:102160007B689A607B685A687B68DB681946104612
:10217000FFF7C6FF02467B685A607B685A687B6837
:102180009B689A420CBF01230023DAB27B681A7461
:1021900000BF0837BD4680BD680A0208440C02082B
:1021A0006C0A020880B584B000AF786039607B6843
:1021B000002B02D03B68002B05D1174B174A382162
:1021C00017480DF047F914200DF062F90346FB6043
:1021D000FB68002B05D1134B104A3B2110480DF032
:1021E00039F9FB687A681A60FB683A68DA60F8685F
:1021F00000F01CF8F86800F0EDF80346002B05D15C
:10220000094B064A412106480DF024F9FB6818469F
:102210001037BD4680BD00BFA40A02085C0C02084E
:102220006C0A0208B40A0208BC0A020880B582B02F
:1022300000AF78607B68002B05D1094B094A4E211D
:1022400009480DF007F97B6800225A607B6800227C
:102250009A607B6800221A7400BF0837BD4680BDB3
:10226000680A0208700C02086C0A020880B584B083
:1022700000AF78607B68002B05D1164B164A5721BA
:1022800016480DF0E7F87B68DB68FB60786800F0C3
:10229000CDF8034683F00103DBB2002B15D07B6839
:1022A0005A687B689B689A4206D37B685A687B6849
:1022B0009B68D31AFB6008E07B68DA687B685B6820
:1022C0001A447B689B68D31AFB60FB68184610377A
:1022D000BD4680BD680A0208840C02086C0A020828
:1022E00080B584B000AF78600B46FB704FF0FF33D1
:1022F000FB607B68002B03D07B681B68002B05D13B
:102300000F4B104A7E2110480DF0A4F8786800F0B9
:102310008DF8034683F00103DBB2002B0BD07B6802
:102320001A687B685B681344FA781A707868FFF75C
:10233000FBFE0023FB60FB6818461037BD4680BDDE
:10234000D80A0208980C02086C0A020880B584B00A
:1023500000AF786039607B68002B06D03B68002BAB
:1023600003D07B681B68002B05D1174B174A8C21C3
:1023700017480DF06FF84FF0FF33FB60786800F0FE
:1023800029F8034683F00103DBB2002B17D07B68EA
:102390001A687B689B6813441A783B681A707B68DC
:1023A0009A687B68DB6819461046FFF7A9FE02466B
:1023B0007B689A607B6800221A740023FB60FB68CC
:1023C00018461037BD4680BDEC0A0208B00C020862
:1023D0006C0A020880B582B000AF78607B68002B81
:1023E00005D10F4B0F4A9D210F480DF033F8786847
:1023F00000F01CF8034683F00103DBB2002B07D08A
:102400007B685A687B689B689A4201D1012300E08F
:10241000002303F00103DBB218460837BD4680BD38
:10242000680A0208C40C02086C0A020880B582B06F
:1024300000AF78607B68002B05D1064B064AA421CB
:1024400006480DF007F87B681B7C18460837BD4628
:1024500080BD00BF680A0208D80C02086C0A020896
:1024600080B582B000AF78600B4A7B6813604FF490
:1024700080710A48FFF796FE0346094A13604FF43D
:1024800080710848FFF78EFE0346074A136000BFBD
:102490000837BD4680BD00BF740A002060070020D9
:1024A00058070020600800205C07002080B500AFBE
:1024B00000F01CF800F05EF800F092F800BF80BD5C
:1024C00080B584B000AF0346FB710023FB60064B70
:1024D0001B68FA7911461846FFF702FFF860FB689F
:1024E00018461037BD4680BD5807002080B582B021
:1024F00000AF1C4B1B681846FFF76CFF034683F0C8
:102500000103DBB2002B29D01DE0164B1B68FA1D1E
:1025100011461846FFF71AFFFB79184600F096F8A7
:102520000346002B14BF01230023DAB20E4B1A70AE
:102530000E4B1B78002B06D00D4B1B68FA79114609
:102540001846FFF7CDFE074B1B681846FFF742FF02
:10255000034683F00103DBB2002BD6D100BF08375E
:10256000BD4680BD58070020710A0020720A002075
:102570005C07002080B582B000AF174B1B6818467F
:10258000FFF728FF034683F00103DBB2002B1ED0C8
:10259000114B1B681846FFF769FE386000237B600B
:1025A0000BE00D4B1A687B680C490B44194610462A
:1025B000FFF7CCFE7B6801337B607A683B689A4208
:1025C000EFD33B689BB21946044801F0C3F900BF42
:1025D0000837BD4680BD00BF5C07002060090020B1
:1025E00080B500AF054B1B78002B04D0034B0022B5
:1025F0001A7000F07BF800BF80BD00BF710A002098
:1026000080B584B000AF786039600023FB600023A0
:10261000BB600FE00C4B18687A68BB6813441B78EA
:102620001946FFF75DFE0246FB681343FB60BB687B
:102630000133BB60BA683B689A42EBD3FB6818462B
:102640001037BD4680BD00BF5C07002080B485B058
:1026500000AF0346FB710023FB60FB790A2B02D01D
:10266000FB790D2B13D11E4B1B785A1CD1B21C4A7F
:1026700011701A461B4B0A219954194B1A781A4BA0
:102680001A70174B00221A700123FB6020E0FB79BF
:102690001B2B0BD1144B01221A70124B1B221A70E8
:1026A0000F4B00221A700123FB6011E00C4B1B78CA
:1026B0000F2B0AD80A4B1B785A1CD1B2084A11704A
:1026C0001946084AFB79535402E0054B00221A7060
:1026D000FB6818461437BD465DF8047B704700BFA1
:1026E000790A0020600A0020700A002080B582B0BC
:1026F00000AF01237B605D4B1B78052B00F2B1809E
:1027000001A252F823F000BF21270108B5270108D4
:10271000DF2701080B280108372801086328010872
:10272000534B1B78312B06D1012000F0F1F84F4BB1
:1027300001221A7096E04E4B1B78322B06D10220F4
:1027400000F0E6F8494B02221A708BE0484B1B78E8
:10275000332B06D1032000F0DBF8444B03221A7020
:1027600080E0434B1B78342B06D1042000F0D0F8D6
:102770003E4B04221A7075E03D4B1B78532B16D14B
:102780003C4B1B6814220021184600F0CBF97860FE
:10279000786800F0E1F8FFF7EDFE40F6B83005F09C
:1027A0002DFA324B00221A7000F07AF85AE000F04D
:1027B00077F857E02E4B1B781B2B05D12B4B0022B3
:1027C0001A7000F06DF84DE02A4B1B68184600F0B7
:1027D00053F8264B00221A7000F062F842E0244BB6
:1027E0001B781B2B05D1214B00221A7000F058F8E2
:1027F00038E0204B1B680433184600F03DF81B4BB3
:1028000000221A7000F04CF82CE0194B1B781B2B9F
:1028100005D1164B00221A7000F042F822E0154B49
:102820001B680833184600F027F8104B00221A7076
:1028300000F036F816E00E4B1B781B2B05D10B4B26
:1028400000221A7000F02CF80CE00A4B1B680C33C5
:10285000184600F011F8054B00221A7000F020F81D
:1028600000E000BF00BF0837BD4680BD780A0020E9
:10287000600A0020740A002080B584B000AF786040
:102880007A68054905480CF051FEF860FB68184667
:102890001037BD4680BD00BF080B0208600A00204B
:1028A000B0B5C6B004AF164B01221A7000F0DEF8C6
:1028B00000F0A0F8134B1B681C68124B1B685B6888
:1028C000104A126892680F490968C968381D0E4D90
:1028D000039502910192009323460C4A4FF48071B4
:1028E0000CF0F0FD0346C7F804313B1DD7F8041186
:1028F0001846FFF785FE00BF07F58477BD46B0BDDB
:10290000720A0020740A00208C0B02080C0B0208CB
:1029100080B5A4B000AF78600D4B01221A7000F0B2
:10292000A5F800F049F807F10C007B68094A8021FE
:102930000CF0C8FD0346C7F88C3007F10C03D7F83C
:102940008C101846FFF75CFE00BF9037BD4680BD77
:10295000720A0020940B020880B5A4B000AF786022
:1029600000F084F800F064F87B68002B0AD107F1CE
:102970000C030F4A802118460CF0A4FD0346C7F84B
:102980008C3009E007F10C030A4A802118460CF04C
:1029900099FD0346C7F88C3007F10C03D7F88C106B
:1029A0001846FFF72DFE00BF9037BD4680BD00BF23
:1029B000B40B0208C00B020880B586B000AF00233C
:1029C0007B6007F1080300221A605A609A603B1D81
:1029D000074A102118460CF075FD03467B613B1D2C
:1029E00079691846FFF70CFE00BF1837BD4680BD59
:1029F000D00B020880B586B000AF00237B6007F1E2
:102A0000080300221A605A609A603B1D074A102191
:102A100018460CF057FD03467B613B1D796918464B
:102A2000FFF7EEFD00BF1837BD4680BDD80B02088A
:102A300080B586B000AF00237B6007F10803002259
:102A40001A605A609A603B1D074A102118460CF024
:102A500039FD03467B613B1D79691846FFF7D0FDC0
:102A600000BF1837BD4680BDE00B020880B586B0B8
:102A700000AF00237B6007F1080300221A605A6050
:102A80009A603B1D074A102118460CF01BFD0346B7
:102A90007B613B1D79691846FFF7B2FD00BF18370F
:102AA000BD4680BDE80B020880B483B000AF0023B0
:102AB0007B600BE00B4A7B68134419780A4A7B68F9
:102AC00013440A461A707B6801337B607B68B3F558
:102AD000006FEFD3002318460C37BD465DF8047B2A
:102AE000704700BF00000508840A002080B500AFD1
:102AF00005F078F80246094B1B68D31A41F26F7251
:102B0000934208D9064B1B68002B04D100F070F8E3
:102B1000034B01221A6000BF80BD00BF7C0A002069
:102B2000800A002080B588B000AFF860B9607A6094
:102B300000237B61BA687B681344B3F5006F02D34E
:102B40004FF0FF331DE00023FB61BB68BB610DE06C
:102B5000FB695A1CFA61FA68134419780B4ABB697D
:102B600013440A461A70BB690133BB61BA697B68BA
:102B70009A42EDD300F03CF87861054B01221A60CF
:102B80007B6918462037BD4680BD00BF840A0020FF
:102B9000800A002080B487B000AFF860B9607A6026
:102BA000BA687B681344B3F5006F02D34FF0FF336C
:102BB00016E000237B61BB683B610CE07B695A1C1B
:102BC0007A61FA68134409493A690A4412781A701A
:102BD0003B6901333B613A697B689A42EED300233B
:102BE00018461C37BD465DF8047B7047840A0020F8
:102BF0002DE9F04FA7B000AF0023FB6706F004F803
:102C00000023FB668E4800F01FF903463B67A023B4
:102C10007B670123BB6707F17C0207F16C03114658
:102C2000184606F0DBF8034687F8973097F8973098
:102C3000002B04D006F00AF84FF0FF33FBE04FF40E
:102C40000063C7F890307E4BC7F88C300023C7F87C
:102C50008830E7E07B4AD7F8883013441B78DBB232
:102C60000022BB63FA63D7E90E23C7E92023D7F814
:102C700088305A1C734B9B5CDBB200229A46934609
:102C80004FF000004FF000014FEA0B2141EA1A61BA
:102C90004FEA0A20D7E9202342EA00063E630B43AD
:102CA0007B63D7E90C23C7E92023D7F888309A1C27
:102CB000644B9B5CDBB20022984691464FF00000CB
:102CC0004FF000014FEA094141EA18414FEA08403C
:102CD000D7E9202342EA0006BE620B43FB62D7E934
:102CE0000A23C7E92023D7F88830DA1C554B9B5CB0
:102CF000DBB200223B667A66D7E918120B461D0A42
:102D00000B461C06D7E9202342EA040139622B4313
:102D10007B62D7E90823C7E92023D7F888301A1D3A
:102D2000484B9B5CDBB20022BB65FA654FF00000AC
:102D30004FF00001BB6D19000020D7E9202342EAC3
:102D40000006BE610B43FB61D7E90623C7E92023D8
:102D5000D7F888305A1D3B4B9B5CDBB200223B65A9
:102D60007A654FF000004FF000013B6D1902002022
:102D7000D7E9202342EA00063E610B437B61D7E995
:102D80000423C7E92023D7F888309A1D2D4B9B5C7C
:102D9000DBB20022BB64FA644FF000004FF0000188
:102DA000BB6C19040020D7E9202342EA0006BE606C
:102DB0000B43FB60D7E90223C7E92023D7F888300B
:102DC000DA1D204B9B5CDBB200223B647A644FF03F
:102DD00000004FF000013B6C19060020D7E92023CA
:102DE00042EA00063E600B437B60D7E90023C7E957
:102DF0002023D7E92023D7F88C10002005F098FE77
:102E0000034687F89730D7F888300833C7F88830FA
:102E1000D7F88C300833C7F88C30D7F89030083B9F
:102E2000C7F89030D7F89030072B3FF613AF05F076
:102E30000DFF97F8973018469C37BD46BDE8F08FD8
:102E400000000508840A002080B485B000AF7860D7
:102E50000023FB600023BB607B6803F17842104BCA
:102E60001B884FF6FF718B4206D00D4B1B689B02EF
:102E700059080C4B0B4001E04FF48023B2FBF3F3F5
:102E8000BB60BB68002B02D10123FB6001E0022381
:102E9000FB60FB6818461437BD465DF8047B70473D
:102EA000E075FF1F00FEFF0180B400AF00BFFDE72B
:102EB00080B400AF00BFFDE780B400AF00BFFDE706
:102EC00080B400AF00BFFDE780B400AF00BFFDE7F6
:102ED00080B400AF00BFBD465DF8047B704780B48E
:102EE00000AF00BFBD465DF8047B704780B400AF03
:102EF00000BFBD465DF8047B704780B500AF04F0AD
:102F00005FFE00BF80BD000080B500AF024806F044
:102F100084FB00BF80BD00BFC804002080B500AFA7
:102F2000024806F07AFB00BF80BD00BF28050020E4
:102F300080B500AF024800F034FE00BF80BD00BF86
:102F40008412002080B582B000AF0F4B1B6E0E4A7A
:102F500043F0010313660C4B1B6E03F001037B600F
:102F60007B68094B9B6D084A43F080539365064B81
:102F70009B6D03F080533B603B6806F041FD00BF52
:102F80000837BD4680BD00BF0010024080B598B034
:102F900000AF786007F10C03542200211846FDF7BA
:102FA00016FC7B681B68154A934222D14FF40053EC
:102FB000FB600023BB6407F10C03184605F06AFBB5
:102FC0000346002B01D0FEF73FFA0D4B9B6D0C4AD8
:102FD00043F4000393650A4B9B6D03F40003BB604D
:102FE000BB6800220021142006F0F5FD142006F035
:102FF0000CFE00BF6037BD4680BD00BF005C0040D6
:103000000010024080B582B000AF78607B68D3F8D2
:10301000D8227B6803F52673194610460AF08AFD0C
:1030200000BF0837BD4680BD80B582B000AF786074
:103030000B46FB707B68D3F8D802FA7879681346A0
:103040009B001344DB000B4403F5B2731A68FB7852
:1030500019460AF0C4FD00BF0837BD4680BD80B5E3
:1030600082B000AF78600B46FB707B68D3F8D80263
:10307000FA78796813469B001344DB000B44243331
:103080001A68FB7819460AF00DFE00BF0837BD46E6
:1030900080BD80B582B000AF78607B68D3F8D8324D
:1030A00018460AF021FF00BF0837BD4680BD80B535
:1030B00084B000AF78600123FB737B685B79022BDF
:1030C00001D0FEF7C1F97B68D3F8D832FA7B1146FC
:1030D00018460AF0CBFE7B68D3F8D83218460AF0BF
:1030E00077FE00BF1037BD4680BD000080B582B0BE
:1030F00000AF78607B68D3F8D83218460AF0C6FE75
:103100007B685B7A002B05D0044B1B69034A43F0B4
:103110000603136100BF0837BD4680BD00ED00E027
:1031200080B582B000AF78607B685B7A002B07D0F7
:10313000084B1B69074A23F00603136100F0F8F9F6
:103140007B68D3F8D83218460AF0B6FE00BF0837BD
:10315000BD4680BD00ED00E080B582B000AF786074
:103160002B4A7B68C2F8D8327B68294AC3F8C4224C
:10317000274B284A1A60264B08221A71244B022238
:103180005A71234B0222DA71214B00221A72204B12
:1031900000225A721E4B00229A721D4B0022DA72D4
:1031A0001B4800F00EFC0346002B01D0FEF74CF943
:1031B0007B68D3F8C40218230022002102F0C7F86C
:1031C0007B68D3F8C40258230022802102F0BFF8A4
:1031D0007B68D3F8C402C0230022812102F0B7F833
:1031E0007B68D3F8C4024FF488730022012102F0F7
:1031F000AEF87B68D3F8C4024FF4807300228221BA
:1032000002F0A5F8002318460837BD4680BD00BF70
:1032100084120020005C004080B584B000AF78606C
:103220000023FB730023BB737B68D3F8C4321846BA
:1032300000F095FC0346FB73FB7B184600F07EF91B
:103240000346BB73BB7B18461037BD4680BD80B5B7
:1032500084B000AF7860084611461A460346FB70FA
:103260000B46BB7013463B800023FB730023BB73EC
:103270007B68D3F8C402BB783A88F97800F0DCFDAB
:103280000346FB73FB7B184600F058F90346BB73FB
:10329000BB7B18461037BD4680BD80B584B000AFFB
:1032A00078600B46FB700023FB730023BB737B68C5
:1032B000D3F8C432FA781146184600F01AFE0346D5
:1032C000FB73FB7B184600F039F90346BB73BB7BED
:1032D00018461037BD4680BD80B584B000AF786019
:1032E0000B46FB700023FB730023BB737B68D3F892
:1032F000C432FA781146184600F0C3FE0346FB7349
:10330000FB7B184600F01AF90346BB73BB7B1846DB
:103310001037BD4680BD80B584B000AF78600B46E5
:10332000FB700023FB730023BB737B68D3F8C432AC
:10333000FA781146184600F0F6FE0346FB73FB7B55
:10334000184600F0FBF80346BB73BB7B18461037EA
:10335000BD4680BD80B485B000AF78600B46FB7081
:103360007B68D3F8C432FB6097F90330002B0BDA8B
:10337000FB7803F07F02F96813469B001344DB00DF
:103380000B4412331B780BE0FB7803F07F02F968E3
:1033900013469B001344DB000B4403F5A9731B7811
:1033A00018461437BD465DF8047B704780B584B07D
:1033B00000AF78600B46FB700023FB730023BB73E8
:1033C0007B68D3F8C432FA781146184600F010FD35
:1033D0000346FB73FB7B184600F0B0F80346BB7353
:1033E000BB7B18461037BD4680BD80B586B000AFA8
:1033F000F8607A603B600B46FB720023FB7500238C
:10340000BB75FB68D3F8C402F97A3B687A6800F0B0
:1034100001FE0346FB75FB7D184600F08FF803465E
:10342000BB75BB7D18461837BD4680BD80B586B0DC
:1034300000AFF8607A603B600B46FB720023FB75BF
:103440000023BB75FB68D3F8C402F97A3B687A683D
:1034500000F097FD0346FB75FB7D184600F06EF803
:103460000346BB75BB7D18461837BD4680BD80B589
:1034700082B000AF78600B46FB707B68D3F8C43233
:10348000FA781146184600F0ADFD03461846083795
:10349000BD4680BD80B582B000AF78600B46FB7042
:1034A000FB78002B02D0012B13D023E07B685B7AE2
:1034B000002B07D000F03CF8104B1B690F4A23F09B
:1034C000060313617B68D3F8D83218460AF0F4FC7F
:1034D00010E07B68D3F8D83218460AF0D7FC7B6836
:1034E0005B7A002B05D0054B1B69044A43F00603A9
:1034F000136100BF00BF0837BD4680BD00ED00E08E
:1035000080B483B000AF7860034B18460C37BD46DB
:103510005DF8047B704700BF6015002080B483B065
:1035200000AF786000BF0C37BD465DF8047B704784
:1035300080B500AFFDF740FD00BF80BD80B485B011
:1035400000AF0346FB710023FB73FB79032B17D8F5
:1035500001A252F823F000BF693501086F35010858
:10356000753501087B3501080023FB730BE003234D
:10357000FB7308E00123FB7305E00323FB7302E008
:103580000323FB7300BFFB7B18461437BD465DF871
:10359000047B704780B500AF0022124912480AF040
:1035A00027FA0346002B01D0FDF74EFF0F490E48C6
:1035B0000AF04EFA0346002B01D0FDF745FF0C49F7
:1035C00009480BF0B1FD0346002B01D0FDF73CFF8D
:1035D00005480AF064FA0346002B01D0FDF734FFDA
:1035E00000BF80BD5C00002080170020FC00002090
:1035F000B000002080B483B000AF03463960FB7197
:103600003B6812221A80034B18460C37BD465DF802
:10361000047B70477C00002080B483B000AF034679
:103620003960FB713B6804221A80034B18460C3743
:10363000BD465DF8047B70479000002080B582B0E5
:1036400000AF03463960FB71FB79002B05D13A6866
:10365000074908480BF00BFA04E03A6804490548AA
:103660000BF005FA024B18460837BD4680BD00BF77
:10367000501A0020F00B020880B582B000AF03465C
:103680003960FB713A68044904480BF0F0F9024BC9
:1036900018460837BD4680BD501A0020080C0208A5
:1036A00080B582B000AF03463960FB713B681A22D7
:1036B0001A8000F043F8024B18460837BD4680BD1B
:1036C0009400002080B582B000AF03463960FB71E2
:1036D000FB79002B05D13A68074908480BF0C7F978
:1036E00004E03A68044905480BF0C1F9024B18465A
:1036F0000837BD4680BD00BF501A00201C0C0208D0
:1037000080B582B000AF03463960FB71FB79002BB6
:1037100005D13A68074908480BF0A9F904E03A686E
:10372000044905480BF0A3F9024B18460837BD467B
:1037300080BD00BF501A0020280C020880B584B05C
:1037400000AF0F4B1B68FB600E4B1B68BB600E4B42
:103750001B687B60FA687B681344FB60FB68002B86
:1037600009D008220949F86800F014F80422084931
:10377000B86800F00FF800BF1037BD4680BD00BF2D
:103780009075FF1F9475FF1F9875FF1F960000200E
:10379000A600002080B487B000AFF860B96013467F
:1037A000FB710023FB750023FB7527E0FB681B0FF3
:1037B000092B0BD8FB681B0FDAB2FB7D5B001946A7
:1037C000BB680B443032D2B21A700AE0FB681B0FA0
:1037D000DAB2FB7D5B001946BB680B443732D2B2CC
:1037E0001A70FB681B01FB60FB7D5B000133BA684C
:1037F000134400221A70FB7D0133FB75FA7DFB79BF
:103800009A42D3D300BF00BF1C37BD465DF8047B8E
:103810007047000080B500AF0022054905480BF055
:1038200098FC054903480BF0B2FC0023184680BD04
:103830005024002080170020501C002080B400AFCE
:1038400000231846BD465DF8047B704780B483B002
:1038500000AF03463960FB711346BB80FB79232B15
:103860004AD801A252F823F0F9380108F9380108C2
:10387000F9380108F9380108F9380108F938010860
:10388000F9380108F9380108F9380108F938010850
:10389000F9380108F9380108F9380108F938010840
:1038A000F9380108F9380108F9380108F938010830
:1038B000F9380108F9380108F9380108F938010820
:1038C000F9380108F9380108F9380108F938010810
:1038D000F9380108F9380108F9380108F938010800
:1038E000F9380108F9380108F9380108F9380108F0
:1038F000F9380108F938010800BF002318460C37D1
:10390000BD465DF8047B704780B584B000AF786039
:10391000396079680E480BF03AFC0D480BF080FCDA
:103920000023FB6009E07A68FB6813441B781846A3
:10393000FEF7C6FDFB680133FB603B681B68FA6855
:103940009A42F0D3002318461037BD4680BD00BF11
:103950008017002080B584B000AF78600B467B8074
:103960000023FB730D4BD3F8BC32BB60BB68D3F8AC
:103970001432002B01D001230BE07B881A467968B2
:1039800006480BF0E6FB05480BF01AFC0346FB73F8
:10399000FB7B18461037BD4680BD00BF8017002056
:1039A00080B487B000AFF860B9601346FB710023A4
:1039B000FB7597F9173018461C37BD465DF8047B38
:1039C000704780B584B000AF78607B68002B01D170
:1039D0000123C0E07B6893F89132DBB2002B06D163
:1039E0007B68002283F890227868FFF7CFFA7B6823
:1039F000032283F891227B681B68184601F02BFD97
:103A00000023FB733EE0FA7B796813469B00134466
:103A1000DB000B44113301221A70FA7B79681346DC
:103A20009B001344DB000B441033FA7B1A70FA7BC3
:103A3000796813469B001344DB000B4413330022C8
:103A40001A70FA7B796813469B001344DB000B4421
:103A5000203300221A60FA7B796813469B001344D6
:103A6000DB000B44243300221A60FB7B79685A1C6C
:103A700013469B001344DB000B4400221A60FB7BBF
:103A80000133FB737B681B79FA7B9A42BBD300231B
:103A9000FB7344E0FA7B796813469B001344DB0018
:103AA0000B4403F2511300221A70FA7B7968134613
:103AB0009B001344DB000B4403F5A873FA7B1A70D8
:103AC000FA7B796813469B001344DB000B4403F236
:103AD000531300221A70FA7B796813469B00134433
:103AE000DB000B4403F5B07300221A60FA7B79689F
:103AF00013469B001344DB000B4403F5B273002212
:103B00001A60FA7B796813469B001344DB000B4470
:103B100003F5B47300221A60FB7B0133FB737B68EF
:103B20001B79FA7B9A42B5D37B6818687B680433AB
:103B300093E8060001F0AAFC7B6800221A737B68F8
:103B4000012283F891227B689B7A012B02D178684D
:103B500001F040FC002318461037BD4680BD80B5FB
:103B600082B000AF78607B6893F89032012B01D16E
:103B7000022312E07B68012283F890227B681B6895
:103B8000184601F051FC7B681B68184603F011FFD2
:103B90007B68002283F89022002318460837BD4630
:103BA00080BD80B584B000AF78607B681B68184624
:103BB00003F016FFF860FB6803F40043002B03D00A
:103BC000786800F004FB10E1FB6803F48063002BCD
:103BD00013D07B681B68B3F844309AB27B681B68CB
:103BE00022F4806292B2A3F844207868FFF75FFA6B
:103BF0000021786800F0FCF8F7E0FB6803F48043EC
:103C0000002B0CD07B681B68B3F844309AB27B68F9
:103C10001B6822F4804292B2A3F84420E5E0FB68DE
:103C200003F40053002B0CD07B681B68B3F84430BE
:103C30009AB27B681B6822F4005292B2A3F8442027
:103C4000D3E0FB6803F48053002B34D07B681B68FF
:103C5000B3F840309AB27B681B6822F0040292B23B
:103C6000A3F840207B681B68B3F840309AB27B68A9
:103C70001B6822F0080292B2A3F840207B6893F8F8
:103C8000C832012B07D17B68002283F8C8220021AB
:103C90007868FFF7FFFB7868FFF742FA7B681B68DC
:103CA000B3F844309AB27B681B6822F4805292B217
:103CB000A3F8442099E0FB6803F40063002B27D0AD
:103CC0007B681B68B3F840309AB27B681B6842F08F
:103CD000080292B2A3F840207B681B68B3F8443016
:103CE0009AB27B681B6822F4006292B2A3F8442067
:103CF0007B681B68B3F840309AB27B681B6842F05F
:103D0000040292B2A3F840207868FFF7EFF96CE064
:103D1000FB6803F08003002B40D07B681B68B3F87E
:103D200044309AB27B681B6822F0800292B2A3F8FA
:103D300044207B6893F8C832002B2BD17B681B682A
:103D4000B3F840309AB27B681B6842F0040292B22A
:103D5000A3F840207B681B68B3F840309AB27B68B8
:103D60001B6842F0080292B2A3F840207B6801224F
:103D700083F8C8227B681B68B3F854309BB29B0859
:103D800003F03C027B68C3F8CC2201217868FFF77E
:103D900081FB2AE07868FFF7A9F926E0FB6803F4C5
:103DA0000073002B0FD07B681B68B3F844309AB2C5
:103DB0007B681B6822F4007292B2A3F844207868F2
:103DC000FFF767F911E0FB6803F48073002B0CD058
:103DD0007B681B68B3F844309AB27B681B6822F496
:103DE000807292B2A3F8442000BF1037BD4680BD58
:103DF00080B582B000AF78600B46FB707B6893F8AB
:103E00009032012B01D1022312E07B68012283F85A
:103E100090227B68FA781A737B681B68FA781146DF
:103E2000184603F0B2FD7B68002283F8902200233D
:103E300018460837BD4680BD80B584B000AF7860B5
:103E4000084611461A460346FB700B463B80134654
:103E5000BB700023FB7297F90330002B0EDAFB785E
:103E600003F0070213469B001344DB0010337A680B
:103E70001344FB60FB6801225A700EE0FB7803F0EC
:103E8000070213469B001344DB0003F5A8737A680E
:103E90001344FB60FB6800225A70FB7803F00703B1
:103EA000DAB2FB681A703A88FB681A61FB68BA7864
:103EB000DA70BB78022B02D1FB6800221A717B6892
:103EC00093F89032012B01D102230EE07B6801228E
:103ED00083F890227B681B68F968184601F0F4FAB1
:103EE0007B68002283F89022FB7A18461037BD4683
:103EF00080BD80B584B000AF78600B46FB7097F949
:103F00000330002B0EDAFB7803F0070213469B0008
:103F10001344DB0010337A681344FB60FB68012212
:103F20005A700EE0FB7803F0070213469B0013441F
:103F3000DB0003F5A8737A681344FB60FB6800227A
:103F40005A70FB7803F00703DAB2FB681A707B68DB
:103F500093F89032012B01D102230EE07B680122FD
:103F600083F890227B681B68F968184601F070FEA0
:103F70007B68002283F89022002318461037BD4644
:103F800080BD80B586B000AFF8607A603B600B46BC
:103F9000FB72FB7A03F0070213469B001344DB001D
:103FA00003F5A873FA6813447B617B697A685A61E8
:103FB0007B693A689A617B690022DA617B69002239
:103FC0005A70FB7A03F00703DAB27B691A70FB6858
:103FD0001B687969184602F028F80023184618373C
:103FE000BD4680BD80B483B000AF78600B46FB70E7
:103FF000FB7803F00702796813469B001344DB004B
:104000000B4403F5B6731B6818460C37BD465DF8C4
:10401000047B704780B586B000AFF8607A603B6083
:104020000B46FB72FB7A03F0070213469B00134416
:10403000DB001033FA6813447B617B697A685A614C
:104040007B693A689A617B69012283F824207B6945
:104050003A681A627B690022DA617B6901225A7030
:10406000FB7A03F00703DAB27B691A70FB681B68FE
:104070007969184601F0D9FF002318461837BD4664
:1040800080BD80B584B000AF78600B46FB70FB78D4
:1040900003F007037A681279934201D901233EE0C5
:1040A00097F90330002B0EDAFB7803F00702134672
:1040B0009B001344DB0010337A681344FB60FB68F9
:1040C00001225A700CE0FA7813469B001344DB007F
:1040D00003F5A8737A681344FB60FB6800225A70EA
:1040E000FB6801229A70FB7803F00703DAB2FB68E1
:1040F0001A707B6893F89032012B01D102230EE0F5
:104100007B68012283F890227B681B68F968184657
:1041100003F03CFB7B68002283F8902200231846C2
:104120001037BD4680BD80B584B000AF78600B46C7
:10413000FB70FB7803F00F037A681279934201D980
:10414000012340E097F90330002B0EDAFB7803F0EF
:10415000070213469B001344DB0010337A681344B4
:10416000FB60FB6801225A700EE0FB7803F0070247
:1041700013469B001344DB0003F5A8737A681344CD
:10418000FB60FB6800225A70FB6800229A70FB7883
:1041900003F00703DAB2FB681A707B6893F8903279
:1041A000012B01D102230EE07B68012283F89022CB
:1041B0007B681B68F968184603F039FB7B680022AE
:1041C00083F89022002318461037BD4680BD80B585
:1041D00096B000AF7860ADE37B681B68B3F84430FD
:1041E000A7F84E30B7F84E30DBB203F00F0387F874
:1041F0004D3097F84D30002B40F06F81B7F84E30BE
:1042000003F01003002B4CD17B681B681B889BB20A
:1042100023F4E14323F07003FB817B681A68FB8978
:104220006FEA43436FEA53439BB213807B681033BA
:104230007B657B681B68B3F850309BB21A467B6D78
:104240001B78DB0013447A681268134403F20243BC
:104250001B88C3F309027B6DDA617B6D5A697B6D44
:10426000DB691A447B6D5A6100217868FEF7F7FE1E
:104270007B681B7BDBB2002B00F05C837B6D9B6952
:10428000002B40F057837B681B7BDBB263F07F031E
:10429000DAB27B681B68A3F84C207B6800221A7393
:1042A00048E37B6803F5A8737B657B681B681B8804
:1042B000A7F84A30B7F84A3003F40063002B32D035
:1042C0007B681B68B3F850309BB21A467B6D1B7835
:1042D000DB0013447A681268134403F206431B8818
:1042E000C3F309027B6DDA617B6818687B6803F5AC
:1042F00026717B6DDA887B6DDB699BB203F0C2FBB4
:104300007B681B681B889AB240F68F7313403B8210
:104310007B681B683A8A42F0800292B21A80786801
:10432000FEF770FE06E3B7F94A30002B80F20283F5
:104330007B681B681B889AB240F68F731340FB831F
:104340007B681B68FA8B42F0800292B21A807B680D
:104350001B68B3F850309BB21A467B6D1B78DB00AC
:1043600013447A681268134403F206431B88C3F3AC
:1043700009027B6DDA617B6DDB69002B19D07B6DE7
:104380005B69002B15D07B6818687B6D59697B6D64
:10439000DA887B6DDB699BB203F074FB7B6D5A6935
:1043A0007B6DDB691A447B6D5A6100217868FEF7EA
:1043B0003BFE7B681B681B88A7F84A30B7F84A3079
:1043C00003F40063002B40F0B582B7F84A3003F4E1
:1043D0004053B3F5405F00F0AD827B681B68BB6162
:1043E0007B681B68B3F850309BB21A46BB69134414
:1043F000BB61BB6903F206437B617B691B889BB28F
:10440000C3F309039AB27B691A807B6D1B693E2B4B
:104410001DD97B6D1B695B097B647B6D1B6903F098
:104420001F03002B02D17B6C013B7B647B691B88E3
:104430009AB27B6C9BB29B029BB213439BB26FEA16
:1044400043436FEA53439AB27B691A8026E07B6D3F
:104450001B69002B0AD17B691B889BB26FEA43431F
:104460006FEA53439AB27B691A8017E07B6D1B6930
:104470005B087B647B6D1B6903F00103002B02D09A
:104480007B6C01337B647B691B889AB27B6C9BB22B
:104490009B029BB213439AB27B691A807B681B68AC
:1044A0001B889BB223F4804323F070037B827B8ABA
:1044B00083F480537B827B8A83F400537B827B6806
:1044C0001A687B8A43F07F4343F47F0343F400433D
:1044D00043F080039BB213802CE27B681B681A4672
:1044E00097F84D309B0013441B88A7F84A30B7F962
:1044F0004A30002B80F2F6807B681B681A4697F8DA
:104500004D309B0013441B889AB240F68F731340C2
:10451000A7F848307B681B681A4697F84D309B0017
:104520001344B7F8482042F0800292B21A8097F8FC
:104530004D2013469B001344DB0003F5A8737A68F3
:1045400013447B657B6D1B7B002B23D17B681B6831
:10455000B3F850309BB21A467B6D1B78DB001344D6
:104560007A681268134403F206431B88C3F30903F5
:10457000A7F85030B7F85030002B00F08E807B68E1
:1045800018687B6D59697B6DDA88B7F8503003F095
:1045900079FA82E07B6DDB78022B0AD1B7F84A30DA
:1045A0001A46796D786800F0D3F90346A7F85030C1
:1045B00073E07B681B681A467B6D1B789B00134475
:1045C0001B889BB223F4E04323F07003A7F852301A
:1045D0007B681B681A467B6D1B789B001A44B7F8F2
:1045E000523043F07F4343F47F0343F4004343F0EE
:1045F000C0039BB213807B681B681A467B6D1B78D7
:104600009B0013441B889BB203F48043002B22D0F1
:104610007B681B68B3F850309BB21A467B6D1B78E1
:10462000DB0013447A681268134403F202431B88C8
:10463000C3F30903A7F85030B7F85030002B2CD043
:104640007B6818687B6D59697B6D1A89B7F85030A3
:1046500003F018FA21E07B681B68B3F850309BB276
:104660001A467B6D1B78DB0013447A68126813448A
:1046700003F206431B88C3F30903A7F85030B7F8C9
:104680005030002B09D07B6818687B6D59697B6DB1
:104690005A89B7F8503003F0F5F97B6DDA69B7F84D
:1046A00050301A447B6DDA617B6D5A69B7F850302F
:1046B0001A447B6D5A617B6D9B69002B05D0B7F85E
:1046C00050207B6D1B699A4206D27B6D1B78194680
:1046D0007868FEF7A9FC05E07B681B68796D1846D1
:1046E00001F0A3FCB7F84A3003F08003002B00F080
:1046F000218197F84D2013469B001344DB001033B3
:104700007A6813447B657B681B681A4697F84D30BE
:104710009B0013441B889BB223F4E14323F07003F6
:10472000A7F842307B681B681A4697F84D309B000B
:104730001A44B7F842306FEA43436FEA53439BB2DF
:1047400013807B6DDB78012B40F0A2807B6D002213
:104750009A617B6D1B7B002B00F09380B7F84A3089
:1047600003F04003002B46D07B6D5B78002B26D1F5
:104770007B681B687B627B681B68B3F850309BB218
:104780001A467B6A13447B627B6D1B78DA007B6A76
:10479000134403F202433B623B6A1B889BB2C3F3A0
:1047A00009039AB23B6A1A803B6A1B889BB26FEA84
:1047B00043436FEA53439AB23B6A1A8061E07B6DD0
:1047C0005B78012B5DD17B681B68FB627B681B6893
:1047D000B3F850309BB21A46FB6A1344FB627B6D00
:1047E0001B78DA00FB6A134403F20243BB62BB6A24
:1047F00000221A8045E07B681B68FB637B6D5B7859
:10480000002B26D17B681B687B637B681B68B3F831
:1048100050309BB21A467B6B13447B637B6D1B78D5
:10482000DA007B6B134403F206433B633B6B1B884C
:104830009BB2C3F309039AB23B6B1A803B6B1B8894
:104840009BB26FEA43436FEA53439AB23B6B1A80C1
:1048500017E07B6D5B78012B13D17B681B68B3F885
:1048600050309BB21A46FB6B1344FB637B6D1B7885
:10487000DA00FB6B134403F20643BB63BB6B0022FD
:104880001A807B6D1B7819467868FEF7E8FB51E0CB
:10489000B7F84A3003F48073002B44D17B681B685F
:1048A000B3F850309BB21A467B6D1B78DB00134483
:1048B0007A681268134403F202431B88C3F30903A6
:1048C000A7F840307B6D9A69B7F840309A4207D913
:1048D0007B6D9A69B7F84030D21A7B6D9A6102E01D
:1048E0007B6D00229A617B6D9B69002B06D17B6DED
:1048F0001B7819467868FEF7B2FB1BE07B6D5A699E
:10490000B7F840301A447B6D5A617B6DDA69B7F8AD
:1049100040301A447B6DDA617B681B68796D1846FC
:1049200001F083FB06E0B7F84A301A46796D7868E3
:1049300000F017F97B681B68B3F844309BB21BB2D8
:10494000002BFFF649AC002318465837BD4680BD02
:1049500080B588B000AFF860B9601346FB80FB8873
:1049600003F48043002B7CD0FB681B68B3F8503005
:104970009BB21A46BB681B78DB001344FA681268C6
:10498000134403F202431B88C3F309037B83BB6810
:104990009A697B8B9A4206D3BB689A697B8BD21A41
:1049A000BB689A6102E0BB6800229A61BB689B69A0
:1049B000002B23D1FB681B681A46BB681B789B0041
:1049C00013441B889BB223F4804323F070033B8382
:1049D0003B8B83F400533B83FB681B681A46BB6820
:1049E0001B789B001A443B8B43F07F4343F47F03C7
:1049F00043F4004343F080039BB21380FB8803F031
:104A00004003002B1FD0FB681B681A46BB681B784D
:104A10009B0013441B889BB223F4E04323F07003F4
:104A2000FB82FB681B681A46BB681B789B001A4414
:104A3000FB8A43F07F4343F47F0343F4004343F096
:104A4000C0039BB213807B8B002B00F08580FB683A
:104A50001868BB685969BB681A897B8B03F012F828
:104A60007AE0FB681B68B3F850309BB21A46BB680B
:104A70001B78DB001344FA681268134403F2064300
:104A80001B88C3F309037B83BB689A697B8B9A42BB
:104A900006D3BB689A697B8BD21ABB689A6102E025
:104AA000BB6800229A61BB689B69002B23D1FB681D
:104AB0001B681A46BB681B789B0013441B889BB27B
:104AC00023F4804323F07003FB83FB8B83F40053B8
:104AD000FB83FB681B681A46BB681B789B001A4463
:104AE000FB8B43F07F4343F47F0343F4004343F0E5
:104AF00080039BB21380FB8803F04003002B1FD17F
:104B0000FB681B681A46BB681B789B0013441B8814
:104B10009BB223F4E04323F07003BB83FB681B6864
:104B20001A46BB681B789B001A44BB8B43F07F433B
:104B300043F47F0343F4004343F0C0039BB213806C
:104B40007B8B002B08D0FB681868BB685969BB6871
:104B50005A897B8B02F096FF7B8B18462037BD4627
:104B600080BD80B5A4B000AFF860B9601346FB808B
:104B7000FB8803F04003002B00F0DB81FB681B681F
:104B8000B3F850309BB21A46BB681B78DB00134465
:104B9000FA681268134403F202431B88C3F3090343
:104BA000A7F88630BB689A69B7F886309A4207D969
:104BB000BB689A69B7F88630D21ABB689A6102E07E
:104BC000BB6800229A61BB689B69002B40F0B980EA
:104BD000BB685B78002B26D1FB681B68FB62FB6817
:104BE0001B68B3F850309BB21A46FB6A1344FB6251
:104BF000BB681B78DA00FB6A134403F20243BB6212
:104C0000BB6A1B889BB2C3F309039AB2BB6A1A80C2
:104C1000BB6A1B889BB26FEA43436FEA53439AB265
:104C2000BB6A1A801AE0BB685B78012B16D1FB685F
:104C30001B687B63FB681B68B3F850309BB21A4655
:104C40007B6B13447B63BB681B78DA007B6B13447C
:104C500003F202433B633B6B00221A80FB681B6834
:104C60007B62BB685B78002B26D1FB681B68FB610D
:104C7000FB681B68B3F850309BB21A46FB691344BB
:104C8000FB61BB681B78DA00FB69134403F206433F
:104C9000BB61BB691B889BB2C3F309039AB2BB69B2
:104CA0001A80BB691B889BB26FEA43436FEA534388
:104CB0009AB2BB691A8017E0BB685B78012B13D1ED
:104CC000FB681B68B3F850309BB21A467B6A1344EA
:104CD0007B62BB681B78DA007B6A134403F20643ED
:104CE0003B623B6A00221A80BB681B781946F86851
:104CF000FEF7B5F9FB8803F48043002B00F0FA823D
:104D0000FB681B681A46BB681B789B0013441B8812
:104D10009BB223F4E04323F07003FB82FB681B6823
:104D20001A46BB681B789B001A44FB8A43F07F43FA
:104D300043F47F0343F4404343F080039BB213806A
:104D4000D8E2FB8803F48043002B21D0FB681B686A
:104D50001A46BB681B789B0013441B889BB223F444
:104D6000E04323F07003A7F88A30FB681B681A46FB
:104D7000BB681B789B001A44B7F88A3043F07F4326
:104D800043F47F0343F4404343F080039BB213801A
:104D9000BB6893F82430012B40F0AC82BB685A69A1
:104DA000B7F886301A44BB685A61BB68DA69B7F84D
:104DB00086301A44BB68DA61BB681A6ABB681B6933
:104DC0009A420BD3BB681B69C7F88C30BB681A6A60
:104DD000D7F88C30D21ABB681A6217E0BB681B6A1E
:104DE000002B08D1B7F88630C7F88C30BB6800229A
:104DF00083F824200AE0BB68002283F82420BB68E3
:104E00001B6AC7F88C30BB6800221A62BB685B78EB
:104E1000002B65D1FB681B68FB63FB681B68B3F85C
:104E200050309BB21A46FB6B1344FB63BB681B7884
:104E3000DA00FB6B134403F20243BB63BB6B1B88BA
:104E40009BB2C3F309039AB2BB6B1A80D7F88C30BC
:104E50003E2B1DD9D7F88C305B09BB64D7F88C305A
:104E600003F01F03002B02D1BB6C013BBB64BB6B87
:104E70001B889AB2BB6C9BB29B029BB213439BB242
:104E80006FEA43436FEA53439AB2BB6B1A8044E024
:104E9000D7F88C30002B0AD1BB6B1B889BB26FEA12
:104EA00043436FEA53439AB2BB6B1A8035E0D7F89D
:104EB0008C305B08BB64D7F88C3003F00103002B07
:104EC00002D0BB6C0133BB64BB6B1B889AB2BB6C5A
:104ED0009BB29B029BB213439AB2BB6B1A801CE03D
:104EE000BB685B78012B18D1FB681B687B64FB688F
:104EF0001B68B3F850309BB21A467B6C13447B643A
:104F0000BB681B78DA007B6C134403F202433B64FA
:104F1000D7F88C309AB23B6C1A80FB681868BB6873
:104F20005969BB681A89D7F88C309BB202F068FDCA
:104F3000E0E1FB681B68B3F850309BB21A46BB68CF
:104F40001B78DB001344FA681268134403F206432B
:104F50001B88C3F30903A7F88630BB689A69B7F8C2
:104F600086309A4207D3BB689A69B7F88630D21A5E
:104F7000BB689A6102E0BB6800229A61BB689B69CA
:104F8000002B40F0C080BB685B78002B26D1FB680B
:104F90001B68FB67FB681B68B3F850309BB21A466E
:104FA000FB6F1344FB67BB681B78DA00FB6F13448D
:104FB00003F20243BB67BB6F1B889BB2C3F30903B9
:104FC0009AB2BB6F1A80BB6F1B889BB26FEA4343D8
:104FD0006FEA53439AB2BB6F1A801AE0BB685B78E2
:104FE000012B16D1FB681B687B66FB681B68B3F856
:104FF00050309BB21A467B6E13447B66BB681B78AD
:10500000DA007B6E134403F202433B663B6E0022E0
:105010001A80FB681B687B67BB685B78002B2BD111
:10502000FB681B68FB66FB681B68B3F850309BB2DB
:105030001A46FB6E1344FB66BB681B78DA00FB6EF6
:10504000134403F20643C7F88030D7F880301B883A
:105050009BB2C3F309039AB2D7F880301A80D7F80D
:1050600080301B889BB26FEA43436FEA53439AB286
:10507000D7F880301A8017E0BB685B78012B13D11A
:10508000FB681B68B3F850309BB21A467B6F134421
:105090007B67BB681B78DA007B6F134403F206431F
:1050A0003B673B6F00221A80BB681B781946F86883
:1050B000FDF7D5FFFB8803F48043002B40F01A81F5
:1050C000FB681B681A46BB681B789B0013441B884F
:1050D0009BB223F4E04323F07003A7F88830FB6809
:1050E0001B681A46BB681B789B001A44B7F88830C7
:1050F00043F07F4343F47F0343F4404343F0800392
:105100009BB21380F6E0FB8803F48043002B21D18F
:10511000FB681B681A46BB681B789B0013441B88FE
:105120009BB223F4E04323F07003A7F84E30FB68F2
:105130001B681A46BB681B789B001A44B7F84E30B0
:1051400043F07F4343F47F0343F4404343F0800341
:105150009BB21380BB6893F82430012B40F0CA80C7
:10516000BB685A69B7F886301A44BB685A61BB6895
:10517000DA69B7F886301A44BB68DA61BB681A6A24
:10518000BB681B699A420BD3BB681B69C7F88C309C
:10519000BB681A6AD7F88C30D21ABB681A6217E05B
:1051A000BB681B6A002B08D1B7F88630C7F88C3073
:1051B000BB68002283F824200AE0BB681B6AC7F89A
:1051C0008C30BB6800221A62BB68002283F824205E
:1051D000FB681B687B65BB685B78002B65D1FB684F
:1051E0001B68FB65FB681B68B3F850309BB21A461E
:1051F000FB6D1344FB65BB681B78DA00FB6D134441
:1052000003F20643BB65BB6D1B889BB2C3F3090366
:105210009AB2BB6D1A80D7F88C303E2B1DD9D7F8C7
:105220008C305B09BB66D7F88C3003F01F03002B72
:1052300002D1BB6E013BBB66BB6D1B889AB2BB6ED5
:105240009BB29B029BB213439BB26FEA43436FEA4C
:1052500053439AB2BB6D1A8041E0D7F88C30002BD3
:105260000AD1BB6D1B889BB26FEA43436FEA53437D
:105270009AB2BB6D1A8032E0D7F88C305B08BB66FF
:10528000D7F88C3003F00103002B02D0BB6E013342
:10529000BB66BB6D1B889AB2BB6E9BB29B029BB276
:1052A00013439AB2BB6D1A8019E0BB685B78012B7F
:1052B00015D1FB681B68B3F850309BB21A467B6D62
:1052C00013447B65BB681B78DA007B6D134403F2E3
:1052D00006433B65D7F88C309AB23B6D1A80FB6869
:1052E0001868BB685969BB685A89D7F88C309BB27B
:1052F00002F086FBFB681B681A46BB681B789B00A4
:1053000013441B889BB223F4E04323F04003BB8289
:10531000BB8A83F01003BB82BB8A83F02003BB826D
:10532000FB681B681A46BB681B789B001A44BB8A43
:1053300043F07F4343F47F0343F4004343F080038F
:105340009BB21380002318469037BD4680BD80B4C1
:1053500087B000AFF8607B600B467B8113463B81D2
:105360007B8903F080039BB2002B0BD07B8903F079
:10537000070213469B001344DB001033FA68134402
:105380007B6109E07A8913469B001344DB0003F537
:10539000A873FA6813447B613B89002B07D17B69B2
:1053A00000221A737B689AB27B69DA800BE07B6912
:1053B00001221A737B689AB27B691A817B681B0C85
:1053C0009AB27B695A81002318461C37BD465DF8A6
:1053D000047B704780B485B000AF78607B681B6841
:1053E000FB607B680122C3F8D0227B68002283F82F
:1053F000C822FB68B3F854309BB243F001039AB261
:10540000FB68A3F85420FB68B3F854309BB243F018
:1054100002039AB2FB68A3F85420002318461437FD
:10542000BD465DF8047B704780B485B000AF7860FE
:105430007B680022A3F844204BF68073FB60FB6876
:105440009AB27B68A3F84020002318461437BD4663
:105450005DF8047B704780B485B000AF78604BF690
:105460008073FB607B68B3F840309AB2FB689BB2F4
:10547000DB439BB213409AB27B68A3F84020002321
:1054800018461437BD465DF8047B704780B485B07C
:1054900000AFF8603B1D83E80600FB680122A3F81B
:1054A0004020FB680022A3F84020FB680022A3F8FC
:1054B0004420FB680022A3F850200023184614372C
:1054C000BD465DF8047B704780B49DB000AF786046
:1054D0003960002387F86F307A683B681B789B003F
:1054E00013441B889BB223F4EC4323F07003A7F80A
:1054F0006C303B68DB78032B1FD801A252F823F0F5
:10550000115501082D550108435501081F55010883
:10551000B7F86C3043F40073A7F86C3012E0B7F8BA
:105520006C3043F4C063A7F86C300BE0B7F86C3014
:1055300043F48063A7F86C3004E0012387F86F30F0
:1055400000E000BF7A683B681B789B001A44B7F8FC
:105550006C3043F07F4343F47F0343F4004343F054
:1055600080039BB213807A683B681B789B001344CE
:105570001B889BB21BB223F4E04323F070031AB2E2
:105580003B681B781BB213431BB2A7F866307A68DE
:105590003B681B789B001A44B7F8663043F07F43A2
:1055A00043F47F0343F4004343F080039BB2138032
:1055B0003B681B7B002B40F078813B685B78002BBD
:1055C00000F084807B68BB617B68B3F850309BB28D
:1055D0001A46BB691344BB613B681B78DA00BB69A0
:1055E000134403F580637B613B68DB885B089BB2F7
:1055F0005B009AB27B691A807A683B681B789B00D3
:1056000013441B887B827B8A03F04003002B1BD052
:105610007A683B681B789B0013441B889BB223F479
:10562000E04323F070033B827A683B681B789B0061
:105630001A443B8A43F07F4343F47F0343F400431F
:1056400043F0C0039BB213803B68DB78012B20D072
:105650007A683B681B789B0013441B889BB223F439
:10566000E04323F04003BB81BB8983F02003BB816F
:105670007A683B681B789B001A44BB8943F07F43E0
:1056800043F47F0343F4004343F080039BB2138051
:10569000D5E27A683B681B789B0013441B889BB259
:1056A00023F4E04323F04003FB817A683B681B78D6
:1056B0009B001A44FB8943F07F4343F47F0343F488
:1056C000004343F080039BB21380B8E27B683B63E6
:1056D0007B68B3F850309BB21A463B6B13443B6374
:1056E0003B681B78DA003B6B134403F20443FB6214
:1056F0003B68DB885B089BB25B009AB2FB6A1A804E
:105700007B68BB627B68B3F850309BB21A46BB6AB9
:105710001344BB623B681B78DA00BB6A134403F294
:1057200006437B627B6A1B889BB2C3F309039AB270
:105730007B6A1A803B681B693E2B1DD93B681B693D
:105740005B09BB663B681B6903F01F03002B02D19A
:10575000BB6E013BBB667B6A1B889AB2BB6E9BB279
:105760009B029BB213439BB26FEA43436FEA5343DE
:105770009AB27B6A1A8026E03B681B69002B0AD12B
:105780007B6A1B889BB26FEA43436FEA53439AB22A
:105790007B6A1A8017E03B681B695B08BB663B6845
:1057A0001B6903F00103002B02D0BB6E0133BB6603
:1057B0007B6A1B889AB2BB6E9BB29B029BB213435F
:1057C0009AB27B6A1A807A683B681B789B00134404
:1057D0001B887B847B8C03F48043002B1BD07A686E
:1057E0003B681B789B0013441B889BB223F4E04367
:1057F00023F070033B847A683B681B789B001A4453
:105800003B8C43F07F4343F47F0343F4404343F036
:1058100080039BB213803B681B78002B24D17A68ED
:105820003B681B789B0013441B889BB223F4804386
:1058300023F07003BB83BB8B83F48053BB83BB8B90
:1058400083F40053BB837A683B681B789B001A443F
:10585000BB8B43F07F4343F47F0343F4004343F0A7
:1058600080039BB21380EAE17A683B681B789B0057
:1058700013441B889BB223F4804323F07003FB8303
:10588000FB8B83F40053FB837A683B681B789B0097
:105890001A44FB8B43F07F4343F47F0343F40043FC
:1058A00043F080039BB21380C9E13B68DB78022B95
:1058B0001ED17A683B681B789B0013441B889BB2FF
:1058C00023F4E04323F07003A7F862307A683B6862
:1058D0001B789B001A44B7F8623043F07F4343F4CF
:1058E0007F0343F4014343F080039BB213801DE028
:1058F0007A683B681B789B0013441B889BB223F497
:10590000E24323F07003A7F864307A683B681B78A1
:105910009B001A44B7F8643043F07F4343F47F039D
:1059200043F4004343F080039BB213807B68FB6524
:105930007B68B3F850309BB21A46FB6D1344FB658D
:105940003B681B78DA00FB6D134403F58063BB658D
:105950003B681B895B089BB25B009AB2BB6D1A80E7
:105960007B687B657B68B3F850309BB21A467B6DD1
:1059700013447B653B681B78DA007B6D134403F2AC
:1059800004433B653B685B895B089BB25B009AB252
:105990003B6D1A803B685B78002B40F093807A68FF
:1059A0003B681B789B0013441B88A7F84030B7F86E
:1059B000403003F48043002B1BD07A683B681B788F
:1059C0009B0013441B889BB223F4E04323F0700335
:1059D000FB877A683B681B789B001A44FB8F43F077
:1059E0007F4343F47F0343F4404343F080039BB27F
:1059F00013807A683B681B789B0013441B88BB8725
:105A0000BB8F03F04003002B1BD07A683B681B78E8
:105A10009B0013441B889BB223F4E04323F07003E4
:105A20007B877A683B681B789B001A447B8F43F026
:105A30007F4343F47F0343F4004343F0C0039BB22E
:105A400013807A683B681B789B0013441B889BB2C9
:105A500023F4804323F070033B873B8F83F4805310
:105A60003B873B8F83F400533B877A683B681B7806
:105A70009B001A443B8F43F07F4343F47F0343F47E
:105A8000004343F080039BB213807A683B681B7825
:105A90009B0013441B889BB223F4E04323F0400394
:105AA000FB867A683B681B789B001A44FB8E43F0A8
:105AB0007F4343F47F0343F4004343F080039BB2EE
:105AC0001380BCE07A683B681B789B0013441B88FA
:105AD000A7F84E30B7F84E3003F48043002B1DD0AA
:105AE0007A683B681B789B0013441B889BB223F4A5
:105AF000E04323F07003A7F84C307A683B681B78CA
:105B00009B001A44B7F84C3043F07F4343F47F03C3
:105B100043F4404343F080039BB213807A683B68B0
:105B20001B789B0013441B88A7F84A30B7F84A300B
:105B300003F04003002B1DD07A683B681B789B0064
:105B400013441B889BB223F4E04323F07003A7F8AF
:105B500048307A683B681B789B001A44B7F8483095
:105B600043F07F4343F47F0343F4004343F0C00317
:105B70009BB213803B68DB78012B24D07A683B68AA
:105B80001B789B0013441B889BB223F4E04323F053
:105B90004003A7F84430B7F8443083F02003A7F857
:105BA00044307A683B681B789B001A44B7F844304D
:105BB00043F07F4343F47F0343F4004343F0800307
:105BC0009BB213801DE07A683B681B789B001344EE
:105BD0001B889BB223F4E04323F04003A7F8463030
:105BE0007A683B681B789B001A44B7F8463043F04C
:105BF0007F4343F47F0343F4004343F080039BB2AD
:105C000013807A683B681B789B0013441B889BB207
:105C100023F4804323F07003A7F842307A683B688E
:105C20001B789B001A44B7F8423043F07F4343F49B
:105C30007F0343F4004343F080039BB2138097F843
:105C40006F3018467437BD465DF8047B704700BF5F
:105C500080B48DB000AF786039603B681B7B002B4F
:105C600040F08E803B685B78002B44D07A683B68BC
:105C70001B789B0013441B88BB81BB8903F0400346
:105C8000002B1BD07A683B681B789B0013441B8851
:105C90009BB223F4E04323F070037B817A683B6876
:105CA0001B789B001A447B8943F07F4343F47F03B6
:105CB00043F4004343F0C0039BB213807A683B680F
:105CC0001B789B0013441B889BB223F4E04323F012
:105CD00040033B817A683B681B789B001A443B89F0
:105CE00043F07F4343F47F0343F4004343F08003D6
:105CF0009BB2138092E17A683B681B789B00134447
:105D00001B887B827B8A03F48043002B1BD07A683C
:105D10003B681B789B0013441B889BB223F4E04331
:105D200023F070033B827A683B681B789B001A441F
:105D30003B8A43F07F4343F47F0343F4404343F003
:105D400080039BB213807A683B681B789B001344E6
:105D50001B889BB223F4804323F07003FB817A6895
:105D60003B681B789B001A44FB8943F07F4343F454
:105D70007F0343F4004343F080039BB213804DE163
:105D80003B685B78002B40F0A5807A683B681B7805
:105D90009B0013441B883B843B8C03F48043002B03
:105DA0001BD07A683B681B789B0013441B889BB20E
:105DB00023F4E04323F07003FB837A683B681B788D
:105DC0009B001A44FB8B43F07F4343F47F0343F46F
:105DD000404343F080039BB213807A683B681B7892
:105DE0009B0013441B88BB83BB8B03F04003002B39
:105DF0001BD07A683B681B789B0013441B889BB2BE
:105E000023F4E04323F070037B837A683B681B78BC
:105E10009B001A447B8B43F07F4343F47F0343F49E
:105E2000004343F0C0039BB213807A683B681B7841
:105E30009B0013441B889BB223F4E04323F07003C0
:105E40003B837A683B681B789B001A443B8B43F08A
:105E50007F4343F47F0343F4004343F0C0039BB20A
:105E600013807A683B681B789B0013441B889BB2A5
:105E700023F4804323F07003FB827A683B681B782D
:105E80009B001A44FB8A43F07F4343F47F0343F4AF
:105E9000004343F080039BB213807A683B681B7811
:105EA0009B0013441B889BB223F4E04323F0400380
:105EB000BB827A683B681B789B001A44BB8A43F01C
:105EC0007F4343F47F0343F4004343F080039BB2DA
:105ED0001380A3E07A683B681B789B0013441B88FF
:105EE000FB85FB8D03F48043002B1BD07A683B6855
:105EF0001B789B0013441B889BB223F4E04323F0E0
:105F00007003BB857A683B681B789B001A44BB8D85
:105F100043F07F4343F47F0343F4404343F0800363
:105F20009BB213807A683B681B789B0013441B88E4
:105F30007B857B8D03F04003002B1BD07A683B6888
:105F40001B789B0013441B889BB223F4E04323F08F
:105F500070033B857A683B681B789B001A443B8D35
:105F600043F07F4343F47F0343F4004343F0C00313
:105F70009BB213807A683B681B789B0013441B8894
:105F80009BB223F4E04323F07003FB847A683B6800
:105F90001B789B001A44FB8C43F07F4343F47F0340
:105FA00043F4404343F080039BB213807A683B681C
:105FB0001B789B0013441B889BB223F4E04323F01F
:105FC0004003BB847A683B681B789B001A44BB8CF7
:105FD00043F07F4343F47F0343F4004343F08003E3
:105FE0009BB213807A683B681B789B0013441B8824
:105FF0009BB223F4804323F070037B847A683B6870
:106000001B789B001A447B8C43F07F4343F47F034F
:1060100043F4004343F080039BB2138000231846EF
:106020003437BD465DF8047B704780B5C2B000AF21
:1060300007F58473A3F58273186007F58473A3F5DD
:106040008473196007F58473A3F584731B685B7808
:10605000012B40F0B78607F58473A3F584731B68A2
:106060009A6907F58473A3F584731B681B699A42C8
:1060700008D907F58473A3F584731B681B69C7F8F7
:10608000043107E007F58473A3F584731B689B69EB
:10609000C7F8043107F58473A3F584731B681B7B71
:1060A000002B3AD107F58473A3F584731B685969F3
:1060B00007F58473A3F584731B68DA88D7F8043175
:1060C0009BB207F58470A0F58270006801F098FC1F
:1060D00007F58473A3F582731B683B6107F584732E
:1060E000A3F582731B68B3F850309BB21A463B6924
:1060F00013443B6107F58473A3F584731B681B7815
:10610000DA003B69134403F20243FB60D7F8043121
:106110009AB2FB681A8000F01FBE07F58473A3F5DE
:1061200084731B68DB78022B40F0628407F584736C
:10613000A3F584731B681A6A07F58473A3F5847347
:106140001B681B699A4240F2DF8307F58473A3F54D
:1061500082731A6807F58473A3F584731B681B7830
:106160009B0013441B889BB223F4E04323F070038D
:10617000A7F8563007F58473A3F582731A6807F5FC
:106180008473A3F584731B681B789B001A44B7F8CB
:10619000563043F07F4343F47F0343F4014343F01D
:1061A00080039BB2138007F58473A3F584731B6887
:1061B0001A6AD7F80431D21A07F58473A3F58473E9
:1061C0001B681A6207F58473A3F582731A6807F5D2
:1061D0008473A3F584731B681B789B0013441B888E
:1061E0009BB203F04003002B00F0C78107F58473D6
:1061F000A3F582731B683B6307F58473A3F584736F
:106200001B685B78002B77D107F58473A3F5827345
:106210001B68BB6207F58473A3F582731B68B3F830
:1062200050309BB21A46BB6A1344BB6207F58473B5
:10623000A3F584731B681B78DA00BB6A134403F26E
:1062400006437B627B6A1B889BB2C3F309039AB245
:106250007B6A1A80D7F804313E2B21D9D7F8043154
:106260005B09C7F80031D7F8043103F01F03002B96
:1062700004D1D7F80031013BC7F800317B6A1B8895
:106280009AB2D7F800319BB29B029BB213439BB2E8
:106290006FEA43436FEA53439AB27B6A1A8050E035
:1062A000D7F80431002B0AD17B6A1B889BB26FEAB6
:1062B00043436FEA53439AB27B6A1A8041E0D7F8AE
:1062C00004315B08C7F80031D7F8043103F001034B
:1062D000002B04D0D7F800310133C7F800317B6AB6
:1062E0001B889AB2D7F800319BB29B029BB2134332
:1062F0009AB27B6A1A8024E007F58473A3F584734D
:106300001B685B78012B1CD107F58473A3F582739E
:106310001B68B3F850309BB21A463B6B13443B6387
:1063200007F58473A3F584731B681B78DA003B6B55
:10633000134403F20643FB62D7F804319AB2FB6AB6
:106340001A8007F58473A3F584731B685B89A7F82B
:10635000763007F58473A3F584731B685969D7F801
:1063600004319BB2B7F8762007F58470A0F58270EF
:10637000006801F045FB07F58473A3F584731B687F
:106380005A69D7F804311A4407F58473A3F5847366
:106390001B685A6107F58473A3F584731B681A6A36
:1063A00007F58473A3F584731B681B699A420FD9A0
:1063B00007F58473A3F584731B681A6AD7F8043150
:1063C000D21A07F58473A3F584731B681A620EE072
:1063D00007F58473A3F584731B681B6AC7F804313F
:1063E00007F58473A3F584731B6800221A6207F50E
:1063F0008473A3F584731B685B78002B77D107F552
:106400008473A3F582731B68BB6107F58473A3F5DE
:1064100082731B68B3F850309BB21A46BB691344B1
:10642000BB6107F58473A3F584731B681B78DA00DE
:10643000BB69134403F202437B617B691B889BB2F7
:10644000C3F309039AB27B691A80D7F804313E2B53
:1064500021D9D7F804315B09C7F8FC30D7F80431EB
:1064600003F01F03002B04D1D7F8FC30013BC7F821
:10647000FC307B691B889AB2D7F8FC309BB29B0238
:106480009BB213439BB26FEA43436FEA53439AB202
:106490007B691A8056E0D7F80431002B0AD17B695A
:1064A0001B889BB26FEA43436FEA53439AB27B69FE
:1064B0001A8047E0D7F804315B08C7F8FC30D7F8FA
:1064C000043103F00103002B04D0D7F8FC30013372
:1064D000C7F8FC307B691B889AB2D7F8FC309BB2B6
:1064E0009B029BB213439AB27B691A802AE007F59C
:1064F0008473A3F584731B685B78012B22D107F5A5
:106500008473A3F582731B683B6207F58473A3F55C
:1065100082731B68B3F850309BB21A463B6A13442F
:106520003B6207F58473A3F584731B681B78DA005C
:106530003B6A134403F20243FB61D7F804319AB279
:10654000FB691A8007F58473A3F584731B681B89A4
:10655000A7F8763007F58473A3F584731B6859692F
:10656000D7F804319BB2B7F8762007F58470A0F510
:106570008270006801F044FAEEE307F58473A3F536
:1065800084731B685B78002B77D107F58473A3F5C0
:1065900082731B68BB6407F58473A3F582731B6861
:1065A000B3F850309BB21A46BB6C1344BB6407F57A
:1065B0008473A3F584731B681B78DA00BB6C1344E7
:1065C00003F202437B647B6C1B889BB2C3F3090319
:1065D0009AB27B6C1A80D7F804313E2B21D9D7F8B8
:1065E00004315B09C7F8F830D7F8043103F01F0312
:1065F000002B04D1D7F8F830013BC7F8F8307B6C9A
:106600001B889AB2D7F8F8309BB29B029BB2134317
:106610009BB26FEA43436FEA53439AB27B6C1A8092
:1066200056E0D7F80431002B0AD17B6C1B889BB253
:106630006FEA43436FEA53439AB27B6C1A8047E098
:10664000D7F804315B08C7F8F830D7F8043103F005
:106650000103002B04D0D7F8F8300133C7F8F83025
:106660007B6C1B889AB2D7F8F8309BB29B029BB226
:1066700013439AB27B6C1A802AE007F58473A3F562
:1066800084731B685B78012B22D107F58473A3F513
:1066900082731B683B6507F58473A3F582731B68DF
:1066A000B3F850309BB21A463B6D13443B6507F577
:1066B0008473A3F584731B681B78DA003B6D134465
:1066C00003F20243FB64D7F804319AB2FB6C1A80E0
:1066D00007F58473A3F584731B681B89A7F87630CC
:1066E00007F58473A3F584731B685969D7F80431DF
:1066F0009BB2B7F8762007F58470A0F58270006829
:1067000001F07EF907F58473A3F584731B685A6959
:10671000D7F804311A4407F58473A3F584731B6812
:106720005A6107F58473A3F584731B681A6A07F529
:106730008473A3F584731B681B699A420FD907F50C
:106740008473A3F584731B681A6AD7F80431D21ACC
:1067500007F58473A3F584731B681A620EE007F5CE
:106760008473A3F584731B681B6AC7F8043107F5AB
:106770008473A3F584731B6800221A6207F584737F
:10678000A3F582731B683B6407F58473A3F58473D8
:106790001B685B78002B77D107F58473A3F58273B0
:1067A0001B68BB6307F58473A3F582731B68B3F89A
:1067B00050309BB21A46BB6B1344BB6307F584731E
:1067C000A3F584731B681B78DA00BB6B134403F2D8
:1067D00006437B637B6B1B889BB2C3F309039AB2AE
:1067E0007B6B1A80D7F804313E2B21D9D7F80431BE
:1067F0005B09C7F8F430D7F8043103F01F03002B0E
:1068000004D1D7F8F430013BC7F8F4307B6B1B8818
:106810009AB2D7F8F4309BB29B029BB213439BB25F
:106820006FEA43436FEA53439AB27B6B1A8050E09E
:10683000D7F80431002B0AD17B6B1B889BB26FEA1F
:1068400043436FEA53439AB27B6B1A8041E0D7F817
:1068500004315B08C7F8F430D7F8043103F00103C2
:10686000002B04D0D7F8F4300133C7F8F4307B6B39
:106870001B889AB2D7F8F4309BB29B029BB21343A9
:106880009AB27B6B1A8024E007F58473A3F58473B6
:106890001B685B78012B1CD107F58473A3F5827309
:1068A0001B68B3F850309BB21A463B6C13443B64F0
:1068B00007F58473A3F584731B681B78DA003B6CBF
:1068C000134403F20643FB63D7F804319AB2FB6B1F
:1068D0001A8007F58473A3F584731B685B89A7F896
:1068E000763007F58473A3F584731B685969D7F86C
:1068F00004319BB2B7F8762007F58470A0F582705A
:10690000006801F07DF827E207F58473A3F584732E
:106910001B681B6AC7F8043107F58473A3F58273FB
:106920001A6807F58473A3F584731B681B789B00B2
:1069300013441B889BB223F4E24323F07003A7F8AF
:10694000623007F58473A3F582731A6807F58473C0
:10695000A3F584731B681B789B001A44B7F8623058
:1069600043F07F4343F47F0343F4004343F0800349
:106970009BB2138007F58473A3F582731B68FB65D4
:1069800007F58473A3F582731B68B3F850309BB28C
:106990001A46FB6D1344FB6507F58473A3F58473F6
:1069A0001B681B78DA00FB6D134403F20243BB65DE
:1069B000D7F804319AB2BB6D1A8007F58473A3F53A
:1069C00084731B681B89A7F8763007F58473A3F5D9
:1069D00084731B685969D7F804319BB2B7F87620E5
:1069E00007F58470A0F58270006801F009F8B3E142
:1069F00007F58473A3F584731B681A6AD7F804310A
:106A0000D21A07F58473A3F584731B681A6207F51D
:106A10008473A3F582731A6807F58473A3F58473EE
:106A20001B681B789B0013441B889BB203F0400338
:106A3000002B00F0C68007F58473A3F582731B68F2
:106A40003B6707F58473A3F584731B685B78002BA1
:106A500077D107F58473A3F582731B68BB6607F5CE
:106A60008473A3F582731B68B3F850309BB21A4647
:106A7000BB6E1344BB6607F58473A3F584731B6870
:106A80001B78DA00BB6E134403F206437B667B6E11
:106A90001B889BB2C3F309039AB27B6E1A80D7F8A6
:106AA00004313E2B21D9D7F804315B09C7F8F03007
:106AB000D7F8043103F01F03002B04D1D7F8F030CE
:106AC000013BC7F8F0307B6E1B889AB2D7F8F030E4
:106AD0009BB29B029BB213439BB26FEA43436FEAA4
:106AE00053439AB27B6E1A8050E0D7F80431002BE2
:106AF0000AD17B6E1B889BB26FEA43436FEA534314
:106B00009AB27B6E1A8041E0D7F804315B08C7F86F
:106B1000F030D7F8043103F00103002B04D0D7F88C
:106B2000F0300133C7F8F0307B6E1B889AB2D7F88B
:106B3000F0309BB29B029BB213439AB27B6E1A80D9
:106B400024E007F58473A3F584731B685B78012B3D
:106B50001CD107F58473A3F582731B68B3F850301A
:106B60009BB21A463B6F13443B6707F58473A3F54A
:106B700084731B681B78DA003B6F134403F20643EF
:106B8000FB66D7F804319AB2FB6E1A8007F584735E
:106B9000A3F584731B685B89A7F8763007F58473C7
:106BA000A3F584731B685969D7F804319BB2B7F811
:106BB000762007F58470A0F58270006800F020FF51
:106BC000CAE007F58473A3F584731B685B78002B18
:106BD00077D107F58473A3F582731B68FB6707F50C
:106BE0008473A3F582731B68B3F850309BB21A46C6
:106BF000FB6F1344FB6707F58473A3F584731B686D
:106C00001B78DA00FB6F134403F20243BB67BB6FD0
:106C10001B889BB2C3F309039AB2BB6F1A80D7F8E3
:106C200004313E2B21D9D7F804315B09C7F8EC3089
:106C3000D7F8043103F01F03002B04D1D7F8EC3050
:106C4000013BC7F8EC30BB6F1B889AB2D7F8EC3029
:106C50009BB29B029BB213439BB26FEA43436FEA22
:106C600053439AB2BB6F1A805CE0D7F80431002B13
:106C70000AD1BB6F1B889BB26FEA43436FEA534351
:106C80009AB2BB6F1A804DE0D7F804315B08C7F8A1
:106C9000EC30D7F8043103F00103002B04D0D7F80F
:106CA000EC300133C7F8EC30BB6F1B889AB2D7F8D1
:106CB000EC309BB29B029BB213439AB2BB6F1A801B
:106CC00030E007F58473A3F584731B685B78012BB0
:106CD00028D107F58473A3F582731B68C7F8843045
:106CE00007F58473A3F582731B68B3F850309BB229
:106CF0001A46D7F884301344C7F8843007F58473F4
:106D0000A3F584731B681B78DA00D7F8843013442A
:106D100003F20243C7F88030D7F804319AB2D7F8AB
:106D200080301A8007F58473A3F584731B681B8970
:106D3000A7F8763007F58473A3F584731B68596947
:106D4000D7F804319BB2B7F8762007F58470A0F528
:106D50008270006800F054FE07F58473A3F5827317
:106D60001A6807F58473A3F584731B681B789B006E
:106D700013441B889BB223F4E04323F040037B8140
:106D80007B8983F010037B817B8983F020037B81E7
:106D900007F58473A3F582731A6807F58473A3F566
:106DA00084731B681B789B001A447B8943F07F43E4
:106DB00043F47F0343F4004343F080039BB213800A
:106DC00000F0DEBC07F58473A3F584731B681B7B9E
:106DD000002B40F0BB8007F58473A3F584731B6818
:106DE0009A6907F58473A3F584731B681B699A423B
:106DF00017D907F58473A3F584731B681B69C7F85B
:106E0000043107F58473A3F584731B689A69D7F876
:106E10000431D21A07F58473A3F584731B689A6151
:106E20000EE007F58473A3F584731B689B69C7F8AC
:106E3000043107F58473A3F584731B6800229A61FB
:106E400007F58473A3F582731B68C7F8903007F5C4
:106E50008473A3F582731B68B3F850309BB21A4653
:106E6000D7F890301344C7F8903007F58473A3F532
:106E700084731B681B78DA00D7F89030134403F250
:106E80000643C7F88C30D7F88C301B889BB2C3F30D
:106E900009039AB2D7F88C301A80D7F804313E2B08
:106EA00024D9D7F804315B09C7F8E830D7F80431A2
:106EB00003F01F03002B04D1D7F8E830013BC7F8DB
:106EC000E830D7F88C301B889AB2D7F8E8309BB2FC
:106ED0009B029BB213439BB26FEA43436FEA534357
:106EE0009AB2D7F88C301A8000F010BCD7F8043171
:106EF000002B0CD1D7F88C301B889BB26FEA434330
:106F00006FEA53439AB2D7F88C301A80FEE3D7F871
:106F100004315B08C7F8E830D7F8043103F0010307
:106F2000002B04D0D7F8E8300133C7F8E830D7F8A1
:106F30008C301B889AB2D7F8E8309BB29B029BB288
:106F400013439AB2D7F88C301A80DFE307F58473C5
:106F5000A3F584731B68DB78022B40F0188207F5D9
:106F60008473A3F584731B685B78002B40F09D80CD
:106F700007F58473A3F582731B68C7F8AC3007F577
:106F80008473A3F582731B68B3F850309BB21A4622
:106F9000D7F8AC301344C7F8AC3007F58473A3F5C9
:106FA00084731B681B78DA00D7F8AC30134403F203
:106FB0000243C7F8A830D7F8A8301B889BB2C3F3A8
:106FC00009039AB2D7F8A8301A8007F58473A3F59D
:106FD00084731B681B693E2B2BD907F58473A3F5BB
:106FE00084731B681B695B09C7F8E43007F5847379
:106FF000A3F584731B681B6903F01F03002B04D1E6
:10700000D7F8E430013BC7F8E430D7F8A8301B8844
:107010009AB2D7F8E4309BB29B029BB213439BB267
:107020006FEA43436FEA53439AB2D7F8A8301A8005
:1070300070E007F58473A3F584731B681B69002B4C
:107040000CD1D7F8A8301B889BB26FEA43436FEA94
:1070500053439AB2D7F8A8301A805BE007F58473DF
:10706000A3F584731B681B695B08C7F8E43007F558
:107070008473A3F584731B681B6903F00103002B61
:1070800004D0D7F8E4300133C7F8E430D7F8A8309B
:107090001B889AB2D7F8E4309BB29B029BB2134391
:1070A0009AB2D7F8A8301A8034E007F58473A3F5B4
:1070B00084731B685B78012B2CD107F58473A3F5CF
:1070C00082731B68C7F8B43007F58473A3F5827325
:1070D0001B68B3F850309BB21A46D7F8B43013444B
:1070E000C7F8B43007F58473A3F584731B681B7865
:1070F000DA00D7F8B430134403F20243C7F8B030D3
:1071000007F58473A3F584731B681B699AB2D7F8DB
:10711000B0301A8007F58473A3F582731B68C7F833
:10712000A43007F58473A3F584731B685B78002B88
:1071300040F09D8007F58473A3F582731B68C7F840
:107140009C3007F58473A3F582731B68B3F8503045
:107150009BB21A46D7F89C301344C7F89C3007F509
:107160008473A3F584731B681B78DA00D7F89C300E
:10717000134403F20643C7F89830D7F898301B88B9
:107180009BB2C3F309039AB2D7F898301A8007F577
:107190008473A3F584731B681B693E2B2BD907F5F9
:1071A0008473A3F584731B681B695B09C7F8E0301F
:1071B00007F58473A3F584731B681B6903F01F0331
:1071C000002B04D1D7F8E030013BC7F8E030D7F806
:1071D00098301B889AB2D7F8E0309BB29B029BB2E2
:1071E00013439BB26FEA43436FEA53439AB2D7F813
:1071F00098301A8069E007F58473A3F584731B68DF
:107200001B69002B0CD1D7F898301B889BB26FEA12
:1072100043436FEA53439AB2D7F898301A8054E048
:1072200007F58473A3F584731B681B695B08C7F8B3
:10723000E03007F58473A3F584731B681B6903F0C2
:107240000103002B04D0D7F8E0300133C7F8E03059
:10725000D7F898301B889AB2D7F8E0309BB29B02DF
:107260009BB213439AB2D7F898301A802DE007F5F5
:107270008473A3F584731B685B78012B25D107F514
:107280008473A3F582731B68B3F850309BB21A461F
:10729000D7F8A4301344C7F8A43007F58473A3F5D6
:1072A00084731B681B78DA00D7F8A430134403F208
:1072B0000643C7F8A03007F58473A3F584731B68F1
:1072C0001B699AB2D7F8A0301A8007F58473A3F52A
:1072D00084731B68DB69002B00F0188207F5847348
:1072E000A3F582731A6807F58473A3F584731B688A
:1072F0001B789B0013441B88A7F89630B7F896308C
:1073000003F48043002B05D0B7F8963003F0400318
:10731000002B0DD1B7F8963003F48043002B40F0DA
:10732000F581B7F8963003F04003002B40F0EE8172
:1073300007F58473A3F582731A6807F58473A3F5C0
:1073400084731B681B789B0013441B889BB223F437
:10735000E04323F07003A7F8943007F58473A3F596
:1073600082731A6807F58473A3F584731B681B780E
:107370009B001A44B7F8943043F07F4343F47F03F3
:1073800043F4004343F0C0039BB21380BEE107F512
:107390008473A3F584731B68DB78012B40F0B48100
:1073A00007F58473A3F584731B689A6907F58473E2
:1073B000A3F584731B681B699A4217D907F5847378
:1073C000A3F584731B681B69C7F8043107F5847340
:1073D000A3F584731B689A69D7F80431D21A07F5AC
:1073E0008473A3F584731B689A610EE007F58473B8
:1073F000A3F584731B689B69C7F8043107F5847390
:10740000A3F584731B6800229A6107F58473A3F5C2
:1074100084731B685B78002B40F0858007F58473CC
:10742000A3F582731B68C7F8CC3007F58473A3F506
:1074300082731B68B3F850309BB21A46D7F8CC3031
:107440001344C7F8CC3007F58473A3F584731B6825
:107450001B78DA00D7F8CC30134403F20243C7F8A4
:10746000C830D7F8C8301B889BB2C3F309039AB25F
:10747000D7F8C8301A80D7F804313E2B23D9D7F873
:1074800004315B09C7F8DC30D7F8043103F01F037F
:10749000002B04D1D7F8DC30013BC7F8DC30D7F83B
:1074A000C8301B889AB2D7F8DC309BB29B029BB2E3
:1074B00013439BB26FEA43436FEA53439AB2D7F840
:1074C000C8301A8060E0D7F80431002B0CD1D7F80F
:1074D000C8301B889BB26FEA43436FEA53439AB2AA
:1074E000D7F8C8301A804FE0D7F804315B08C7F8E6
:1074F000DC30D7F8043103F00103002B04D0D7F8B7
:10750000DC300133C7F8DC30D7F8C8301B889AB2BA
:10751000D7F8DC309BB29B029BB213439AB2D7F8E8
:10752000C8301A8030E007F58473A3F584731B68B4
:107530005B78012B28D107F58473A3F582731B6850
:10754000C7F8D43007F58473A3F582731B68B3F8CA
:1075500050309BB21A46D7F8D4301344C7F8D43011
:1075600007F58473A3F584731B681B78DA00D7F8DA
:10757000D430134403F20243C7F8D030D7F80431B3
:107580009AB2D7F8D0301A8007F58473A3F58273C6
:107590001B68C7F8C43007F58473A3F584731B68B0
:1075A0005B78002B40F0858007F58473A3F5827328
:1075B0001B68C7F8BC3007F58473A3F582731B689A
:1075C000B3F850309BB21A46D7F8BC301344C7F812
:1075D000BC3007F58473A3F584731B681B78DA004D
:1075E000D7F8BC30134403F20643C7F8B830D7F8D5
:1075F000B8301B889BB2C3F309039AB2D7F8B830EE
:107600001A80D7F804313E2B23D9D7F804315B090F
:10761000C7F8D830D7F8043103F01F03002B04D18A
:10762000D7F8D830013BC7F8D830D7F8B8301B8826
:107630009AB2D7F8D8309BB29B029BB213439BB24D
:107640006FEA43436FEA53439AB2D7F8B8301A80CF
:107650005CE0D7F80431002B0CD1D7F8B8301B8888
:107660009BB26FEA43436FEA53439AB2D7F8B830FC
:107670001A804BE0D7F804315B08C7F8D830D7F848
:10768000043103F00103002B04D0D7F8D8300133C4
:10769000C7F8D830D7F8B8301B889AB2D7F8D830A6
:1076A0009BB29B029BB213439AB2D7F8B8301A80B0
:1076B0002CE007F58473A3F584731B685B78012BBA
:1076C00024D107F58473A3F582731B68B3F8503097
:1076D0009BB21A46D7F8C4301344C7F8C43007F534
:1076E0008473A3F584731B681B78DA00D7F8C43061
:1076F000134403F20643C7F8C030D7F804319AB2F6
:10770000D7F8C0301A8001E001233AE007F584730E
:10771000A3F582731A6807F58473A3F584731B6855
:107720001B789B0013441B889BB223F4804323F0F7
:107730007003A7F88A30B7F88A3083F48053A7F82B
:107740008A30B7F88A3083F40053A7F88A3007F5F7
:107750008473A3F582731A6807F58473A3F58473A1
:107760001B681B789B001A44B7F88A3043F07F43AC
:1077700043F47F0343F4004343F080039BB2138040
:107780000023184607F58477BD4680BD80B485B0D8
:1077900000AF786039603B685B78002B20D07A6856
:1077A0003B681B789B0013441B889BB223F4E04387
:1077B00023F04003BB81BB8983F01003BB817A684F
:1077C0003B681B789B001A44BB8943F07F4343F41A
:1077D0007F0343F4004343F080039BB213801FE018
:1077E0007A683B681B789B0013441B889BB223F488
:1077F000804323F07003FB81FB8983F48053FB817A
:107800007A683B681B789B001A44FB8943F07F43EE
:1078100043F47F0343F4004343F080039BB213809F
:10782000002318461437BD465DF8047B704780B4CA
:1078300087B000AF786039603B681B7B002B40F05D
:107840009D803B685B78002B4CD07A683B681B7846
:107850009B0013441B883B823B8A03F04003002BB0
:107860001BD07A683B681B789B0013441B889BB233
:1078700023F4E04323F07003FB817A683B681B78B4
:107880009B001A44FB8943F07F4343F47F0343F496
:10789000004343F0C0039BB213803B68DB78012BAD
:1078A0006CD07A683B681B789B0013441B889BB2A2
:1078B00023F4E04323F04003BB81BB8983F0200322
:1078C000BB817A683B681B789B001A44BB8943F0F4
:1078D0007F4343F47F0343F4004343F080039BB2B0
:1078E00013804BE07A683B681B789B0013441B882D
:1078F000FB82FB8A03F48043002B1BD07A683B6831
:107900001B789B0013441B889BB223F4E04323F0B5
:107910007003BB827A683B681B789B001A44BB8A61
:1079200043F07F4343F47F0343F4404343F0800339
:107930009BB213807A683B681B789B0013441B88BA
:107940009BB223F4804323F070037B827B8A83F411
:1079500080537B827B8A83F400537B827A683B6806
:107960001B789B001A447B8A43F07F4343F47F03D8
:1079700043F4004343F080039BB213800023184676
:107980001C37BD465DF8047B704780B483B000AF00
:1079900078600B46FB70FB78002B03D17B6880225C
:1079A000A3F84C20002318460C37BD465DF8047B35
:1079B000704780B483B000AF78607B68B3F858300C
:1079C0009BB26FEA43436FEA53439AB27B68A3F8D2
:1079D0005820002318460C37BD465DF8047B7047DD
:1079E00080B485B000AF78607B68B3F844309BB258
:1079F000FB60FB6818461437BD465DF8047B704792
:107A000080B48BB000AFF860B96011461A460B46DF
:107A1000FB801346BB80BB8801335B08BB61FB68FE
:107A20007B61BB68FB61FA887B69134403F5806363
:107A30003B62BB697B621BE0FB691B787B82FB6955
:107A400001331B781B021AB2B7F9123013431BB271
:107A50007B823B6A7A8A1A803B6A02333B62FB690B
:107A60000133FB61FB690133FB617B6A013B7B6294
:107A70007B6A002BE0D100BF00BF2C37BD465DF80C
:107A8000047B704780B48BB000AFF860B9601146DA
:107A90001A460B46FB801346BB80BB885B089BB233
:107AA000BB61FB687B61BB68FB61FA887B6913443F
:107AB00003F580633B62BB697B6218E03B6A1B880D
:107AC0009BB23B613B6A02333B623B69DAB2FB69C2
:107AD0001A70FB690133FB613B691B0ADAB2FB696F
:107AE0001A70FB690133FB617B6A013B7B627B6A35
:107AF000002BE3D1BB8803F001039BB2002B07D01E
:107B00003B6A1B889BB23B613B69DAB2FB691A7026
:107B100000BF2C37BD465DF8047B704780B582B04E
:107B200000AF0023FB71032002F04AF80F2000F0A1
:107B30000DF80346002B02D00123FB7101E0FBF797
:107B400001FAFB7918460837BD4680BD80B584B080
:107B500000AF78600023FB73164B1B68002B22D00C
:107B6000154B1A68134B1B684FF47A71B1FBF3F392
:107B7000B2FBF3F3184602F056F80346002B0FD180
:107B80007B680F2B09D8002279684FF0FF3002F094
:107B900022F80A4A7B68136007E00123FB7304E0C4
:107BA0000123FB7301E00123FB73FB7B18461037B5
:107BB000BD4680BDC8000020EC000020C4000020AD
:107BC00080B400AF054B1A68054B1B681344034A89
:107BD000136000BFBD465DF8047B7047502C002049
:107BE000C800002080B400AF034B1B681846BD4698
:107BF0005DF8047B704700BF502C002080B584B036
:107C000000AF7860FFF7EEFFB8607B68FB60FB6851
:107C1000B3F1FF3F04D0094B1B68FA681344FB60C3
:107C200000BFFFF7DFFF0246BB68D31AFA689A422B
:107C3000F7D800BF00BF1037BD4680BDC800002088
:107C400080B588B000AF78607B68002B01D101233C
:107C5000FEE27B681B6803F00103002B75D0974B95
:107C60009B6803F00C03BB61944BDB6803F00303D8
:107C70007B61BB690C2B02D17B69032B02D0BB69F2
:107C8000082B0BD18D4B1B6803F40033002B5BD00A
:107C90007B685B68002B57D10123D9E27B685B6866
:107CA000B3F5803F06D1854B1B68844A43F480338B
:107CB00013601DE07B685B68B3F5A02F0CD17F4B90
:107CC0001B687E4A43F4802313607C4B1B687B4A0D
:107CD00043F4803313600BE0784B1B68774A23F43E
:107CE00080331360754B1B68744A23F48023136040
:107CF0007B685B68002B13D0FFF774FF386108E0E6
:107D0000FFF770FF02463B69D31A642B01D90323A6
:107D10009EE26A4B1B6803F40033002BF0D014E0A2
:107D2000FFF760FF386108E0FFF75CFF02463B6940
:107D3000D31A642B01D903238AE2604B1B6803F436
:107D40000033002BF0D100E000BF7B681B6803F01C
:107D50000203002B75D0594B9B6803F00C03BB61E9
:107D6000564BDB6803F003037B61BB690C2B02D12C
:107D70007B69022B02D0BB69042B1FD14F4B1B68C0
:107D800003F48063002B05D07B68DB68002B01D1F6
:107D900001235DE2494B5B6823F0FE427B681B696F
:107DA0001B06464913434B60454B1B681846FFF7BB
:107DB000CDFE0346002B43D0012349E27B68DB68FC
:107DC000002B23D03D4B1B683C4A43F48073136067
:107DD000FFF708FF386108E0FFF704FF02463B6940
:107DE000D31A022B01D9032332E2344B1B6803F46C
:107DF0008063002BF0D0314B5B6823F0FE427B6840
:107E00001B691B062D4913434B601AE02B4B1B6863
:107E10002A4A23F480731360FFF7E4FE386108E018
:107E2000FFF7E0FE02463B69D31A022B01D9032378
:107E30000EE2224B1B6803F48063002BF0D100E0BC
:107E400000BF7B681B6803F00803002B41D07B68F0
:107E50005B69002B1CD0194BD3F89430174A43F0C0
:107E60000103C2F89430FFF7BDFE386108E0FFF768
:107E7000B9FE02463B69D31A022B01D90323E7E17D
:107E80000E4BD3F8943003F00203002BEFD020E028
:107E90000A4BD3F89430094A23F00103C2F8943016
:107EA000FFF7A0FE38610DE0FFF79CFE02463B693C
:107EB000D31A022B06D90323CAE100BF00100240E7
:107EC000C40000208C4BD3F8943003F00203002B45
:107ED000EAD17B681B6803F00403002B00F0A68046
:107EE0000023FB77844B9B6D03F08053002B01D163
:107EF000012300E00023002B0DD07F4B9B6D7E4AB9
:107F000043F0805393657C4B9B6D03F08053FB6083
:107F1000FB680123FB77794B1B6803F48073002B0C
:107F200018D1764B1B68754A43F480731360FFF7D2
:107F300059FE386108E0FFF755FE02463B69D31A47
:107F4000022B01D9032383E16C4B1B6803F480737C
:107F5000002BF0D07B689B68012B08D1664BD3F8CF
:107F60009030654A43F00103C2F8903024E07B680A
:107F70009B68052B10D1604BD3F890305E4A43F0DC
:107F80000403C2F890305C4BD3F890305A4A43F067
:107F90000103C2F890300FE0574BD3F89030564AA7
:107FA00023F00103C2F89030534BD3F89030524A7B
:107FB00023F00403C2F890307B689B68002B16D036
:107FC000FFF710FE38610AE0FFF70CFE02463B693E
:107FD000D31A41F28832934201D9032338E1464B48
:107FE000D3F8903003F00203002BEDD015E0FFF73B
:107FF000F9FD38610AE0FFF7F5FD02463B69D31A47
:1080000041F28832934201D9032321E13A4BD3F85C
:10801000903003F00203002BEDD1FB7F012B05D143
:10802000354B9B6D344A23F0805393657B681B6806
:1080300003F02003002B3CD07B689B69002B1CD0F5
:108040002D4BD3F898302C4A43F00103C2F89830F6
:10805000FFF7C8FD386108E0FFF7C4FD02463B6941
:10806000D31A022B01D90323F2E0234BD3F8983023
:1080700003F00203002BEFD01BE01F4BD3F8983026
:108080001D4A23F00103C2F89830FFF7ABFD3861B9
:1080900008E0FFF7A7FD02463B69D31A022B01D97E
:1080A0000323D5E0144BD3F8983003F00203002BE0
:1080B000EFD17B68DB69002B00F0C9800E4B9B6819
:1080C00003F00C030C2B00F083807B68DB69022B30
:1080D0005ED1094B1B68084A23F080731360FFF7D9
:1080E00081FD38610CE0FFF77DFD02463B69D31A44
:1080F000022B05D90323ABE00010024000700040C2
:10810000554B1B6803F00073002BECD1524BDA681F
:10811000524B13407A68116A7A68526A013A120126
:1081200011437A68926A120211437A68126B5208FC
:10813000013A520511437A68526B5208013A5206CD
:1081400011437A68D26AD2060A4343491343CB608B
:10815000414B1B68404A43F0807313603E4BDB6821
:108160003D4A43F08073D360FFF73CFD386108E07F
:10817000FFF738FD02463B69D31A022B01D90323CE
:1081800066E0354B1B6803F00073002BF0D05EE017
:10819000314B1B68304A23F080731360FFF722FDD8
:1081A000386108E0FFF71EFD02463B69D31A022B37
:1081B00001D903234CE0284B1B6803F00073002B0C
:1081C000F0D1254BDA682449254B1340CB603EE0C3
:1081D0007B68DB69012B01D1012339E01E4BDB6891
:1081E0007B617B6903F003027B681B6A9A422CD196
:1081F0007B6903F0F0027B685B6A013B1B019A42DA
:1082000023D17B6903F4FE427B689B6A1B029A427E
:108210001BD17B6903F078427B68DB6ADB069A42FC
:1082200013D17B6903F4C0027B681B6B5B08013BC5
:108230005B059A4209D17B6903F0C0627B685B6B86
:108240005B08013B5B069A4201D0012300E000235A
:1082500018462037BD4680BD001002400C809F01AB
:10826000FCFFEEFE80B586B000AF78603960002379
:108270007B617B68002B01D101231EE1914B1B68C0
:1082800003F00F033A689A4210D98E4B1B6823F013
:108290000F028C493B6813430B608A4B1B6803F049
:1082A0000F033A689A4201D0012306E17B681B68FC
:1082B00003F00103002B73D07B685B68032B29D18B
:1082C000814B1B6803F00073002B01D10123F4E004
:1082D00000F09CF938613B697C4A93423FD97A4B64
:1082E0009B6803F0F003002B09D07B681B6803F048
:1082F0000203002B33D07B689B68002B2FD1724B7D
:108300009B6823F0F003704A43F08003936080235E
:108310007B6124E07B685B68022B07D16A4B1B689A
:1083200003F40033002B09D10123C6E0664B1B6820
:1083300003F48063002B01D10123BEE000F0CEF8EE
:1083400038613B69614A934209D95F4B9B6823F0CE
:10835000F0035D4A43F08003936080237B615A4BB6
:108360009B6823F003027B685B68574913438B606B
:10837000FFF738FCF8600AE0FFF734FC0246FB68C0
:10838000D31A41F28832934201D9032395E04E4B30
:108390009B6803F00C027B685B689B009A42EBD100
:1083A0007B681B6803F00203002B23D07B681B68EB
:1083B00003F00403002B05D0434B9B68424A43F46F
:1083C000E06393607B681B6803F00803002B07D011
:1083D0003D4B9B6823F47C533B4A43F4E06393603A
:1083E000394B9B6823F0F0027B689B683649134346
:1083F0008B6008E07B69802B05D1334B9B68324A48
:1084000023F0F00393602F4B1B6803F00F033A68CF
:108410009A421DD22B4B1B6823F00F0229493B685F
:1084200013430B60FFF7DEFBF8600AE0FFF7DAFBAF
:108430000246FB68D31A41F28832934201D90323E2
:108440003BE0204B1B6803F00F033A689A42EDD1E2
:108450007B681B6803F00403002B08D01A4B9B6851
:1084600023F4E0627B68DB68174913438B607B6809
:108470001B6803F00803002B09D0134B9B6823F4FF
:1084800060527B681B69DB000F4913438B6000F06F
:1084900025F802460C4B9B681B0903F00F030C499F
:1084A000CB5C03F01F0322FA03F30A4A13600A4B62
:1084B0001B681846FFF74AFB034618461837BD46A7
:1084C00080BD00BF002002400010024000B4C40480
:1084D000140D0208EC000020C400002080B487B016
:1084E00000AF2C4B9B6803F00C03042B02D12A4BEA
:1084F0003B6147E0274B9B6803F00C03082B02D13C
:10850000254B3B613EE0234B9B6803F00C030C2B97
:1085100036D1204BDB6803F00303FB601D4BDB68A7
:108520001B0903F00F030133BB60FB68032B0CD165
:10853000194ABB68B2FBF3F3164AD268120A02F07A
:108540007F0202FB03F37B610CE0134ABB68B2FBC2
:10855000F3F3104AD268120A02F07F0202FB03F31F
:108560007B6100BF0B4BDB685B0E03F00303013341
:108570005B007B607A697B68B2FBF3F33B6101E0EF
:1085800000233B613B6918461C37BD465DF8047B00
:10859000704700BF001002400024F40080B400AF18
:1085A000034B1B681846BD465DF8047B704700BF4F
:1085B000EC00002080B500AFFFF7F0FF0246064B4D
:1085C0009B681B0A03F007030449CB5C03F01F03FD
:1085D00022FA03F3184680BD00100240240D020861
:1085E00080B500AFFFF7DAFF0246064B9B68DB0A57
:1085F00003F007030449CB5C03F01F0322FA03F3E3
:10860000184680BD00100240240D020880B487B0D7
:1086100000AF1E4BDB6803F003033B611B4BDB68C1
:108620001B0903F00F030133FB603B69032B0CD1E3
:10863000174AFB68B2FBF3F3144AD268120A02F03D
:108640007F0202FB03F37B610CE0114AFB68B2FB83
:10865000F3F30E4AD268120A02F07F0202FB03F320
:108660007B6100BF094BDB685B0E03F00303013342
:108670005B00BB607A69BB68B2FBF3F37B607B682D
:1086800018461C37BD465DF8047B70470010024059
:108690000024F40080B586B000AF78600023FB743E
:1086A0000023BB747B681B6803F40023002B00F0DD
:1086B000988000237B74434B9B6D03F08053002B09
:1086C0000DD1404B9B6D3F4A43F0805393653D4B2A
:1086D0009B6D03F08053BB60BB6801237B743A4BF6
:1086E0001B68394A43F480731360FFF77BFAF86024
:1086F00009E0FFF777FA0246FB68D31A022B02D98A
:108700000323FB7405E0304B1B6803F48073002BDC
:10871000EFD0FB7C002B59D12A4BD3F8903003F4D7
:1087200040737B617B69002B1ED07B681B6D7A696F
:108730009A4219D0234BD3F8903023F440737B61D5
:10874000204BD3F890301F4A43F48033C2F8903066
:108750001C4BD3F890301B4A23F48033C2F890307E
:10876000184A7B69C2F890307B6903F00103002B43
:1087700016D0FFF737FAF8600BE0FFF733FA02463E
:10878000FB68D31A41F28832934202D90323FB7467
:1087900006E00C4BD3F8903003F00203002BECD032
:1087A000FB7C002B0BD1074BD3F8903023F44072A5
:1087B0007B681B6D03491343C1F8903008E0FB7CD4
:1087C000BB7405E00010024000700040FB7CBB74ED
:1087D0007B7C012B05D1A74B9B6DA64A23F08053D0
:1087E00093657B681B6803F00103002B0AD0A14B43
:1087F000D3F8883023F003027B685B689D491343FC
:10880000C1F888307B681B6803F00203002B0AD094
:10881000984BD3F8883023F00C027B689B6895490D
:108820001343C1F888307B681B6803F00403002BF6
:108830000AD0904BD3F8883023F030027B68DB6895
:108840008C491343C1F888307B681B6803F0080328
:10885000002B0AD0874BD3F8883023F0C0027B6806
:108860001B6984491343C1F888307B681B6803F097
:108870001003002B0AD07F4BD3F8883023F44072CA
:108880007B685B697B491343C1F888307B681B6850
:1088900003F02003002B0AD0764BD3F8883023F462
:1088A00040627B689B6973491343C1F888307B68D9
:1088B0001B6803F04003002B0AD06E4BD3F88830BE
:1088C00023F440527B68DB696A491343C1F888305E
:1088D0007B681B6803F08003002B0AD0654BD3F83C
:1088E000883023F440427B681B6A62491343C1F815
:1088F00088307B681B6803F48073002B0AD05D4BC3
:10890000D3F8883023F440327B685B6A59491343BB
:10891000C1F888307B681B6803F40033002B0AD051
:10892000544BD3F89C3023F003027B689B6A514977
:108930001343C1F89C307B681B6803F40073002B61
:108940000AD04C4BD3F8883023F440227B68DB6A92
:1089500048491343C1F888307B681B6803F480637F
:10896000002B15D0434BD3F8883023F440127B689A
:108970001B6B40491343C1F888307B681B6BB3F510
:10898000801F05D13B4BDB683A4A43F48013D36028
:108990007B681B6803F40063002B15D0354BD3F8BC
:1089A000883023F440027B685B6B32491343C1F883
:1089B00088307B685B6BB3F5800F05D12D4BDB688E
:1089C0002C4A43F48013D3607B681B6803F4805304
:1089D000002B15D0274BD3F8883023F040727B68EA
:1089E0009B6B24491343C1F888307B689B6BB3F1C0
:1089F000807F05D11F4BDB681E4A43F48013D36090
:108A00007B681B6803F40053002B15D0194BD3F877
:108A1000883023F040627B68DB6B16491343C1F852
:108A200088307B68DB6BB3F1006F05D1114BDB68DD
:108A3000104A43F48013D3607B681B6803F48043BF
:108A4000002B19D00B4BD3F8883023F040627B68A1
:108A50001B6C08491343C1F888307B681B6CB3F169
:108A6000006F09D1034BDB68024A43F48013D360E3
:108A700002E000BF001002407B681B6803F4004363
:108A8000002B15D0294BD3F8883023F040527B6857
:108A90005B6C26491343C1F888307B685B6CB3F18B
:108AA000805F05D1214BDB68204A43F48033D360DB
:108AB0007B681B6803F48033002B15D01B4BD3F865
:108AC000883023F040427B689B6C18491343C1F8FF
:108AD00088307B689B6CB3F1804F05D1134BDB680A
:108AE000124A43F48033D3607B681B6803F480230D
:108AF000002B15D00D4BD3F89C3023F440127B682B
:108B0000DB6C0A491343C1F89C307B68DB6CB3F51E
:108B1000001F05D1054BDB68044A43F48013D36082
:108B2000BB7C18461837BD4680BD00BF0010024010
:108B300080B586B000AFF860B960C7E900230023B4
:108B40003B612F4B1B78012B01D1022353E02C4BAF
:108B500001221A704FF47A7000F092F80346FB7508
:108B6000FB7D002B43D1264B00225A60254B1B680E
:108B700003F48063002B09D0224B1B68214A23F4A5
:108B8000806313601E4B02221A7702E01C4B002206
:108B90001A77FB68002B07D1D7E90023B86800F0EB
:108BA000C1F801233B6110E0FB68012B02D0FB6898
:108BB000022B0AD13B681946B86800F0D9F8FB6867
:108BC000022B02D14FF480233B614FF47A7000F006
:108BD00057F80346FB753B69002B06D0094B5A69D1
:108BE0003B69DB43074913404B6100F00FFA044B2C
:108BF00000221A70FB7D18461837BD4680BD00BFA5
:108C0000CC0000200020024080B483B000AF0023DD
:108C1000FB710B4B5B69002B0BDA094B094A9A601D
:108C2000074B094A9A60064B5B69002B01DA012366
:108C3000FB71FB7918460C37BD465DF8047B704725
:108C40000020024023016745AB89EFCD80B483B09B
:108C500000AF0123FB71094B5B69084A43F00043F5
:108C60005361064B5B69002B01DA0023FB71FB7932
:108C700018460C37BD465DF8047B70470020024063
:108C800080B584B000AF7860FEF7ACFFF86009E013
:108C9000FEF7A8FF0246FB68D31A7A689A4201D20F
:108CA000032337E01D4B1B6903F48033B3F5803F8A
:108CB000EED01A4B1A694CF2FA331340BB60BB6812
:108CC000002B1DD0164B5A68BB681343144A5360DF
:108CD000BB68B3F1805F07D3104B9A69BB6803F0A0
:108CE00070430E4913438B61BB6823F07043002B24
:108CF00004D00A4ABB6823F070431361012309E0E2
:108D0000064B1B6903F00103012B02D1034B012227
:108D10001A61002318461037BD4680BD002002406E
:108D2000CC00002080B485B000AFF860C7E9002314
:108D30000E4B5B690D4A43F001035361FB683A68CF
:108D40001A60BFF36F8F00BFD7E900014FF0000238
:108D50004FF000030A000023F968043113460B604A
:108D600000BF1437BD465DF8047B70470020024009
:108D700080B489B000AF786039604023FB777B68AE
:108D8000BB613B687B61144B5B69134A43F48023EE
:108D90005361EFF31083FB60FB683B6172B600BF69
:108DA0007B691A68BB691A60BB690433BB617B6964
:108DB00004337B61FB7F013BFB77FB7F002BEFD113
:108DC0003B69BB60BB6883F3108800BF00BF2437DA
:108DD000BD465DF8047B70470020024080B584B03A
:108DE00000AF78603960494B1B78012B01D1022319
:108DF00087E0464B01221A704FF47A70FFF740FF6C
:108E00000346FB73FB7B002B77D1404B00225A605B
:108E10003F4B1B6803F40073002B13D03C4B1B68C3
:108E200003F48063002B09D0394B1B68384A23F4C4
:108E300080631360354B03221A7716E0334B01220F
:108E40001A7712E0324B1B6803F48063002B09D0C1
:108E50002F4B1B682E4A23F4806313602B4B022296
:108E60001A7702E0294B00221A777B681B68012BD6
:108E700013D17B685B68184600F04CF84FF47A70A9
:108E8000FFF7FEFE0346FB73214B5B69204A23F488
:108E9000004323F0040353612DE03B684FF0FF32A1
:108EA0001A607B689B68BB601DE07B685B68194645
:108EB000B86800F067F84FF47A70FFF7E1FE0346F8
:108EC000FB73134B5B69124A23F47E7323F0020396
:108ED0005361FB7B002B03D03B68BA681A600AE041
:108EE000BB680133BB607B689A687B68DB681344AE
:108EF000BA689A42D9D300F089F8044B00221A705C
:108F0000FB7B18461037BD4680BD00BFCC0000205B
:108F10000020024080B483B000AF7860184B1B6A19
:108F200003F48003002B16D07B6803F00103002BB1
:108F300005D0134B5B69124A43F0040353617B680D
:108F400003F00203002B0ED00D4B5B690C4A43F477
:108F50000043536107E00A4B5B69094A43F400434D
:108F600043F004035361064B5B69054A43F48033C5
:108F7000536100BF0C37BD465DF8047B704700BFEE
:108F80000020024080B483B000AF786039601E4B8F
:108F90001B6A03F48003002B06D11B4B5B691A4A42
:108FA00023F40063536111E03B6803F00103002BDD
:108FB00006D0154B5B69144A23F40063536105E046
:108FC000114B5B69104A43F4006353610E4B5B69BC
:108FD00023F47E727B68DB0003F4FF630A491343CA
:108FE0004B61094B5B69084A43F002035361064B2E
:108FF0005B69054A43F48033536100BF0C37BD46BB
:109000005DF8047B704700BF0020024080B483B04D
:1090100000AF214B1B7FFB71FB79012B02D0FB7949
:10902000032B17D11D4B1B681C4A23F400731360DC
:109030001A4B1B68194A43F400631360174B1B68F3
:10904000164A23F400631360144B1B68134A43F45D
:1090500000731360FB79022B02D0FB79032B11D133
:109060000E4B1B680D4A43F4805313600B4B1B6877
:109070000A4A23F480531360084B1B68074A43F4E1
:1090800080631360044B00221A7700BF0C37BD4683
:109090005DF8047B704700BFCC0000200020024038
:1090A00080B487B000AF7860396000237B615AE1FB
:1090B0003B681A6801217B6901FA03F31340FB60E6
:1090C000FB68002B00F04C813B685B6803F00303F6
:1090D000012B05D03B685B6803F00303022B30D102
:1090E0007B689B683B617B695B00032202FA03F3A8
:1090F000DB433A6913403B613B68DA687B695B009C
:1091000002FA03F33A6913433B617B683A699A6058
:109110007B685B683B6101227B6902FA03F3DB43F6
:109120003A6913403B613B685B681B0903F001022D
:109130007B6902FA03F33A6913433B617B683A693E
:109140005A603B685B6803F00303032B17D07B680E
:10915000DB683B617B695B00032202FA03F3DB43BC
:109160003A6913403B613B689A687B695B0002FA8D
:1091700003F33A6913433B617B683A69DA603B6801
:109180005B6803F00303022B23D17B69DA087B6859
:10919000083253F822303B617B6903F007039B00E0
:1091A0000F2202FA03F3DB433A6913403B613B6849
:1091B0001A697B6903F007039B0002FA03F33A691B
:1091C00013433B617B69DA087B680832396943F8ED
:1091D00022107B681B683B617B695B00032202FAFB
:1091E00003F3DB433A6913403B613B685B6803F080
:1091F00003027B695B0002FA03F33A6913433B61A4
:109200007B683A691A603B685B6803F44033002B63
:1092100000F0A6805B4B1B6E5A4A43F001031366B5
:10922000584B1B6E03F00103BB60BB68564A7B6959
:109230009B08023352F823303B617B6903F0030340
:109240009B000F2202FA03F3DB433A6913403B61B0
:109250007B68B3F1904F1FD07B684C4A934219D082
:109260007B684B4A934213D07B684A4A93420DD0A5
:109270007B68494A934207D07B68484A934201D1B0
:1092800005230AE0062308E0042306E0032304E0A4
:10929000022302E0012300E000237A6902F00302C6
:1092A000920093403A6913433B6137497B699B08BD
:1092B00002333A6941F82320394B9B683B61FB68D4
:1092C000DB433A6913403B613B685B6803F48013FE
:1092D000002B03D03A69FB6813433B61304A3B697A
:1092E00093602F4BDB683B61FB68DB433A691340BB
:1092F0003B613B685B6803F40013002B03D03A69C1
:10930000FB6813433B61264A3B69D360244B5B688F
:109310003B61FB68DB433A6913403B613B685B6838
:1093200003F40033002B03D03A69FB6813433B611D
:109330001B4A3B6953601A4B1B683B61FB68DB436C
:109340003A6913403B613B685B6803F48033002B50
:1093500003D03A69FB6813433B61114A3B691360D0
:109360007B6901337B613B681A687B6922FA03F3EE
:10937000002B7FF49DAE00BF00BF1C37BD465DF8DB
:10938000047B7047001002400000014000040048C8
:1093900000080048000C0048001000480014004875
:1093A0000004014080B485B000AF78600B467B803C
:1093B0007B681A697B881340002B02D00123FB7362
:1093C00001E00023FB73FB7B18461437BD465DF8B4
:1093D000047B704780B584B000AF78607B68002B59
:1093E00001D101238DE07B681B681A46474B9A42E6
:1093F0000FD87B681B681A46454B1344454AA2FBAD
:1094000003231B099A007B685A647B68424A1A64EA
:109410000EE07B681B681A46404B13443D4AA2FB92
:1094200003231B099A007B685A647B683C4A1A64D0
:109430007B68022283F825207B681B681B68FB6021
:10944000FB6823F4FF4323F07003FB607B689A689A
:109450007B68DB681A437B681B691A437B685B691E
:109460001A437B689B691A437B68DB691A437B68F4
:109470001B6A1343FA681343FB607B681B68FA6836
:109480001A60786800F0B6F97B689B68B3F5804F86
:1094900002D17B6800225A607B685A687B689B6CAB
:1094A000D2B21A607B68DB6C7A68126D5A607B6896
:1094B0005B68002B10D07B685B68042B0CD8786845
:1094C00000F0D6F97B685B6D00221A607B689B6DAB
:1094D0007A68D26D5A6008E07B6800225A657B6822
:1094E00000229A657B680022DA657B680022DA63D5
:1094F0007B68012283F825207B68002283F82420E2
:10950000002318461037BD4680BD00BF0704024047
:10951000F8FFFDBFCDCCCCCC00000240F8FBFDBF76
:109520000004024080B586B000AFF860B9607A6090
:109530003B600023FB75FB6893F82430012B01D1BD
:10954000022366E0FB68012283F82420FB6893F87D
:109550002530DBB2012B55D1FB68022283F8252090
:10956000FB680022DA63FB681B681A68FB681B68EB
:1095700022F001021A603B687A68B968F86800F066
:10958000FBF8FB681B6B002B08D0FB681B681A6894
:10959000FB681B6842F00E021A600FE0FB681B6854
:1095A0001A68FB681B6822F004021A60FB681B68DB
:1095B0001A68FB681B6842F00A021A60FB689B6C21
:1095C0001B6803F48033002B07D0FB689B6C1A6880
:1095D000FB689B6C42F480721A60FB685B6D002B29
:1095E00007D0FB685B6D1A68FB685B6D42F48072A4
:1095F0001A60FB681B681A68FB681B6842F001026E
:109600001A6005E0FB68002283F824200223FB7522
:10961000FB7D18461837BD4680BD80B584B000AFCD
:1096200078607B681B6C1B68FB607B681B681B6831
:10963000BB607B685B6C03F01F0304229A40FB68ED
:109640001340002B26D0BB6803F00403002B21D06D
:109650007B681B681B6803F02003002B07D17B6825
:109660001B681A687B681B6822F004021A607B681A
:109670005B6C03F01F027B681B6C042101FA02F291
:109680005A607B681B6B002B71D07B681B6B786802
:1096900098476CE07B685B6C03F01F0302229A40E2
:1096A000FB681340002B2ED0BB6803F00203002B95
:1096B00029D07B681B681B6803F02003002B0BD1AB
:1096C0007B681B681A687B681B6822F00A021A60B4
:1096D0007B68012283F825207B685B6C03F01F0206
:1096E0007B681B6C022101FA02F25A607B6800223F
:1096F00083F824207B68DB6A002B38D07B68DB6A28
:109700007868984733E07B685B6C03F01F0308229E
:109710009A40FB681340002B2AD0BB6803F0080373
:10972000002B25D07B681B681A687B681B6822F0B9
:109730000E021A607B685B6C03F01F027B681B6C77
:10974000012101FA02F25A607B680122DA637B6828
:10975000012283F825207B68002283F824207B687F
:109760005B6B002B04D07B685B6B7868984700BF0D
:1097700000BF1037BD4680BD80B485B000AFF86033
:10978000B9607A603B60FB68DB6CFA68126D5A6006
:10979000FB685B6D002B04D0FB689B6DFA68D26D93
:1097A0005A60FB685B6C03F01F02FB681B6C0121B5
:1097B00001FA02F25A60FB681B683A685A60FB685B
:1097C0009B68102B08D1FB681B687A689A60FB685D
:1097D0001B68BA68DA6007E0FB681B68BA689A60C1
:1097E000FB681B687A68DA6000BF1437BD465DF815
:1097F000047B704780B487B000AF78607B681B68DB
:109800001A46164B9A4202D8154B7B6101E0154B64
:109810007B617B693B617B681B68DBB2083B124A5A
:10982000A2FB03231B09FB607B685B6C9B089A000F
:109830003B6913441A467B689A647B680B4ADA6476
:10984000FB6803F01F0301229A407B681A6500BF82
:109850001C37BD465DF8047B704700BF070402401B
:109860000008024020080240CDCCCCCC8008024049
:1098700080B485B000AF78607B685B68DBB2FB606A
:10988000FA680B4B13449B001A467B685A657B6849
:10989000084A9A65FB68013B03F01F0301229A40C6
:1098A0007B68DA6500BF1437BD465DF8047B7047FE
:1098B0003F8200104009024080B485B000AF78605C
:1098C0007B68002B41D14B4B1B6803F4C063B3F59D
:1098D000806F31D1474BD3F88030464A23F48073F0
:1098E000C2F88030434B1B6823F4C063414A43F401
:1098F00000731360404B1B68322202FB03F33F4AA4
:10990000A2FB03239B0C0133FB6002E0FB68013BDD
:10991000FB60384B5B6903F48063B3F5806F02D161
:10992000FB68002BF2D1334B5B6903F48063B3F522
:10993000806F58D1032357E02E4BD3F880302D4A47
:1099400023F48073C2F880304DE07B68B3F5007F6C
:1099500041D1284B1B6803F4C063B3F5806F31D14C
:10996000244BD3F88030234A43F48073C2F880300C
:10997000204B1B6823F4C0631E4A43F4007313603A
:109980001D4B1B68322202FB03F31C4AA2FB03237C
:109990009B0C0133FB6002E0FB68013BFB60154B55
:1099A0005B6903F48063B3F5806F02D1FB68002B21
:1099B000F2D1104B5B6903F48063B3F5806F12D171
:1099C000032311E00B4BD3F880300A4A43F4807331
:1099D000C2F8803007E0074B1B6823F4C063054AD8
:1099E00043F480631360002318461437BD465DF8C6
:1099F000047B704700700040EC00002083DE1B43B6
:109A000080B400AF054B9B68044A43F480439360E5
:109A100000BFBD465DF8047B704700BF007000408A
:109A200080B485B000AF78607B6803F00703FB600B
:109A30000C4BDB68BB60BA684FF6FF031340BB609A
:109A4000FB681A02BB68134343F0BF6343F400335F
:109A5000BB60044ABB68D36000BF1437BD465DF8E5
:109A6000047B704700ED00E080B400AF044BDB687E
:109A70001B0A03F007031846BD465DF8047B7047D8
:109A800000ED00E080B483B000AF0346FB7197F9AE
:109A90000730002B0BDBFB7903F01F02074997F916
:109AA00007305B09012000FA02F241F8232000BFD1
:109AB0000C37BD465DF8047B704700BF00E100E055
:109AC00080B483B000AF03463960FB7197F907306B
:109AD000002B0ADB3B68DAB20C4997F90730120118
:109AE000D2B20B4483F800230AE03B68DAB208499B
:109AF000FB7903F00F03043B1201D2B20B441A7638
:109B000000BF0C37BD465DF8047B704700E100E004
:109B100000ED00E080B489B000AFF860B9607A6011
:109B2000FB6803F00703FB61FB69C3F10703042B28
:109B300028BF0423BB61FB690433062B02D9FB69F0
:109B4000033B00E000237B614FF0FF32BB6902FA68
:109B500003F3DA43BB681A407B699A404FF0FF3148
:109B60007B6901FA03F3D9437B680B401343184622
:109B70002437BD465DF8047B7047000080B582B095
:109B800000AF78607B68013BB3F1807F01D3012394
:109B90000FE00A4A7B68013B53600F214FF0FF3012
:109BA000FFF78EFF054B00229A60044B07221A60D4
:109BB000002318460837BD4680BD00BF10E000E016
:109BC00080B582B000AF78607868FFF729FF00BFEA
:109BD0000837BD4680BD80B586B000AF0346B9608A
:109BE0007A60FB73FFF740FF78617A68B96878693B
:109BF000FFF790FF024697F90F3011461846FFF71E
:109C00005FFF00BF1837BD4680BD80B582B000AF92
:109C10000346FB7197F907301846FFF733FF00BF83
:109C20000837BD4680BD80B582B000AF78607868E7
:109C3000FFF7A4FF034618460837BD4680BD80B431
:109C400083B000AF786039607B689B6823F47C1236
:109C50003B681A437B689A6000BF0C37BD465DF8CD
:109C6000047B704780B483B000AF786039607B6854
:109C70009B6823F0E0723B681A437B689A6000BFE0
:109C80000C37BD465DF8047B704780B483B000AFED
:109C900078607B689B6803F0E07318460C37BD461C
:109CA0005DF8047B7047000080B487B000AFF860B7
:109CB000B9607A603B60FB6860331A46BB689B0002
:109CC00013447B617B691A68084B13407A6802F081
:109CD000F8413A680A43134343F000427B691A6033
:109CE00000BF1C37BD465DF8047B704700F0FF03E2
:109CF00080B485B000AF786039607B6860331A4605
:109D00003B689B001344FB60FB681B6803F0F8434F
:109D100018461437BD465DF8047B704780B487B0A1
:109D200000AFF860B9607A60FB6860331A46BB68C0
:109D30009B0013447B617B691B6823F000427B68B6
:109D40001A437B691A6000BF1C37BD465DF8047B6F
:109D5000704780B487B000AFF860B9607A60FB6884
:109D600060331A46BB689B0013447B617B691B68A8
:109D700023F080727B681A437B691A6000BF1C372E
:109D8000BD465DF8047B704780B487B000AFF860D3
:109D9000B9607A60FB6860331A46BB689B00134465
:109DA0007B617B691B6823F000727B681A437B69C7
:109DB0001A6000BF1C37BD465DF8047B704780B455
:109DC00083B000AF786039607B685B6923F0004244
:109DD0003B681A437B685A6100BF0C37BD465DF88B
:109DE000047B704780B483B000AF78607B68DB6829
:109DF00003F44063002B01D1012300E00023184647
:109E00000C37BD465DF8047B704780B487B000AF67
:109E1000F860B9607A60FB6830331A46BB681B0A89
:109E20009B0003F00C0313447B617B691A68BB68D9
:109E300003F01F031F2101FA03F3DB431A407B6881
:109E40009B0E03F01F01BB6803F01F0301FA03F32D
:109E50001A437B691A6000BF1C37BD465DF8047B5E
:109E6000704780B487B000AFF860B9607A60FB6873
:109E700014331A46BB685B0E9B0003F004031344C3
:109E80007B617B691A68BB681B0D03F01F03072108
:109E900001FA03F3DB431A40BB681B0D03F01F03F9
:109EA000796801FA03F31A437B691A6000BF1C3713
:109EB000BD465DF8047B704780B485B000AFF860A4
:109EC000B9607A60FB68D3F8B020BB68C3F31203B3
:109ED000DB431A407B6803F018030849D940BB688C
:109EE0000B40C3F312031A43FB68C3F8B02000BF52
:109EF0001437BD465DF8047B704700BFFFFF0700C5
:109F000080B483B000AF78607B689B6803F01F0368
:109F100018460C37BD465DF8047B704780B483B0AB
:109F200000AF78607B689B6823F0204323F03F03F9
:109F30007A68936000BF0C37BD465DF8047B7047BC
:109F400080B483B000AF78607B689B6803F00053F7
:109F5000B3F1005F01D1012300E0002318460C3764
:109F6000BD465DF8047B704780B483B000AF786075
:109F70007B689B6823F0104323F03F0343F080523B
:109F80007B689A6000BF0C37BD465DF8047B704764
:109F900080B483B000AF78607B689B6803F0805327
:109FA000B3F1805F01D1012300E0002318460C3794
:109FB000BD465DF8047B704780B483B000AF786025
:109FC0007B689B6823F0004323F03F0343F00102CA
:109FD0007B689A6000BF0C37BD465DF8047B704714
:109FE00080B483B000AF78607B689B6823F0004347
:109FF00023F03F0343F002027B689A6000BF0C37F6
:10A00000BD465DF8047B704780B483B000AF7860D4
:10A010007B689B6803F00103012B01D1012300E061
:10A02000002318460C37BD465DF8047B704780B4AA
:10A0300083B000AF78607B689B6803F00203022B5B
:10A0400001D1012300E0002318460C37BD465DF81E
:10A05000047B704780B483B000AF78607B689B68F6
:10A0600023F0004323F03F0343F004027B689A602F
:10A0700000BF0C37BD465DF8047B704780B483B0E9
:10A0800000AF78607B689B6803F00403042B01D168
:10A09000012300E0002318460C37BD465DF8047B21
:10A0A000704780B483B000AF78607B689B6803F032
:10A0B0000803082B01D1012300E0002318460C37C8
:10A0C000BD465DF8047B704790B589B000AF7860FD
:10A0D0000023FB770023FB607B68002B01D1012369
:10A0E000A9E17B685B69002B7B68DB6D002B09D1E4
:10A0F0007868F7F72FFB7B6800221A667B680022DE
:10A1000083F858207B681B681846FFF719FF034641
:10A11000002B04D07B681B681846FFF7FFFE7B68A6
:10A120001B681846FFF734FF0346002B15D17B68E8
:10A130001B681846FFF718FF9C4B1B689B099C4A3D
:10A14000A2FB03239B0901335B00FB6002E0FB6879
:10A15000013BFB60FB68002BF9D17B681B6818464C
:10A16000FFF716FF0346002B0DD17B68DB6D43F034
:10A1700010027B68DA657B681B6E43F001027B6826
:10A180001A660123FB777B681B681846FFF776FF8A
:10A1900078617B68DB6D03F01003002B40F0428197
:10A1A0007B69002B40F03E817B68DB6D23F481737B
:10A1B00043F002027B68DA657B681B681846FFF78C
:10A1C00023FF0346002B41D17B681B68B3F1A04FEE
:10A1D00004D07B681B68774A93420FD14FF0A040B0
:10A1E000FFF712FF04467348FFF70EFF03462343B1
:10A1F000002B0CBF01230023DBB212E06E48FFF7F7
:10A2000003FF04466D48FFF7FFFE03461C436C48FE
:10A21000FFF7FAFE03462343002B0CBF0123002364
:10A22000DBB2002B12D07B681B68B3F1A04F04D0C7
:10A230007B681B685F4A934201D1624A00E0624A30
:10A240007B685B6819461046FFF7F9FC7B685B7F0B
:10A250005A037B68DB6B1A437B68DB681A437B68B5
:10A260009B681A437B6893F824301B041343BB613B
:10A270007B6893F82430012B06D17B689B6A013BF5
:10A280005B04BA691343BB617B68DB6A002B09D0AE
:10A290007B68DB6A03F478727B681B6B1343BA69D3
:10A2A0001343BB617B681B68DA68484B13407A68CC
:10A2B0001268B9690B43D3607B681B681B6923F084
:10A2C00040617B685A6B7B681B680A431A617B6834
:10A2D0001B681846FFF7E5FE38617B69002B7FD1CC
:10A2E0003B69002B7CD17B681B7F9A037B6893F8CA
:10A2F00038305B001343BB617B681B68DB6823F469
:10A30000804323F002037A681268B9690B43D36073
:10A310007B681B69002B17D07B681B681A697B68F8
:10A320001B6842F480321A617B681B68D3F8C03026
:10A3300023F47F5323F03F037A6811697A68126827
:10A340000B43C2F8C03013E07B681B681A697B6856
:10A350001B6822F480321A617B681B68D3F8C03016
:10A360007A68126823F47F5323F03F03C2F8C030A9
:10A370007B6893F84030012B2AD17B681B681B69EE
:10A3800023F4FF6323F004037A68516C7A68926CBB
:10A3900011437A68D26C11437A68126D0A431A43EA
:10A3A0007B681B6842F001021A6119E0EC00002092
:10A3B000632D3E05000100500004005000050050D0
:10A3C0000006005000030050000700500740F0FF57
:10A3D0007B681B681A697B681B6822F001021A619E
:10A3E0007B685B69012B0CD17B681B681B6B23F0BE
:10A3F0000F017B681B6A5A1E7B681B680A431A633D
:10A4000007E07B681B681A6B7B681B6822F00F02F1
:10A410001A637B68DB6D23F0030343F001027B6862
:10A42000DA6507E07B68DB6D43F010027B68DA6574
:10A430000123FB77FB7F18462437BD4690BD00BF44
:10A4400080B586B000AFF860B9607A60FB681B68C1
:10A45000B3F1A04F04D0FB681B685A4A934201D164
:10A46000594B00E0594B1846FFF74AFD3861FB682D
:10A470001B681846FFF702FE0346002B40F09B8046
:10A48000FB6893F85830012B01D1022396E0FB685A
:10A49000012283F85820FB681B684D4A934208D07C
:10A4A0003B69002B05D03B69052B02D03B69092B8A
:10A4B0007AD1F86800F0ECFC0346FB75FB7D002BBD
:10A4C0006DD1FB68DB6D23F4706323F0010343F46B
:10A4D0008072FB68DA65FB681B683A4A934209D0D0
:10A4E000FB681B683B4A934202D0FB681B6803E091
:10A4F000394B01E04FF0A043FA681268934202D052
:10A500003B69002B05D1FB68DB6D23F48012FB68EF
:10A51000DA65FB68DB6D03F48053002B06D0FB6823
:10A520001B6E23F00602FB681A6602E0FB6800223D
:10A530001A66FB685B6D294ADA62FB685B6D284A24
:10A540001A63FB685B6D274A5A63FB681B681C2211
:10A550001A60FB68002283F85820FB681B685A6861
:10A56000FB681B6842F010025A60FB681B68DA68DF
:10A57000FB681B6842F00102DA60FB68586DFB68FB
:10A580001B6840331946BA687B68FEF7CBFF034669
:10A59000FB75FB681B681846FFF75CFD0DE0FB6868
:10A5A000002283F8582008E00123FB75FB68002295
:10A5B00083F8582001E00223FB75FB7D184618370D
:10A5C000BD4680BD00010050000300500007005050
:10A5D0000006005000050050000400507BB0010848
:10A5E00053B101086FB1010880B483B000AF786047
:10A5F00000BF0C37BD465DF8047B704780B483B064
:10A6000000AF786000BF0C37BD465DF8047B704733
:10A6100080B5B6B000AF78603960002387F8D730D6
:10A620000023FB607B6893F85830012B02D1022392
:10A6300000F013BC7B68012283F858207B681B68FC
:10A640001846FFF71BFD0346002B40F0F3837B68A1
:10A6500018683B6859683B681B681A46FFF7D5FBCA
:10A660007B681B681846FFF709FDC7F8D0007B68B8
:10A670001B681846FFF715FDC7F8CC00D7F8D03097
:10A68000002B40F0D981D7F8CC30002B40F0D4819A
:10A690003B689B68B3F1004F0FD17B6818683B683B
:10A6A0001B6800221946FFF7DCFB7B681B684FF034
:10A6B00000411846FFF783FB0EE07B6818683B6893
:10A6C00019683B689B681A46FFF7CBFB7B681B68E1
:10A6D00000211846FFF773FB3B685A697B681B68CB
:10A6E000DB68DB0803F003035B0002FA03F3C7F83F
:10A6F000C8303B681B69042B22D07B6818683B6814
:10A7000019693B681A68D7F8C830FFF7CDFA7B683B
:10A7100018683B6819693B689B691A46FFF719FB83
:10A720007B6818683B6819693B681B7F012B02D165
:10A730004FF0007300E000231A46FFF725FB7BE192
:10A740007B681B6800211846FFF7D2FA0346C3F363
:10A750001203002B0AD17B681B6800211846FFF703
:10A76000C7FA03469B0E03F01F021EE07B681B68BE
:10A7700000211846FFF7BCFA0346C7F8BC30D7F8EB
:10A78000BC3093FAA3F3C7F8B830D7F8B830C7F89D
:10A79000C030D7F8C030002B01D1202304E0D7F817
:10A7A000C030B3FA83F3DBB21A463B681B68C3F3CD
:10A7B0001203002B05D13B681B689B0E03F01F039F
:10A7C00018E03B681B68C7F8B030D7F8B03093FA90
:10A7D000A3F3C7F8AC30D7F8AC30C7F8B430D7F82B
:10A7E000B430002B01D1202304E0D7F8B430B3FA01
:10A7F00083F3DBB29A4206D17B681B6800220021FA
:10A800001846FFF78BFA7B681B6801211846FFF793
:10A810006FFA0346C3F31203002B0AD17B681B684F
:10A8200001211846FFF764FA03469B0E03F01F024E
:10A830001EE07B681B6801211846FFF759FA0346A2
:10A84000C7F8A430D7F8A43093FAA3F3C7F8A03020
:10A85000D7F8A030C7F8A830D7F8A830002B01D11E
:10A86000202304E0D7F8A830B3FA83F3DBB21A460A
:10A870003B681B68C3F31203002B05D13B681B68C0
:10A880009B0E03F01F0318E03B681B68C7F8983065
:10A89000D7F8983093FAA3F3C7F89430D7F89430E8
:10A8A000C7F89C30D7F89C30002B01D1202304E05E
:10A8B000D7F89C30B3FA83F3DBB29A4206D17B68B7
:10A8C0001B68002201211846FFF728FA7B681B68E5
:10A8D00002211846FFF70CFA0346C3F31203002BBC
:10A8E0000AD17B681B6802211846FFF701FA03466C
:10A8F0009B0E03F01F021EE07B681B6802211846B6
:10A90000FFF7F6F90346C7F88C30D7F88C3093FA86
:10A91000A3F3C7F88830D7F88830C7F89030D7F855
:10A920009030002B01D1202304E0D7F89030B3FA07
:10A9300083F3DBB21A463B681B68C3F31203002B98
:10A9400005D13B681B689B0E03F01F0316E03B68B4
:10A950001B68C7F88030D7F8803093FAA3F3FB6701
:10A96000FB6FC7F88430D7F88430002B01D1202347
:10A9700004E0D7F88430B3FA83F3DBB29A4206D10D
:10A980007B681B68002202211846FFF7C7F97B6825
:10A990001B6803211846FFF7ABF90346C3F3120304
:10A9A000002B0AD17B681B6803211846FFF7A0F92A
:10A9B00003469B0E03F01F0217E07B681B68032110
:10A9C0001846FFF795F903467B677B6F93FAA3F36D
:10A9D0003B673B6FBB67BB6F002B01D1202303E0BC
:10A9E000BB6FB3FA83F3DBB21A463B681B68C3F351
:10A9F0001203002B05D13B681B689B0E03F01F035D
:10AA000011E03B681B68BB66BB6E93FAA3F37B66E1
:10AA10007B6EFB66FB6E002B01D1202303E0FB6EF7
:10AA2000B3FA83F3DBB29A4206D17B681B6800223B
:10AA300003211846FFF772F97B681B681846FFF779
:10AA4000E3FA0346002B40F03D817B6818683B68C1
:10AA500019683B68DB681A46FFF72EFA3B68DB682B
:10AA6000A24A934240F02E817B6818683B681B68BD
:10AA7000C3F31203002B0BD13B681B689B0E013301
:10AA800003F01F03092B94BF01230023DBB219E05D
:10AA90003B681B68FB65FB6D93FAA3F3BB65BB6D5D
:10AAA0003B663B6E002B01D1202303E03B6EB3FAE3
:10AAB00083F3DBB2013303F01F03092B94BF01239F
:10AAC0000023DBB2002B79D03B681B68C3F3120371
:10AAD000002B07D13B681B689B0E01339B0603F0DC
:10AAE000F84215E03B681B683B653B6D93FAA3F3A6
:10AAF000FB64FB6C7B657B6D002B01D1202303E0A5
:10AB00007B6DB3FA83F3DBB201339B0603F0F842AB
:10AB10003B681B68C3F31203002B09D13B681B6819
:10AB20009B0E013303F01F03012101FA03F317E029
:10AB30003B681B687B647B6C93FAA3F33B643B6CC0
:10AB4000BB64BB6C002B01D1202303E0BB6CB3FAC8
:10AB500083F3DBB2013303F01F03012101FA03F396
:10AB600042EA03013B681B68C3F31203002B0AD1BE
:10AB70003B681B689B0E013303F01F0213465B000A
:10AB800013441B0518E03B681B68BB63BB6B93FA5F
:10AB9000A3F37B637B6BFB63FB6B002B01D1202357
:10ABA00003E0FB6BB3FA83F3DBB2013303F01F0264
:10ABB00013465B0013441B050B437EE03B681B6898
:10ABC000C3F31203002B07D13B681B689B0E0133B4
:10ABD0009B0603F0F84215E03B681B68FB62FB6ACA
:10ABE00093FAA3F3BB62BB6A3B633B6B002B01D1BF
:10ABF000202303E03B6BB3FA83F3DBB201339B0604
:10AC000003F0F8423B681B68C3F31203002B09D121
:10AC10003B681B689B0E013303F01F03012101FAFF
:10AC200003F317E03B681B683B623B6A93FAA3F3AC
:10AC3000FB61FB697B627B6A002B01D1202303E06F
:10AC40007B6AB3FA83F3DBB2013303F01F03012104
:10AC500001FA03F342EA03013B681B68C3F31203E2
:10AC6000002B0DD13B681B689B0E013303F01F02C4
:10AC700013465B0013441E3B1B0543F000731BE0AF
:10AC80003B681B687B617B6993FAA3F33B613B697B
:10AC9000BB61BB69002B01D1202303E0BB69B3FA80
:10ACA00083F3DBB2013303F01F0213465B0013444E
:10ACB0001E3B1B0543F000730B433A68926819462C
:10ACC000FFF7CFF83B681A68094B1340002B00F0E0
:10ACD000BE807B681B68B3F1A04F04D07B681B6803
:10ACE000044A93420AD1044B09E000BF00007F40B0
:10ACF000000008800001005000030050594B184626
:10AD0000FEF7C3FFC7F8C4003B681B68564A93426E
:10AD100004D03B681B68554A93423AD1D7F8C430F7
:10AD200003F40003002B34D17B681B68B3F1A04F00
:10AD300005D07B681B684E4A934240F085807B6853
:10AD40001B68B3F1A04F04D07B681B68494A93424B
:10AD500001D1494A00E0434AD7F8C43043F4000324
:10AD600019461046FEF77EFF444B1B689B09444A78
:10AD7000A2FB03239B095A1C13465B0013449B0050
:10AD8000FB6002E0FB68013BFB60FB68002BF9D134
:10AD90005AE03B681B683B4A934225D1D7F8C43040
:10ADA00003F08073002B1FD17B681B68314A9342EC
:10ADB00004D17B681B68344A934247D07B681B6888
:10ADC000B3F1A04F04D07B681B682A4A934201D19B
:10ADD000294A00E0234AD7F8C43043F0807319466B
:10ADE0001046FEF73FFF31E03B681B68274A93425D
:10ADF0002DD1D7F8C43003F48003002B27D17B6812
:10AE00001B681C4A934222D07B681B68B3F1A04F99
:10AE100004D07B681B68174A934201D1164A00E0B0
:10AE2000104AD7F8C43043F4800319461046FEF7A1
:10AE300019FF0CE07B68DB6D43F020027B68DA656C
:10AE4000012387F8D73002E000BF00E000BF7B6835
:10AE5000002283F8582097F8D7301846D837BD46D7
:10AE600080BD00BF00070050000021C31000C0904B
:10AE7000000600500001005000030050EC000020CC
:10AE8000632D3E05000052C700050050000084CB32
:10AE900080B584B000AF78600023BB607B681B681E
:10AEA0001846FFF7B1F80346002B76D17B681B6884
:10AEB0009A683C4B1340002B0DD07B68DB6D43F050
:10AEC00010027B68DA657B681B6E43F001027B68C9
:10AED0001A66012362E07B681B681846FFF76CF86E
:10AEE0007B681B68B3F1A04F04D07B681B682E4AB7
:10AEF000934201D12D4B00E02D4B1846FEF7C5FEC5
:10AF0000034603F40003002B13D02A4B1B689B0954
:10AF1000294AA2FB03239B095A1C13465B001344D6
:10AF20009B00BB6002E0BB68013BBB60BB68002BC1
:10AF3000F9D1FCF757FEF86028E07B681B681846DB
:10AF4000FFF762F80346002B04D17B681B681846A4
:10AF5000FFF732F8FCF746FE0246FB68D31A022BD5
:10AF600014D97B681B681B6803F00103012B0DD00B
:10AF70007B68DB6D43F010027B68DA657B681B6ED3
:10AF800043F001027B681A66012307E07B681B68B7
:10AF90001B6803F00103012BCFD1002318461037A3
:10AFA000BD4680BD3F0000800001005000030050FE
:10AFB00000070050EC000020632D3E0580B584B0F2
:10AFC00000AF78607B681B681846FFF730F8F860C0
:10AFD0007B681B681846FFF717F80346002B47D01D
:10AFE000FB68002B44D17B681B689B6803F00D0352
:10AFF000012B0CD17B681B681846FEF7F1FF7B68BC
:10B000001B6803221A60FCF7EDFDB86029E07B683D
:10B01000DB6D43F010027B68DA657B681B6E43F0E2
:10B0200001027B681A66012323E0FCF7DBFD024680
:10B03000BB68D31A022B14D97B681B689B6803F08A
:10B040000103002B0DD07B68DB6D43F010027B68A1
:10B05000DA657B681B6E43F001027B681A66012388
:10B0600007E07B681B689B6803F00103002BDCD1C1
:10B07000002318461037BD4680BD80B584B000AFB0
:10B0800078607B689B6AFB60FB68DB6D03F05003B4
:10B09000002B4BD1FB68DB6D43F40072FB68DA6573
:10B0A000FB681B681B6803F00803002B21D0FB68BA
:10B0B0001B681846FEF796FE0346002B32D0FB684D
:10B0C0001B68DB6803F40053002B2BD1FB68DB6D9E
:10B0D00023F48072FB68DA65FB68DB6D03F4805350
:10B0E000002B1FD1FB68DB6D43F00102FB68DA65C2
:10B0F00018E0FB681B68DB6803F00203002B11D12A
:10B10000FB68DB6D23F48072FB68DA65FB68DB6D3E
:10B1100003F48053002B05D1FB68DB6D43F0010283
:10B12000FB68DA65F868F5F793FF0EE0FB68DB6D06
:10B1300003F01003002B03D0F868FFF75FFA04E078
:10B14000FB685B6D5B6B7868984700BF1037BD4646
:10B1500080BD80B584B000AF78607B689B6AFB607F
:10B16000F868FFF741FA00BF1037BD4680BD80B5D3
:10B1700084B000AF78607B689B6AFB60FB68DB6D26
:10B1800043F04002FB68DA65FB681B6E43F0040283
:10B19000FB681A66F868FFF731FA00BF1037BD4642
:10B1A00080BD80B483B000AF78607B689B6803F09B
:10B1B0000103012B01D1012300E0002318460C37C5
:10B1C000BD465DF8047B704780B483B000AF786003
:10B1D00039607B689B6823F0404323F03F033A6863
:10B1E00002F08042134343F000427B689A6000BF44
:10B1F0000C37BD465DF8047B704780B483B000AF68
:10B2000078607B689B6803F00043B3F1004F01D185
:10B21000012300E0002318460C37BD465DF8047B8F
:10B22000704780B483B000AF78607B689B6803F0A0
:10B230000403042B01D1012300E0002318460C373E
:10B24000BD465DF8047B704780B584B000AF786080
:10B2500039600023BB607B6893F85830012B01D123
:10B2600002234DE07B68012283F858207868FFF7BD
:10B27000A5FE0346FB73FB7B002B36D17B68DB6DA1
:10B2800023F4885323F0020343F002027B68DA655B
:10B290007B681B6839681846FFF796FF14E0BB68A7
:10B2A0000133BB60BB68184A93420DD97B68DB6DE4
:10B2B00023F0120343F010027B68DA657B680022FA
:10B2C00083F8582001231BE07B681B681846FFF7B2
:10B2D00094FF0346002BE2D17B68DB6D23F0030370
:10B2E00043F001027B68DA6505E07B68DB6D43F0C3
:10B2F00010027B68DA657B68002283F85820FB7BAC
:10B3000018461037BD4680BD01DE040090B5A1B0DF
:10B3100000AF78603960002387F87F307B6893F84E
:10B320005830012B01D10223E7E07B68012283F82A
:10B33000582000237B660023BB667B681B68B3F143
:10B34000A04F02D16F4BBB6009E07B681B686E4A5F
:10B35000934202D16D4BBB6001E00023BB60BB6830
:10B36000002B0BD17B68DB6D43F020027B68DA6534
:10B370007B68002283F858200123BEE0BB68184692
:10B38000FFF74FFFB8677B681B681846FFF749FF58
:10B390000346002B40F0A080BB6F002B40F09C8048
:10B3A0007B681B68B3F1A04F04D07B681B68554ACB
:10B3B000934201D1564B00E0564B7B673B681B68BC
:10B3C000002B4BD07B6F9B6823F460423B6859682D
:10B3D0007B6893F838305B030B431A437B6F9A60AA
:10B3E0007B681B68B3F1A04F04D07B681B68454A9B
:10B3F00093420FD14FF0A040FFF7D3FE04464148DF
:10B40000FFF7CFFE03462343002B0CBF012300238D
:10B41000DBB212E03C48FFF7C4FE04463B48FFF7AE
:10B42000C0FE03461C433C48FFF7BBFE03462343D4
:10B43000002B0CBF01230023DBB2002B56D07B6F07
:10B440009B6823F4716323F00F033A6811683A682C
:10B4500092680A431A437B6F9A6047E07B6F9B6850
:10B4600023F460427B6F9A607B681B68B3F1A04F46
:10B4700004D07B681B68234A93420FD14FF0A04051
:10B48000FFF78FFE04461F48FFF78BFE034623435A
:10B49000002B0CBF01230023DBB212E01A48FFF798
:10B4A00080FE04461948FFF77CFE03461C431A48F9
:10B4B000FFF777FE03462343002B0CBF0123002335
:10B4C000DBB2002B12D07B6F9B6823F4716323F0F7
:10B4D0000F037A6F936009E07B68DB6D43F0200215
:10B4E0007B68DA65012387F87F3000E000BF7B6866
:10B4F000002283F8582097F87F3018468437BD46DD
:10B5000090BD00BF00010050000400500005005035
:10B5100000030050000700500006005080B582B0C4
:10B5200000AF78607B68002B01D101238DE07B6840
:10B5300093F84130DBB2002B06D17B68002283F800
:10B5400040207868F6F77CFA7B68242283F8412053
:10B550007B681B681A687B681B6822F001021A600E
:10B560007B685A687B681B6822F070621A617B688E
:10B570001B689A687B681B6822F400429A607B68AB
:10B58000DB68012B07D17B689A687B681B6842F4F3
:10B5900000429A6006E07B689A687B681B6842F408
:10B5A00004429A607B68DB68022B08D17B681B68C9
:10B5B0005A687B681B6842F400625A6007E07B6847
:10B5C0001B685A687B681B6822F400625A607B68BB
:10B5D0001B685B687A68126843F0007343F40043A9
:10B5E00053607B681B68DA687B681B6822F4004242
:10B5F000DA607B681A697B685B6942EA03017B68F1
:10B600009B691A027B681B680A43DA607B68D96908
:10B610007B681A6A7B681B680A431A607B681B6830
:10B620001A687B681B6842F001021A607B6800227E
:10B630005A647B68202283F841207B6800221A63C9
:10B640007B68002283F84220002318460837BD4655
:10B6500080BD80B483B000AF786039607B6893F8B8
:10B660004130DBB2202B38D17B6893F84030012B7E
:10B6700001D1022332E07B68012283F840207B68FD
:10B68000242283F841207B681B681A687B681B684A
:10B6900022F001021A607B681B681A687B681B68CD
:10B6A00022F480521A607B681B6819687B681B68EB
:10B6B0003A680A431A607B681B681A687B681B68D3
:10B6C00042F001021A607B68202283F841207B68E7
:10B6D000002283F84020002300E0022318460C37A4
:10B6E000BD465DF8047B704780B485B000AF7860DC
:10B6F00039607B6893F84130DBB2202B39D17B680D
:10B7000093F84030012B01D1022333E07B68012202
:10B7100083F840207B68242283F841207B681B68E3
:10B720001A687B681B6822F001021A607B681B683C
:10B730001B68FB60FB6823F47063FB603B681B02C3
:10B74000FA681343FB607B681B68FA681A607B68C1
:10B750001B681A687B681B6842F001021A607B68EC
:10B76000202283F841207B68002283F840200023B8
:10B7700000E0022318461437BD465DF8047B70478D
:10B7800080B582B000AF78607B68002B01D10123C7
:10B7900049E07B6893F83D30DBB2002B06D17B6833
:10B7A000002283F83C207868F6F746FB7B6802228B
:10B7B00083F83D207B681A687B680433194610467D
:10B7C00000F03AFC7B68012283F848207B68012264
:10B7D00083F83E207B68012283F83F207B680122AA
:10B7E00083F840207B68012283F841207B68012296
:10B7F00083F842207B68012283F843207B68012282
:10B8000083F844207B68012283F845207B6801226D
:10B8100083F846207B68012283F847207B68012259
:10B8200083F83D20002318460837BD4680BD000040
:10B8300080B485B000AF78607B6893F83D30DBB2B0
:10B84000012B01D001234CE07B68022283F83D20CC
:10B850007B681B68264A934222D07B681B68B3F141
:10B86000804F1DD07B681B68224A934218D07B68AA
:10B870001B68214A934213D07B681B681F4A93427E
:10B880000ED07B681B681E4A934209D07B681B68F8
:10B890001C4A934204D07B681B681B4A934215D113
:10B8A0007B681B689A68194B1340FB60FB68062B8A
:10B8B00015D0FB68B3F5803F11D07B681B681A6810
:10B8C0007B681B6842F001021A6008E07B681B6815
:10B8D0001A687B681B6842F001021A6000E000BF32
:10B8E000002318461437BD465DF8047B704700BF3F
:10B8F000002C01400004004000080040000C004003
:10B9000000340140004001400050014007000100A8
:10B9100080B582B000AF78607B68002B01D1012335
:10B9200049E07B6893F83D30DBB2002B06D17B68A1
:10B93000002283F83C20786800F041F87B680222FE
:10B9400083F83D207B681A687B68043319461046EB
:10B9500000F072FB7B68012283F848207B6801229B
:10B9600083F83E207B68012283F83F207B68012218
:10B9700083F840207B68012283F841207B68012204
:10B9800083F842207B68012283F843207B680122F0
:10B9900083F844207B68012283F845207B680122DC
:10B9A00083F846207B68012283F847207B680122C8
:10B9B00083F83D20002318460837BD4680BD80B47B
:10B9C00083B000AF786000BF0C37BD465DF8047BE4
:10B9D0007047000080B584B000AF786039603B6884
:10B9E000002B09D17B6893F83E30DBB2012B14BFEA
:10B9F00001230023DBB23CE03B68042B09D17B68C8
:10BA000093F83F30DBB2012B14BF01230023DBB2DC
:10BA10002FE03B68082B09D17B6893F84030DBB2FC
:10BA2000012B14BF01230023DBB222E03B680C2B67
:10BA300009D17B6893F84130DBB2012B14BF01239D
:10BA40000023DBB215E03B68102B09D17B6893F82B
:10BA50004230DBB2012B14BF01230023DBB208E02C
:10BA60007B6893F84330DBB2012B14BF0123002322
:10BA7000DBB2002B01D00123A6E03B68002B04D1F0
:10BA80007B68022283F83E2023E03B68042B04D12C
:10BA90007B68022283F83F201BE03B68082B04D11F
:10BAA0007B68022283F8402013E03B680C2B04D112
:10BAB0007B68022283F841200BE03B68102B04D105
:10BAC0007B68022283F8422003E07B68022283F82D
:10BAD00043207B681B6801223968184600F026FF66
:10BAE0007B681B683A4A934218D07B681B68394AC6
:10BAF000934213D07B681B68374A93420ED07B6811
:10BB00001B68364A934209D07B681B68344A9342CB
:10BB100004D07B681B68334A934201D1012300E0C3
:10BB20000023002B07D07B681B685A6C7B681B685E
:10BB300042F400425A647B681B68254A934222D033
:10BB40007B681B68B3F1804F1DD07B681B68264A59
:10BB5000934218D07B681B68244A934213D07B68B9
:10BB60001B68234A93420ED07B681B68194A934294
:10BB700009D07B681B68184A934204D07B681B6815
:10BB8000184A934215D17B681B689A68194B134079
:10BB9000FB60FB68062B15D0FB68B3F5803F11D026
:10BBA0007B681B681A687B681B6842F001021A6098
:10BBB00008E07B681B681A687B681B6842F001021A
:10BBC0001A6000E000BF002318461037BD4680BD54
:10BBD000002C01400034014000400140004401407D
:10BBE00000480140005001400004004000080040AF
:10BBF000000C00400700010080B586B000AFF8607F
:10BC0000B9607A600023FB75FB6893F83C30012B28
:10BC100001D10223FFE0FB68012283F83C207B680E
:10BC2000142B00F2F08001A252F823F081BC01082D
:10BC300007BE010807BE010807BE0108C1BC010814
:10BC400007BE010807BE010807BE010803BD0108C1
:10BC500007BE010807BE010807BE010843BD010871
:10BC600007BE010807BE010807BE010885BD01081F
:10BC700007BE010807BE010807BE0108C5BD0108CF
:10BC8000FB681B68B968184600F08AFAFB681B68F5
:10BC90009A69FB681B6842F008029A61FB681B689E
:10BCA0009A69FB681B6822F004029A61FB681B68B2
:10BCB0009969BB681A69FB681B680A439A61A5E029
:10BCC000FB681B68B968184600F004FBFB681B683A
:10BCD0009A69FB681B6842F400629A61FB681B6802
:10BCE0009A69FB681B6822F480629A61FB681B6892
:10BCF0009969BB681B691A02FB681B680A439A6151
:10BD000084E0FB681B68B968184600F077FBFB68A5
:10BD10001B68DA69FB681B6842F00802DA61FB689D
:10BD20001B68DA69FB681B6822F00402DA61FB68B1
:10BD30001B68D969BB681A69FB681B680A43DA612A
:10BD400064E0FB681B68B968184600F0E9FBFB6813
:10BD50001B68DA69FB681B6842F40062DA61FB6801
:10BD60001B68DA69FB681B6822F48062DA61FB6891
:10BD70001B68D969BB681B691A02FB681B680A4308
:10BD8000DA6143E0FB681B68B968184600F05CFCA8
:10BD9000FB681B681A6DFB681B6842F008021A6595
:10BDA000FB681B681A6DFB681B6822F004021A65A9
:10BDB000FB681B68196DBB681A69FB681B680A433E
:10BDC0001A6523E0FB681B68B968184600F0A6FCFA
:10BDD000FB681B681A6DFB681B6842F400621A65F9
:10BDE000FB681B681A6DFB681B6822F480621A6589
:10BDF000FB681B68196DBB681B691A02FB681B682E
:10BE00000A431A6502E00123FB7500BFFB680022AC
:10BE100083F83C20FB7D18461837BD4680BD00BF27
:10BE200080B584B000AF786039600023FB737B6815
:10BE300093F83C30012B01D10223EEE07B68012214
:10BE400083F83C207B68022283F83D207B681B68D6
:10BE50009B68BB60BB6823F4441323F07703BB608B
:10BE6000BB6823F47F43BB607B681B68BA689A6039
:10BE70003B681B686B4A934200F0B980694A934261
:10BE800000F2BE80684A934200F0B180664A934255
:10BE900000F2B680654A934200F0A980634A93425B
:10BEA00000F2AE80624A934200F0A180604A934261
:10BEB00000F2A6805F4A934200F099805D4A934267
:10BEC00000F29E80B3F1101F00F09180B3F1101FBB
:10BED00000F29680B3F5801F00F08980B3F5801FD3
:10BEE00000F28E80B3F5005F3ED0B3F5005F00F244
:10BEF0008780B3F5805F00F08680B3F5805F7FD8E0
:10BF0000702B1AD0702B7BD8602B50D0602B77D839
:10BF1000502B3CD0502B73D8402B58D0402B6FD88F
:10BF2000302B64D0302B6BD8202B60D0202B67D8DF
:10BF3000002B5CD0102B5AD062E07B6818683B68FD
:10BF400099683B685A683B68DB6800F0CFFC7B6807
:10BF50001B689B68BB60BB6843F07703BB607B6872
:10BF60001B68BA689A604FE07B6818683B689968FC
:10BF70003B685A683B68DB6800F0B8FC7B681B686C
:10BF80009A687B681B6842F480429A603CE07B6858
:10BF900018683B6859683B68DB681A4600F02AFC61
:10BFA0007B681B685021184600F083FC2CE07B68FE
:10BFB00018683B6859683B68DB681A4600F049FC22
:10BFC0007B681B686021184600F073FC1CE07B68EE
:10BFD00018683B6859683B68DB681A4600F00AFC41
:10BFE0007B681B684021184600F063FC0CE07B680E
:10BFF0001A683B681B681946104600F05AFC03E0BB
:10C000000123FB7300E000BF7B68012283F83D2021
:10C010007B68002283F83C20FB7B18461037BD4626
:10C0200080BD00BF700010005000100040001000E4
:10C03000300010002000100080B485B000AF7860A0
:10C0400039607B681B68FB607B684C4A934217D061
:10C050007B68B3F1804F13D07B68494A93420FD07D
:10C060007B68484A93420BD07B68474A934207D08B
:10C070007B68464A934203D07B68454A934208D185
:10C08000FB6823F07003FB603B685B68FA6813434E
:10C09000FB607B68394A934223D07B68B3F1804FC1
:10C0A0001FD07B68364A93421BD07B68354A934247
:10C0B00017D07B68344A934213D07B68334A93424B
:10C0C0000FD07B68334A93420BD07B68324A93424D
:10C0D00007D07B68314A934203D07B682C4A934255
:10C0E00008D1FB6823F44073FB603B68DB68FA68A7
:10C0F0001343FB60FB6823F080023B685B691343DA
:10C10000FB607B68FA681A603B689A687B68DA6251
:10C110003B681A687B689A627B68184A934213D01E
:10C120007B681A4A93420FD07B681A4A93420BD01D
:10C130007B68194A934207D07B68184A934203D020
:10C140007B68134A934203D13B681A697B681A6380
:10C150007B6801225A617B681B6903F00103012B94
:10C1600005D17B681B6923F001027B681A6100BF5F
:10C170001437BD465DF8047B704700BF002C0140BA
:10C180000004004000080040000C00400034014062
:10C19000005001400040014000440140004801407F
:10C1A00080B487B000AF786039607B681B6A7B61C0
:10C1B0007B681B6A23F001027B681A627B685B68FC
:10C1C0003B617B689B69FB60FB6823F4803323F051
:10C1D0007003FB60FB6823F00303FB603B681B6894
:10C1E000FA681343FB607B6923F002037B613B68C1
:10C1F0009B687A6913437B617B68304A934213D012
:10C200007B682F4A93420FD07B682E4A93420BD013
:10C210007B682D4A934207D07B682C4A934203D017
:10C220007B682B4A93420CD17B6923F008037B6126
:10C230003B68DB687A6913437B617B6923F0040305
:10C240007B617B681D4A934213D07B681C4A9342F2
:10C250000FD07B681B4A93420BD07B681A4A9342EB
:10C2600007D07B68194A934203D07B68184A9342EF
:10C2700011D13B6923F480733B613B6923F4007364
:10C280003B613B685B693A6913433B613B689B696F
:10C290003A6913433B617B683A695A607B68FA6884
:10C2A0009A613B685A687B685A637B687A691A624C
:10C2B00000BF1C37BD465DF8047B7047002C014071
:10C2C000003401400040014000440140004801406A
:10C2D0000050014080B487B000AF786039607B685F
:10C2E0001B6A7B617B681B6A23F010027B681A6201
:10C2F0007B685B683B617B689B69FB60FB6823F044
:10C30000807323F4E043FB60FB6823F44073FB601D
:10C310003B681B681B02FA681343FB607B6923F0D0
:10C3200020037B613B689B681B017A6913437B6137
:10C330007B682C4A934207D07B682B4A934203D0F8
:10C340007B682A4A93420DD17B6923F080037B618D
:10C350003B68DB681B017A6913437B617B6923F0CF
:10C3600040037B617B681F4A934213D07B681E4A5F
:10C3700093420FD07B681E4A93420BD07B681D4AC4
:10C38000934207D07B681C4A934203D07B68174ACC
:10C39000934213D13B6923F480633B613B6923F4EF
:10C3A00000633B613B685B699B003A6913433B61F7
:10C3B0003B689B699B003A6913433B617B683A6920
:10C3C0005A607B68FA689A613B685A687B689A632E
:10C3D0007B687A691A6200BF1C37BD465DF8047B32
:10C3E000704700BF002C0140003401400050014064
:10C3F00000400140004401400048014080B487B043
:10C4000000AF786039607B681B6A7B617B681B6A60
:10C4100023F480727B681A627B685B683B617B688F
:10C42000DB69FB60FB6823F4803323F07003FB605F
:10C43000FB6823F00303FB603B681B68FA68134347
:10C44000FB607B6923F400737B613B689B681B0284
:10C450007A6913437B617B682B4A934207D07B68E0
:10C460002A4A934203D07B68294A93420DD17B69C3
:10C4700023F400637B613B68DB681B027A6913432A
:10C480007B617B6923F480637B617B681E4A9342F6
:10C4900013D07B681D4A93420FD07B681D4A93429C
:10C4A0000BD07B681C4A934207D07B681B4A93429F
:10C4B00003D07B68164A934213D13B6923F480531F
:10C4C0003B613B6923F400533B613B685B691B01A3
:10C4D0003A6913433B613B689B691B013A6913430B
:10C4E0003B617B683A695A607B68FA68DA613B684D
:10C4F0005A687B68DA637B687A691A6200BF1C3706
:10C50000BD465DF8047B7047002C014000340140BB
:10C5100000500140004001400044014000480140FB
:10C5200080B487B000AF786039607B681B6A7B613C
:10C530007B681B6A23F480527B681A627B685B68A5
:10C540003B617B68DB69FB60FB6823F0807323F44D
:10C55000E043FB60FB6823F44073FB603B681B68AF
:10C560001B02FA681343FB607B6923F400537B6171
:10C570003B689B681B037A6913437B617B682C4A89
:10C58000934207D07B682B4A934203D07B682A4AA8
:10C5900093420DD17B6923F400437B613B68DB68E8
:10C5A0001B037A6913437B617B6923F480437B61BE
:10C5B0007B681F4A934213D07B681E4A93420FD078
:10C5C0007B681E4A93420BD07B681D4A934207D07A
:10C5D0007B681C4A934203D07B68174A934213D16D
:10C5E0003B6923F480433B613B6923F400433B6197
:10C5F0003B685B699B013A6913433B613B689B69FC
:10C600009B013A6913433B617B683A695A607B68D6
:10C61000FA68DA613B685A687B681A647B687A69F1
:10C620001A6200BF1C37BD465DF8047B704700BF2F
:10C63000002C014000340140005001400040014006
:10C64000004401400048014080B487B000AF7860EA
:10C6500039607B681B6A3B617B681B6A23F480320C
:10C660007B681A627B685B687B617B681B6DFB6023
:10C67000FB6823F4803323F07003FB603B681B6886
:10C68000FA681343FB603B6923F400333B613B686A
:10C690009B681B043A6913433B617B68194A9342C8
:10C6A00013D07B68184A93420FD07B68174A934295
:10C6B0000BD07B68164A934207D07B68154A934299
:10C6C00003D07B68144A934209D17B6923F48033F9
:10C6D0007B613B685B691B027A6913437B617B6802
:10C6E0007A695A607B68FA681A653B685A687B68A1
:10C6F0009A647B683A691A6200BF1C37BD465DF8D0
:10C70000047B7047002C0140003401400040014090
:10C7100000440140004801400050014080B487B00F
:10C7200000AF786039607B681B6A3B617B681B6A7D
:10C7300023F480127B681A627B685B687B617B688C
:10C740001B6DFB60FB6823F0807323F4E043FB6008
:10C750003B681B681B02FA681343FB603B6923F4C8
:10C7600000133B613B689B681B053A6913433B61BF
:10C770007B681A4A934213D07B68194A93420FD0C0
:10C780007B68184A93420BD07B68174A934207D0C4
:10C790007B68164A934203D07B68154A934209D1BD
:10C7A0007B6923F480237B613B685B699B027A6928
:10C7B00013437B617B687A695A607B68FA681A6503
:10C7C0003B685A687B68DA647B683A691A6200BF22
:10C7D0001C37BD465DF8047B704700BF002C01404C
:10C7E0000034014000400140004401400048014045
:10C7F0000050014080B487B000AFF860B9607A6043
:10C80000FB681B6A7B61FB681B6A23F00102FB6803
:10C810001A62FB689B693B613B6923F0F0033B6153
:10C820007B681B013A6913433B617B6923F00A0370
:10C830007B617A69BB6813437B61FB683A699A61E3
:10C84000FB687A691A6200BF1C37BD465DF8047B3D
:10C85000704780B487B000AFF860B9607A60FB6859
:10C860001B6A7B61FB681B6A23F01002FB681A627B
:10C87000FB689B693B613B6923F470433B617B68C8
:10C880001B033A6913433B617B6923F0A0037B617F
:10C89000BB681B017A6913437B61FB683A699A6143
:10C8A000FB687A691A6200BF1C37BD465DF8047BDD
:10C8B000704780B485B000AF786039607B689B6852
:10C8C000FB60FB6823F4401323F07003FB603A68BD
:10C8D000FB68134343F00703FB607B68FA689A60C8
:10C8E00000BF1437BD465DF8047B704780B487B045
:10C8F00000AFF860B9607A603B60FB689B687B6161
:10C900007B6923F47F437B613B681A027B681A438F
:10C91000BB6813437A6913437B61FB687A699A6049
:10C9200000BF1C37BD465DF8047B704780B487B0FC
:10C9300000AFF860B9607A60BB6803F01F030122A2
:10C9400002FA03F37B61FB681A6A7B69DB431A40D6
:10C95000FB681A62FB681A6ABB6803F01F037968F8
:10C9600001FA03F31A43FB681A6200BF1C37BD4685
:10C970005DF8047B7047000080B485B000AF78603C
:10C9800039607B6893F83C30012B01D1022374E0BD
:10C990007B68012283F83C207B68022283F83D20DB
:10C9A0007B681B685B68FB607B681B689B68BB607F
:10C9B0007B681B68344A934209D07B681B68334A02
:10C9C000934204D07B681B68314A934208D1FB68CC
:10C9D00023F47003FB603B685B68FA681343FB60F9
:10C9E000FB6823F0007323F07003FB603B681B6857
:10C9F000FA681343FB607B681B68FA685A607B68BF
:10CA00001B68214A934222D07B681B68B3F1804F98
:10CA10001DD07B681B681F4A934218D07B681B6837
:10CA20001D4A934213D07B681B681C4A93420ED068
:10CA30007B681B68154A934209D07B681B68184ABB
:10CA4000934204D07B681B68114A93420CD1BB68A7
:10CA500023F08003BB603B689B68BA681343BB60EC
:10CA60007B681B68BA689A607B68012283F83D2066
:10CA70007B68002283F83C20002318461437BD460B
:10CA80005DF8047B704700BF002C0140003401407A
:10CA9000005001400004004000080040000C00402D
:10CAA0000040014080B485B000AF78603960002359
:10CAB000FB607B6893F83C30012B01D1022378E0C6
:10CAC0007B68012283F83C20FB6823F0FF023B686F
:10CAD000DB681343FB60FB6823F440723B689B6890
:10CAE0001343FB60FB6823F480623B685B6813437D
:10CAF000FB60FB6823F400623B681B681343FB6028
:10CB0000FB6823F480523B681B691343FB60FB689E
:10CB100023F400523B685B691343FB60FB6823F41A
:10CB200080423B681B6B1343FB60FB6823F470225D
:10CB30003B689B691B041343FB60FB6823F0805236
:10CB40003B68DB691343FB607B681B681C4A9342AC
:10CB500009D07B681B681B4A934204D07B681B6822
:10CB6000194A93421CD1FB6823F470023B689B6A0C
:10CB70001B051343FB60FB6823F080723B681B6A54
:10CB80001343FB60FB6823F000723B685B6A13434E
:10CB9000FB60FB6823F000523B68DB6A1343FB60D9
:10CBA0007B681B68FA685A647B68002283F83C2023
:10CBB000002318461437BD465DF8047B704700BF5C
:10CBC000002C0140003401400050014080B582B08B
:10CBD00000AF78607B68002B01D1012342E07B68C5
:10CBE000D3F88830002B06D17B68002283F884209C
:10CBF0007868F5F72DFA7B682422C3F888207B68D3
:10CC00001B681A687B681B6822F001021A607B6847
:10CC10009B6A002B02D0786800F0B2FB786800F0C5
:10CC2000B3F80346012B01D101231BE07B681B688D
:10CC30005A687B681B6822F490425A607B681B68C4
:10CC40009A687B681B6822F02A029A607B681B68DE
:10CC50001A687B681B6842F001021A60786800F06D
:10CC600031FC034618460837BD4680BD80B58AB002
:10CC700002AFF860B9603B601346FB80FB68D3F8F5
:10CC80008830202B7BD1BB68002B02D0FB88002B87
:10CC900001D1012374E0FB680022C3F89020FB68F7
:10CCA0002122C3F88820FAF79DFF7861FB68FA8893
:10CCB000A3F85420FB68FA88A3F85620FB689B6809
:10CCC000B3F5805F08D1FB681B69002B04D10023FA
:10CCD000FB61BB68BB6103E0BB68FB610023BB6118
:10CCE00030E03B6800937B6900228021F86800F007
:10CCF00093FC0346002B05D0FB682022C3F8882054
:10CD000003233DE0FB69002B0BD1BB691B881A464E
:10CD1000FB681B68C2F308029A62BB690233BB61FD
:10CD200007E0FB691A78FB681B689A62FB690133AC
:10CD3000FB61FB68B3F856309BB2013B9AB2FB68CB
:10CD4000A3F85620FB68B3F856309BB2002BC8D12D
:10CD50003B6800937B6900224021F86800F05CFC8E
:10CD60000346002B05D0FB682022C3F8882003234C
:10CD700006E0FB682022C3F88820002300E002239D
:10CD800018462037BD4680BD2DE9B04F8CB000AFAE
:10CD90007861002387F82A307B699A687B691B6970
:10CDA0001A437B695B691A437B69DB691343FB6246
:10CDB0007B691B681A68AA4B13407A691268F96A82
:10CDC0000B4313607B691B685B6823F440517B69EC
:10CDD000DA687B691B680A435A607B699B69FB625E
:10CDE0007B691B689F4A934204D07B691B6AFA6A7D
:10CDF0001343FB627B691B689B6823F06E4323F43B
:10CE000030637A691268F96A0B4393607B691B6827
:10CE1000DB6A23F00F017B695A6A7B691B680A434E
:10CE2000DA627B691B68904A934225D18F4BD3F815
:10CE3000883003F00303032B1AD801A252F823F021
:10CE400051CE010861CE010859CE010869CE010812
:10CE5000012387F82B3016E1022387F82B3012E1EB
:10CE6000042387F82B300EE1082387F82B300AE1E2
:10CE7000102387F82B3006E17B691B687C4A9342BC
:10CE800038D17A4BD3F8883003F00C030C2B2DD813
:10CE900001A252F823F000BFCDCE0108EDCE01086B
:10CEA000EDCE0108EDCE0108DDCE0108EDCE010882
:10CEB000EDCE0108EDCE0108D5CE0108EDCE01087A
:10CEC000EDCE0108EDCE0108E5CE0108002387F87C
:10CED0002B30D8E0022387F82B30D4E0042387F8E6
:10CEE0002B30D0E0082387F82B30CCE0102387F8D4
:10CEF0002B30C8E07B691B685E4A934225D15B4BAF
:10CF0000D3F8883003F03003302B16D0302B18D8EC
:10CF1000202B0AD0202B14D8002B02D0102B08D0A5
:10CF20000FE0002387F82B30ADE0022387F82B3089
:10CF3000A9E0042387F82B30A5E0082387F82B30DD
:10CF4000A1E0102387F82B309DE07B691B684A4ADB
:10CF5000934225D1454BD3F8883003F0C003C02B52
:10CF600016D0C02B18D8802B0AD0802B14D8002BB9
:10CF700002D0402B08D00FE0002387F82B3082E04E
:10CF8000022387F82B307EE0042387F82B307AE0E9
:10CF9000082387F82B3076E0102387F82B3072E0D7
:10CFA0007B691B68354A93422AD1304BD3F88830CD
:10CFB00003F44073B3F5407F1AD0B3F5407F1BD81C
:10CFC000B3F5007F0CD0B3F5007F15D8002B03D04C
:10CFD000B3F5807F08D00FE0002387F82B3052E0B4
:10CFE000022387F82B304EE0042387F82B304AE0E9
:10CFF000082387F82B3046E0102387F82B3042E0D7
:10D000007B691B68174A93423AD1184BD3F8883092
:10D0100003F44063B3F5406F1AD0B3F5406F1BD8EB
:10D02000B3F5006F0CD0B3F5006F15D8002B03D00B
:10D03000B3F5806F08D00FE0002387F82B3022E093
:10D04000022387F82B301EE0042387F82B301AE0E8
:10D05000082387F82B3016E0102387F82B3012E0D6
:10D06000F369FFCF0080004000380140001002400B
:10D070000044004000480040004C00400050004088
:10D08000102387F82B307B691B68AE4A934240F02F
:10D09000978097F82B30082B23D801A252F823F061
:10D0A000C5D00108E3D00108CDD00108E3D00108C4
:10D0B000D3D00108E3D00108E3D00108E3D0010890
:10D0C000DBD00108FBF776FA786210E09E4B7B62BA
:10D0D0000DE0FBF703FA786209E04FF400437B624E
:10D0E00005E000237B62012387F82A3000BF7B6ABA
:10D0F000002B00F030817B695B6A944A32F8133070
:10D100001A467B6AB3FBF2F3BB617B695A6813462C
:10D110005B001344BA699A4205D37B695B681B03C1
:10D12000BA699A4203D9012387F82A3013E17B6A4E
:10D130000022BB60FA607B695B6A844A32F8133074
:10D140009BB200223B607A60D7E90023D7E9020155
:10D15000F3F766F802460B46104619464FF00002F8
:10D160004FF000030B0243EA106302027969496839
:10D17000490800200C46054612EB040843EB05095C
:10D180007B695B6800229A46934652465B4640465E
:10D190004946F3F745F802460B4613463B623B6AA5
:10D1A000B3F5407F08D33B6AB3F5801F04D27B6997
:10D1B0001B683A6ADA60CEE0012387F82A30CAE0B9
:10D1C0007B69DB69B3F5004F66D197F82B30082BEC
:10D1D00027D801A252F823F0FDD1010805D2010899
:10D1E0000DD2010823D2010813D2010823D201086D
:10D1F00023D2010823D201081BD20108FBF7DAF978
:10D20000786214E0FBF7ECF9786210E04E4B7B6239
:10D210000DE0FBF763F9786209E04FF400437B62AD
:10D2200005E000237B62012387F82A3000BF7B6A78
:10D23000002B00F090807B695B6A444A32F813301F
:10D240001A467B6AB3FBF2F35A007B695B685B08A2
:10D250001A447B695B68B2FBF3F33B623B6A0F2BBA
:10D2600016D93B6AB3F5803F12D23B6A9BB223F0DA
:10D270000F03FB833B6A5B089BB203F007039AB280
:10D28000FB8B1343FB837B691B68FA8BDA6062E0DC
:10D29000012387F82A305EE097F82B30082B28D836
:10D2A00001A252F823F000BFCDD20108D5D2010867
:10D2B000DDD20108F3D20108E3D20108F3D201085C
:10D2C000F3D20108F3D20108EBD20108FBF772F99F
:10D2D000786214E0FBF784F9786210E01A4B7B6205
:10D2E0000DE0FBF7FBF8786209E04FF400437B6246
:10D2F00005E000237B62012387F82A3000BF7B6AA8
:10D30000002B28D07B695B6A104A32F813301A462A
:10D310007B6AB3FBF2F27B695B685B081A447B694A
:10D320005B68B2FBF3F33B623B6A0F2B10D93B6A9D
:10D33000B3F5803F0CD23B6A9AB27B691B68DA6016
:10D3400009E000BF008000400024F400EC0C02085B
:10D35000012387F82A307B690122A3F86A207B69C0
:10D360000122A3F868207B6900225A677B690022AA
:10D370009A6797F82A3018463037BD46BDE8B08F17
:10D3800080B483B000AF78607B689B6A03F00803C9
:10D39000002B0AD07B681B685B6823F400417B6824
:10D3A0009A6B7B681B680A435A607B689B6A03F030
:10D3B0000103002B0AD07B681B685B6823F40031F3
:10D3C0007B68DA6A7B681B680A435A607B689B6AE1
:10D3D00003F00203002B0AD07B681B685B6823F410
:10D3E00080317B681A6B7B681B680A435A607B68D4
:10D3F0009B6A03F00403002B0AD07B681B685B6800
:10D4000023F480217B685A6B7B681B680A435A604F
:10D410007B689B6A03F01003002B0AD07B681B68B3
:10D420009B6823F480517B68DA6B7B681B680A4336
:10D430009A607B689B6A03F02003002B0AD07B680C
:10D440001B689B6823F400517B681A6C7B681B681F
:10D450000A439A607B689B6A03F04003002B1AD052
:10D460007B681B685B6823F480117B685A6C7B685F
:10D470001B680A435A607B685B6CB3F5801F0AD156
:10D480007B681B685B6823F4C0017B689A6C7B68CF
:10D490001B680A435A607B689B6A03F08003002B79
:10D4A0000AD07B681B685B6823F400217B68DA6C18
:10D4B0007B681B680A435A6000BF0C37BD465DF8A5
:10D4C000047B704780B598B002AF78607B6800221B
:10D4D000C3F89020FAF786FB78657B681B681B68A9
:10D4E00003F00803082B2FD16FF07E4300937B6D70
:10D4F00000224FF40011786800F08EF80346002BEC
:10D5000022D07B681B68BB63BB6B53E8003F7B6327
:10D510007B6B23F080033B657B681B681A463B6D81
:10D520007B643A64396C7A6C41E80023FB63FB6BE3
:10D53000002BE6D17B682022C3F888207B6800227C
:10D5400083F88420032363E07B681B681B6803F077
:10D550000403042B49D16FF07E4300937B6D0022BE
:10D560004FF48001786800F057F80346002B3CD058
:10D570007B681B687B627B6A53E8003F3B623B6AC7
:10D5800023F49073FB647B681B681A46FB6C3B6357
:10D59000FA62F96A3A6B41E80023BB62BB6A002B6E
:10D5A000E6D17B681B6808333B613B6953E8003F69
:10D5B000FB60FB6823F00103BB647B681B680833D6
:10D5C000BA6CFA61BB61B969FA6941E800237B6111
:10D5D0007B69002BE5D17B682022C3F88C207B6817
:10D5E000002283F88420032312E07B682022C3F802
:10D5F00088207B682022C3F88C207B680022DA66B2
:10D600007B6800221A677B68002283F8842000234D
:10D6100018465837BD4680BD80B584B000AFF8606D
:10D62000B9603B601346FB714FE0BB69B3F1FF3F4C
:10D630004BD0FAF7D7FA02463B68D31ABA699A4236
:10D6400002D3BB69002B01D103234EE0FB681B68AA
:10D650001B6803F00403002B37D0BB68802B34D049
:10D66000BB68402B31D0FB681B68DB6903F0080303
:10D67000082B10D1FB681B6808221A62F86800F0BA
:10D6800038F8FB680822C3F89020FB68002283F872
:10D690008420012329E0FB681B68DB6903F4006335
:10D6A000B3F5006F11D1FB681B684FF400621A627A
:10D6B000F86800F01EF8FB682022C3F89020FB6891
:10D6C000002283F8842003230FE0FB681B68DA69DB
:10D6D000BB681340BA689A420CBF01230023DBB237
:10D6E0001A46FB799A42A0D0002318461037BD464F
:10D6F00080BD80B495B000AF78607B681B687B63A9
:10D700007B6B53E8003F3B633B6B23F49073FB64FC
:10D710007B681B681A46FB6C3B64FA63F96B3A6CD6
:10D7200041E80023BB63BB6B002BE6D17B681B6821
:10D7300008333B623B6A53E8003FFB61FB6923F01F
:10D74000805323F00103BB647B681B680833BA6C09
:10D75000FA62BB62B96AFA6A41E800237B627B6ABB
:10D76000002BE3D17B68DB6E012B18D17B681B6833
:10D77000FB60FB6853E8003FBB60BB6823F010030D
:10D780007B647B681B681A467B6CBB617A61796934
:10D79000BA6941E800233B613B69002BE6D17B6815
:10D7A0002022C3F88C207B680022DA667B68002286
:10D7B0005A6700BF5437BD465DF8047B704780B49C
:10D7C00085B000AF78607B6893F88430012B01D17D
:10D7D000022327E07B68012283F884207B682422CF
:10D7E000C3F888207B681B681B68FB607B681B682C
:10D7F0001A687B681B6822F001021A60FB6823F03C
:10D800000053FB607B6800225A667B681B68FA68DD
:10D810001A607B682022C3F888207B68002283F886
:10D820008420002318461437BD465DF8047B7047FA
:10D8300080B584B000AF786039607B6893F884303D
:10D84000012B01D102232DE07B68012283F8842083
:10D850007B682422C3F888207B681B681B68FB60F8
:10D860007B681B681A687B681B6822F001021A60DB
:10D870007B681B689B6823F060417B681B683A6883
:10D880000A439A60786800F04FF87B681B68FA6872
:10D890001A607B682022C3F888207B68002283F806
:10D8A0008420002318461037BD4680BD80B584B063
:10D8B00000AF786039607B6893F88430012B01D128
:10D8C00002232DE07B68012283F884207B682422D8
:10D8D000C3F888207B681B681B68FB607B681B683B
:10D8E0001A687B681B6822F001021A607B681B685B
:10D8F0009B6823F060617B681B683A680A439A6002
:10D90000786800F011F87B681B68FA681A607B6819
:10D910002022C3F888207B68002283F8842000231B
:10D9200018461037BD4680BD80B485B000AF786022
:10D930007B685B6E002B08D17B680122A3F86A200C
:10D940007B680122A3F8682031E00823FB730823D9
:10D95000BB737B681B689B685B0EDBB203F007033D
:10D960007B737B681B689B685B0FDBB203F007036C
:10D970003B73BB7B3A7B11498A5C02FB03F33A7B26
:10D980000F498A5C93FBF2F39AB27B68A3F86A2092
:10D99000FB7B7A7B09498A5C02FB03F37A7B0849AB
:10D9A0008A5C93FBF2F39AB27B68A3F8682000BF0D
:10D9B0001437BD465DF8047B704700BF040D0208B4
:10D9C0000C0D020880B400AF074BD3F88830064A2C
:10D9D00043F47003C2F88830034B044A9A6000BFD6
:10D9E000BD465DF8047B704700ED00E000000108D3
:10D9F00080B586B000AFF860B9601346FB71FB6874
:10DA0000002B01D103231FE0FB680022C3F8B822DA
:10DA1000FB680022C3F8C022FB680022C3F8CC22B6
:10DA2000BB68002B03D0FB68BA68C3F8B422FB685C
:10DA3000012283F89C22FB68FA791A70F868F5F7DE
:10DA40008BFB0346FB75FB7D18461837BD4680BD32
:10DA500080B584B000AF786039600023FB813B68FB
:10DA6000002B01D1032316E07B683A68C3F8B82283
:10DA70007B68D3F8B832DB6A002B0BD07B68D3F815
:10DA8000B832DB6A07F10E021046984702467B68FF
:10DA9000C3F8CC22002318461037BD4680BD80B5A0
:10DAA00082B000AF78607868F5F7B6FB0346184699
:10DAB0000837BD4680BD80B483B000AF78600023D6
:10DAC00018460C37BD465DF8047B704780B584B0BE
:10DAD00000AF78600B46FB700323FB737B68D3F8C1
:10DAE000B832002B09D07B68D3F8B8321B68FA78BB
:10DAF0001146786898470346FB73FB7B184610373E
:10DB0000BD4680BD80B582B000AF78600B46FB702B
:10DB10007B68D3F8B832002B07D07B68D3F8B832D3
:10DB20005B68FA78114678689847002318460837EA
:10DB3000BD4680BD80B584B000AF786039607B6839
:10DB400003F2AA233968184600F046FF7B680122D9
:10DB5000C3F894227B68B3F8B0321A467B68C3F8E6
:10DB600098227B6893F8AA3203F01F03022B1AD085
:10DB7000022B22D8002B02D0012B0AD01DE07B689B
:10DB800003F2AA231946786800F0EEF90346FB7306
:10DB900020E07B6803F2AA231946786800F052FA65
:10DBA0000346FB7316E07B6803F2AA2319467868E4
:10DBB00000F091FA0346FB730CE07B6893F8AA32FD
:10DBC00023F07F03DBB219467868F5F785FB03463F
:10DBD000FB7300BFFB7B18461037BD4680BD80B588
:10DBE00086B000AFF8600B467A60FB72FB7A002BC0
:10DBF00038D1FB6803F5AA733B61FB68D3F8943214
:10DC0000032B4AD13B699A683B69DB689A4213D976
:10DC10003B699A683B69DB68D21A3B699A603B6949
:10DC2000DA683B699B68934228BF13461A467968B5
:10DC3000F86800F0C5FF30E0FB6893F89C32DBB277
:10DC4000032B0BD1FB68D3F8B8321B69002B05D02E
:10DC5000FB68D3F8B8321B69F8689847F86800F099
:10DC6000C0FF1AE0FB6893F89C32DBB2032B14D19F
:10DC7000FB68D3F8B8329B69002B0ED0FB68D3F851
:10DC8000B8329B69FA7A1146F86898470346FB75E3
:10DC9000FB7D002B01D0FB7D00E0002318461837E8
:10DCA000BD4680BD80B586B000AFF8600B467A6097
:10DCB000FB72FB7A002B6BD1FB6814333B61FB6872
:10DCC000D3F89432022B56D13B699A683B69DB68E2
:10DCD0009A4214D93B699A683B69DB68D21A3B695E
:10DCE0009A603B699B681A467968F86800F03AFFC9
:10DCF000002300220021F868F5F798FB3BE03B6920
:10DD0000DA683B699B689A421CD13B695A683B6957
:10DD1000DB689A4216D33B695A68FB68D3F898329D
:10DD20009A420FD200220021F86800F01BFFFB6826
:10DD30000022C3F89822002300220021F868F5F79A
:10DD400075FB18E0FB6893F89C32DBB2032B0BD118
:10DD5000FB68D3F8B832DB68002B05D0FB68D3F83A
:10DD6000B832DB68F86898478021F868F5F7B4FAAC
:10DD7000F86800F049FFFB6893F8A032012B22D12C
:10DD8000F868FFF798FEFB68002283F8A0221AE0EB
:10DD9000FB6893F89C32DBB2032B14D1FB68D3F8F9
:10DDA000B8325B69002B0ED0FB68D3F8B8325B69E0
:10DDB000FA7A1146F86898470346FB75FB7D002BFD
:10DDC00001D0FB7D00E0002318461837BD4680BD1A
:10DDD00080B582B000AF78607B68012283F89C2216
:10DDE0007B680022C3F894227B6800225A607B681B
:10DDF0000022C3F8A4227B68D3F8B832002B01D1EB
:10DE000003232FE07B68D3F8BC32002B0FD07B6854
:10DE1000D3F8B8325B68002B09D07B68D3F8B832EE
:10DE20005B687A685268D2B2114678689847402396
:10DE3000002200217868F5F70AFA7B680122A3F82E
:10DE400064217B684022C3F86021402300228021A6
:10DE50007868F5F7FCF97B6801229A847B68402298
:10DE60001A62002318460837BD4680BD80B483B0CF
:10DE700000AF78600B46FB707B68FA781A74002359
:10DE800018460C37BD465DF8047B704780B483B0FC
:10DE900000AF78607B6893F89C32DAB27B6883F8D5
:10DEA0009D227B68042283F89C22002318460C37AD
:10DEB000BD465DF8047B704780B483B000AF7860E6
:10DEC0007B6893F89C32DBB2042B06D17B6893F815
:10DED0009D32DAB27B6883F89C22002318460C3707
:10DEE000BD465DF8047B704780B582B000AF7860B6
:10DEF0007B68D3F8B832002B01D1032312E07B6892
:10DF000093F89C32DBB2032B0BD17B68D3F8B83289
:10DF1000DB69002B05D07B68D3F8B832DB69786801
:10DF20009847002318460837BD4680BD80B487B0A7
:10DF300000AF78607B687B617B691B787B827B6943
:10DF400001337B617B691B783B823B8A1B021AB2DF
:10DF5000B7F9123013431BB2FB81FB8918461C37FB
:10DF6000BD465DF8047B704780B584B000AF786033
:10DF700039600023FB733B681B7803F06003402B80
:10DF800005D0402B53D8002B0BD0202B4FD17B68D2
:10DF9000D3F8B8329B683968786898470346FB73B2
:10DFA0004AE03B685B78092B3BD801A252F823F08A
:10DFB00005E0010819E0010823E001080FE001086D
:10DFC00023E00108E3DF0108D9DF010823E00108AD
:10DFD000FBDF0108EDDF01083968786800F0DEF941
:10DFE00024E03968786800F06DFB1FE039687868D4
:10DFF00000F0ACFB0346FB7318E03968786800F06A
:10E000004BFC13E03968786800F07CFC0EE039685E
:10E01000786800F0ABFC09E03968786800F0BAFC79
:10E0200004E03968786800F011FD00BF04E0396849
:10E03000786800F00BFD00BFFB7B18461037BD462B
:10E0400080BD00BF80B584B000AF78603960002328
:10E05000FB733B681B7803F06003402B05D0402B1B
:10E060002FD8002B01D0202B2BD17B6893F89C322A
:10E07000DBB2013B022B1DD83B689B88DBB2012B36
:10E0800013D87B68D3F8B8329B68396878689847AA
:10E090000346FB733B68DB88002B10D1FB7B002B16
:10E0A0000DD1786800F09DFD09E03968786800F0CE
:10E0B000CDFC04E03968786800F0C8FC00E000BFDF
:10E0C00004E03968786800F0C1FC00BFFB7B1846AB
:10E0D0001037BD4680BD80B584B000AF7860396030
:10E0E0000023FB733B689B88BB733B681B7803F082
:10E0F0006003402B07D0402B00F24581002B0CD051
:10E10000202B40F040817B68D3F8B8329B68396897
:10E11000786898470346FB733AE13B685B78032BCA
:10E1200007D0032B00F32981002B7FD0012B3CD09B
:10E1300023E17B6893F89C32DBB2022B02D0032BE5
:10E1400016D02CE0BB7B002B0DD0BB7B802B0AD0E4
:10E15000BB7B19467868F5F7BFF880217868F5F73A
:10E16000BBF800BF20E03968786800F06FFC1BE066
:10E170003B685B88002B0ED1BB7B002B0BD0BB7B9D
:10E18000802B08D03B68DB88002B04D1BB7B194671
:10E190007868F5F7A1F8786800F023FD04E03968A5
:10E1A000786800F053FC00BFECE07B6893F89C3289
:10E1B000DBB2022B02D0032B16D030E0BB7B002B4E
:10E1C0000DD0BB7B802B0AD0BB7B19467868F5F756
:10E1D00083F880217868F5F77FF800BF25E039687B
:10E1E000786800F033FC20E03B685B88002B1BD193
:10E1F000BB7B03F07F03002B04D0BB7B1946786800
:10E20000F5F789F8786800F0ECFC7B68D3F8B83251
:10E210009B683968786898470346FB7304E039685F
:10E22000786800F013FC00E000BFABE07B6893F877
:10E230009C32DBB2022B02D0032B32D097E0BB7BA7
:10E24000002B07D0BB7B802B04D03968786800F0A6
:10E25000FDFB91E097F90E30002B0BDABB7B03F04E
:10E260007F0213469B0013449B0010337A681344CB
:10E2700004330BE0BB7B03F07F0213469B00134487
:10E280009B0003F5A8737A6813440433BB60BB6832
:10E2900000221A60BB6802221946786800F047FC29
:10E2A0006AE097F90E30002B11DABB7B03F00F0206
:10E2B000796813469B0013449B000B4424331B884E
:10E2C000002B17D13968786800F0C0FB54E0BB7BA5
:10E2D00003F00F02796813469B0013449B000B4424
:10E2E00003F5B2731B88002B04D13968786800F0FD
:10E2F000ADFB41E097F90E30002B0BDABB7B03F04E
:10E300007F0213469B0013449B0010337A6813442A
:10E3100004330BE0BB7B03F07F0213469B001344E6
:10E320009B0003F5A8737A6813440433BB60BB7B7E
:10E33000002B02D0BB7B802B03D1BB6800221A606C
:10E340000EE0BB7B19467868F5F704F80346002B0E
:10E3500003D0BB6801221A6002E0BB6800221A6089
:10E36000BB6802221946786800F0E1FB04E03968D6
:10E37000786800F06BFB00BF04E03968786800F053
:10E3800065FB00BF04E03968786800F05FFB00BF00
:10E39000FB7B18461037BD4680BD000080B584B0B9
:10E3A00000AF7860396000233B810023FB600023CD
:10E3B000FB723B685B881B0A9BB2013B0E2B00F291
:10E3C000528101A252F823F039E4010851E4010816
:10E3D00091E4010867E6010867E6010807E601081D
:10E3E00033E6010867E6010867E6010867E6010809
:10E3F00067E6010867E6010867E6010867E60108C5
:10E4000005E401087B68D3F8B432DB69002B0BD03C
:10E410007B68D3F8B432DB697A68127C07F10801B3
:10E4200010469847F86026E13968786800F00EFBDE
:10E43000FB7A0133FB721EE17B68D3F8B4321B68B0
:10E440007A68127C07F1080110469847F86012E1DB
:10E450007B681B7C002B0DD17B68D3F8B8329B6A9C
:10E4600007F1080210469847F860FB680133022262
:10E470001A7000E17B68D3F8B832DB6A07F1080252
:10E4800010469847F860FB68013302221A70F2E0E8
:10E490003B685B88DBB2052B00F2AC8001A252F82E
:10E4A00023F000BFBDE40108F1E4010825E50108FF
:10E4B00059E501088DE50108C1E501087B68D3F83D
:10E4C000B4325B68002B0BD07B68D3F8B4325B6846
:10E4D0007A68127C07F1080110469847F86091E0CD
:10E4E0003968786800F0B2FAFB7A0133FB7289E090
:10E4F0007B68D3F8B4329B68002B0BD07B68D3F8D1
:10E50000B4329B687A68127C07F10801104698477C
:10E51000F86077E03968786800F098FAFB7A0133A0
:10E52000FB726FE07B68D3F8B432DB68002B0BD052
:10E530007B68D3F8B432DB687A68127C07F1080193
:10E5400010469847F8605DE03968786800F07EFA18
:10E55000FB7A0133FB7255E07B68D3F8B4321B6958
:10E56000002B0BD07B68D3F8B4321B697A68127C1D
:10E5700007F1080110469847F86043E03968786869
:10E5800000F064FAFB7A0133FB723BE07B68D3F85E
:10E59000B4325B69002B0BD07B68D3F8B4325B6973
:10E5A0007A68127C07F1080110469847F86029E064
:10E5B0003968786800F04AFAFB7A0133FB7221E08F
:10E5C0007B68D3F8B4329B69002B0BD07B68D3F8FF
:10E5D000B4329B697A68127C07F1080110469847AB
:10E5E000F8600FE03968786800F030FAFB7A0133A0
:10E5F000FB7207E03968786800F028FAFB7A01338B
:10E60000FB7200BF37E07B681B7C002B09D17B6865
:10E61000D3F8B8325B6B07F1080210469847F860F0
:10E6200029E03968786800F011FAFB7A0133FB724F
:10E6300021E07B681B7C002B0DD17B68D3F8B832BE
:10E640001B6B07F1080210469847F860FB6801331E
:10E6500007221A700FE03968786800F0F7F9FB7A42
:10E660000133FB7207E03968786800F0EFF9FB7A54
:10E670000133FB7200BFFB7A002B1ED13B68DB88A5
:10E68000002B16D03B89002B0ED03B68DA883B89E3
:10E69000934228BF13469BB23B813B891A46F968D7
:10E6A000786800F044FA09E03968786800F0CEF93B
:10E6B00004E0786800F095FA00E000BF1037BD462E
:10E6C00080BD00BF80B584B000AF786039603B6822
:10E6D0009B88002B31D13B68DB88002B2DD13B6818
:10E6E0005B887F2B29D83B685B88DBB203F07F0314
:10E6F000FB737B6893F89C32DBB2032B04D139683F
:10E70000786800F0A3F91DE07B68FA7B83F89E220D
:10E71000FB7B19467868F4F749FE786800F061FAE7
:10E72000FB7B002B04D07B68022283F89C2209E04B
:10E730007B68012283F89C2204E03968786800F045
:10E7400085F900BF00BF1037BD4680BD80B584B0DD
:10E7500000AF786039600023FB733B685B88DAB2F6
:10E760004C4B1A704B4B1B78012B05D939687868D4
:10E7700000F06CF9032388E07B6893F89C32DBB2ED
:10E78000022B02D0032B25D071E0424B1B78002BCB
:10E790001CD0404B1B781A467B685A603D4B1B7857
:10E7A00019467868FFF792F90346FB73FB7B002B51
:10E7B00004D03968786800F049F965E0786800F0BD
:10E7C00010FA7B68032283F89C225DE0786800F0F1
:10E7D00008FA59E02F4B1B78002B12D17B680222DC
:10E7E00083F89C222B4B1B781A467B685A60294B76
:10E7F0001B7819467868FFF785F9786800F0F1F919
:10E8000042E0244B1B781A467B685B689A422AD008
:10E810007B685B68DBB219467868FFF773F91D4BBC
:10E820001B781A467B685A601A4B1B781946786821
:10E83000FFF74CF90346FB73FB7B002B0FD03968C5
:10E84000786800F003F97B685B68DBB2194678688A
:10E85000FFF758F97B68022283F89C2214E078685D
:10E8600000F0BFF910E0786800F0BBF90CE03968FF
:10E87000786800F0EBF8074B1B7819467868FFF7CB
:10E8800041F90323FB7300BFFB7B18461037BD46DD
:10E8900080BD00BF542C002080B582B000AF7860EE
:10E8A00039603B68DB88012B04D03968786800F058
:10E8B000CDF823E07B6893F89C32DBB2022B02DCBC
:10E8C000002B03DC15E0032B0BD012E07B68002249
:10E8D0009A607B68083301221946786800F027F9AE
:10E8E0000CE07B68043301221946786800F01FF9B8
:10E8F00004E03968786800F0A9F800BF00BF083765
:10E90000BD4680BD80B582B000AF786039607B685D
:10E9100093F89C32DBB2013B022B1ED83B68DB88AC
:10E92000022B04D03968786800F090F81AE07B6810
:10E930000122DA607B68D3F8A432002B05D07B6813
:10E94000DB6843F002027B68DA607B680C330222EA
:10E950001946786800F0EBF804E03968786800F050
:10E9600075F800BF00BF0837BD4680BD80B582B0D6
:10E9700000AF786039603B685B88012B06D17B680B
:10E980000122C3F8A422786800F02BF900BF0837F1
:10E99000BD4680BD80B582B000AF786039607B68CD
:10E9A00093F89C32DBB2013B022B0BD83B685B88AF
:10E9B000012B0CD17B680022C3F8A422786800F0F8
:10E9C00010F904E03968786800F040F800E000BF12
:10E9D00000BF0837BD4680BD80B584B000AF786009
:10E9E00039603B68FB60FB681A787B681A70FB68CB
:10E9F0000133FB60FB681A787B685A70FB6801334F
:10EA0000FB60F868FFF792FA03461A467B685A8063
:10EA1000FB680133FB60FB680133FB60F868FFF7BC
:10EA200085FA03461A467B689A80FB680133FB60CF
:10EA3000FB680133FB60F868FFF778FA03461A4673
:10EA40007B68DA8000BF1037BD4680BD80B582B0DC
:10EA500000AF7860396080217868F4F73DFC0021D0
:10EA60007868F4F739FC00BF0837BD4680BD80B533
:10EA700086B000AFF860B9607A600023FB75FB6870
:10EA8000002B36D0FB683B61386900F036F803464E
:10EA900001339BB25B009AB27B681A80FB7DBA6837
:10EAA00013447A6812781A70FB7D0133FB75FB7D85
:10EAB000BA68134403221A70FB7D0133FB7513E01F
:10EAC000FB7DBA6813443A6912781A703B690133C6
:10EAD0003B61FB7D0133FB75FB7DBA68134400226B
:10EAE0001A70FB7D0133FB753B691B78002BE7D166
:10EAF00000E000BF1837BD4680BD80B485B000AFD0
:10EB000078600023FB737B68BB6005E0FB7B01330F
:10EB1000FB73BB680133BB60BB681B78002BF5D16E
:10EB2000FB7B18461437BD465DF8047B704780B503
:10EB300084B000AFF860B9607A60FB680222C3F865
:10EB40009422FB687A689A61FB687A68DA617B686C
:10EB5000BA680021F868F4F748FC0023184610371B
:10EB6000BD4680BD80B584B000AFF860B9607A6002
:10EB70007B68BA680021F868F4F737FC0023184670
:10EB80001037BD4680BD80B584B000AFF860B96075
:10EB90007A60FB680322C3F89422FB687A68C3F8A2
:10EBA0005821FB687A68C3F85C217B68BA68002149
:10EBB000F868F4F73BFC002318461037BD4680BDCB
:10EBC00080B584B000AFF860B9607A607B68BA68DD
:10EBD0000021F868F4F72AFC002318461037BD46D8
:10EBE00080BD80B582B000AF78607B680422C3F836
:10EBF00094220023002200217868F4F7F6FB00231A
:10EC000018460837BD4680BD80B582B000AF786039
:10EC10007B680522C3F89422002300220021786833
:10EC2000F4F704FC002318460837BD4680BD80B5C4
:10EC300084B000AF78600B46FB704FF40770F4F7B8
:10EC40005FFCF860FB68002B05D17B680022C3F8ED
:10EC5000BC22022366E07B68FA68C3F8BC227B68AA
:10EC60001B7C002B19D14FF400730222812178689C
:10EC7000F4F7EDFA7B6801221A874FF40073022241
:10EC800001217868F4F7E3FA7B680122A3F8782180
:10EC90007B681022A3F84E2016E040230222812137
:10ECA0007868F4F7D4FA7B6801221A87402302229D
:10ECB00001217868F4F7CBFA7B680122A3F8782168
:10ECC0007B681022A3F84E20082303228221786853
:10ECD000F4F7BDFA7B680122A3F84C207B68D3F8D7
:10ECE000C0321B689847FB680022C3F81422FB68F7
:10ECF0000022C3F818227B681B7C002B09D1FB681B
:10ED0000D3F804224FF4007301217868F4F78EFBE6
:10ED100007E0FB68D3F80422402301217868F4F768
:10ED200085FB002318461037BD4680BD80B582B0F4
:10ED300000AF78600B46FB7081217868F4F7ADFA7C
:10ED40007B6800221A8701217868F4F7A6FA7B68AD
:10ED50000022A3F8782182217868F4F79EFA7B6874
:10ED60000022A3F84C207B680022A3F84E207B6889
:10ED7000D3F8BC32002B0ED07B68D3F8C0325B686E
:10ED800098477B68D3F8BC321846F4F7C7FB7B681A
:10ED90000022C3F8BC22002318460837BD4680BDB8
:10EDA00080B586B000AF786039607B68D3F8BC323C
:10EDB0003B6100237B7300237B810023FB753B6950
:10EDC000002B01D10323AFE03B681B7803F0600305
:10EDD000002B3FD0202B40F09F803B68DB88002B2E
:10EDE0002ED03B681B785BB2002B16DA7B68D3F819
:10EDF000C0329B683A68507839693A68D288984737
:10EE00003B68DB88072B28BF0723FB813B69FA8916
:10EE100019467868FFF78BFE85E03B685A783B69B6
:10EE200083F800223B68DB88DAB23B6983F8012271
:10EE300039693B68DB881A467868FFF7A4FE72E000
:10EE40007B68D3F8C0329B683A68507800223968F2
:10EE5000984768E03B685B780B2B52D801A252F8C8
:10EE600023F000BF95EE010811EF010803EF010840
:10EE700003EF010803EF010803EF010803EF0108A6
:10EE800003EF010803EF010803EF0108BFEE0108DB
:10EE9000E9EE01087B6893F89C32DBB2032B07D1C3
:10EEA00007F10A03022219467868FFF740FE32E0B4
:10EEB00039687868FFF7CAFD0323FB752BE07B6890
:10EEC00093F89C32DBB2032B07D107F10D0301222B
:10EED00019467868FFF72BFE1DE039687868FFF760
:10EEE000B5FD0323FB7516E07B6893F89C32DBB21B
:10EEF000032B0FD039687868FFF7A8FD0323FB7553
:10EF000008E039687868FFF7A1FD0323FB7502E08C
:10EF100000BF08E000BF06E039687868FFF796FD9B
:10EF20000323FB7500BFFB7D18461837BD4680BD27
:10EF300080B584B000AF78600B46FB707B68D3F877
:10EF4000C432FB607B68D3F8BC32002B01D10323B1
:10EF50004FE07B68D3F8BC32BB60FA78796813461F
:10EF60009B0013449B000B4418331B68002B29D0D3
:10EF7000FA78796813469B0013449B000B441833BE
:10EF80001A68F978F8680B469B000B44DB000344D1
:10EF900020331B68B2FBF3F101FB03F3D31A002B00
:10EFA00010D1FA78796813469B0013449B000B44F8
:10EFB000183300221A60F978002300227868F4F7E9
:10EFC00014FA15E0BB680022C3F814227B68D3F85A
:10EFD000C0321B69002B0BD07B68D3F8C0321B6991
:10EFE000BA68D2F80802BA6802F50471FA7898474C
:10EFF000002318461037BD4680BD80B584B000AFF1
:10F0000078600B46FB707B68D3F8BC32FB607B6892
:10F01000D3F8BC32002B01D1032315E0FB7819464D
:10F020007868F4F724FA0246FB68C3F80C227B6880
:10F03000D3F8C032DB68FA68D2F80402FA6802F545
:10F04000037211469847002318461037BD4680BD0D
:10F0500080B584B000AF78607B68D3F8BC32FB60C9
:10F06000FB68002B01D103231AE07B68D3F8C03280
:10F07000002B14D0FB6893F80032FF2B0FD07B6875
:10F08000D3F8C0329B68FA6892F80002F968FA680F
:10F0900092F801229847FB68FF2283F800220023A0
:10F0A00018461037BD4680BD80B483B000AF78608D
:10F0B0007B6843221A80034B18460C37BD465DF827
:10F0C000047B70477801002080B483B000AF786083
:10F0D0007B6843221A80034B18460C37BD465DF807
:10F0E000047B70473401002080B483B000AF7860A7
:10F0F0007B6843221A80034B18460C37BD465DF8E7
:10F10000047B7047BC01002080B483B000AF7860FE
:10F110007B680A221A80034B18460C37BD465DF8FF
:10F12000047B7047F000002080B483B000AF7860AB
:10F1300039603B68002B01D1032304E07B683A6807
:10F14000C3F8C022002318460C37BD465DF8047B87
:10F15000704780B487B000AFF860B9607A60FB6830
:10F16000D3F8BC327B617B69002B01D1032308E01B
:10F170007B69BA68C3F808227B697A68C3F81022F1
:10F18000002318461C37BD465DF8047B704780B4E9
:10F1900085B000AF786039607B68D3F8BC32FB6023
:10F1A000FB68002B01D1032304E0FB683A68C3F835
:10F1B0000422002318461437BD465DF8047B7047CF
:10F1C00080B584B000AF78607B68D3F8BC32BB6098
:10F1D0000123FB737B68D3F8BC32002B01D10323DE
:10F1E0001AE0BB68D3F81432002B14D1BB6801229B
:10F1F000C3F81422BB68D3F810227B68DA62BB68BC
:10F20000D3F80822BB68D3F8103281217868F4F76C
:10F21000ECF80023FB73FB7B18461037BD4680BD1E
:10F2200080B584B000AF78607B68D3F8BC32FB60F7
:10F230007B68D3F8BC32002B01D1032316E07B6836
:10F240001B7C002B09D1FB68D3F804224FF4007318
:10F2500001217868F4F7EAF807E0FB68D3F80422A4
:10F26000402301217868F4F7E1F8002318461037AD
:10F27000BD4680BD80B586B000AF7860144A154B9E
:10F28000D31A7B617B693B61134B1B68002B02D156
:10F29000114B124A1A60104B1A687B6813443A6982
:10F2A0009A4207D200F06CF903460C221A604FF024
:10F2B000FF3309E0084B1B68FB60074B1A687B684B
:10F2C0001344054A1360FB6818461837BD4680BDD5
:10F2D0000000022000080000582C0020602C0020B4
:10F2E00080B400AF01231846BD465DF8047B70472B
:10F2F00080B582B000AF7860396000F041F9034614
:10F3000016221A604FF0FF3318460837BD4680BDFD
:10F3100080B582B000AF78604FF0FF317868FFF7BA
:10F32000E7FF00BFFDE780B586B000AFF860B960C9
:10F330007A6000237B610AE0AFF300800146BB687E
:10F340005A1CBA60CAB21A707B6901337B617A6950
:10F350007B689A42F0DB7B6818461837BD4680BD53
:10F3600080B586B000AFF860B9607A6000237B6139
:10F3700009E0BB685A1CBA601B781846F2F752F8CD
:10F380007B6901337B617A697B689A42F1DB7B6838
:10F3900018461837BD4680BD80B483B000AF786092
:10F3A0004FF0FF3318460C37BD465DF8047B7047BD
:10F3B00080B483B000AF786039603B684FF400528E
:10F3C0005A60002318460C37BD465DF8047B704731
:10F3D00080B483B000AF7860012318460C37BD4677
:10F3E0005DF8047B704780B485B000AFF860B96009
:10F3F0007A60002318461437BD465DF8047B7047D9
:10F400000D488546FEF7DEFA0C480D490D4A0023EB
:10F4100002E0D458C4500433C4188C42F9D30A4AC9
:10F420000A4C002301E013600432A242FBD3F1F73F
:10F430001DFAF1F7F7FBFEE70000022000000020B4
:10F4400000020020C80E0208000200205C2C0020F0
:10F45000FEE700001FB514461A46094B1B68054617
:10F46000D86854B9074B1C46CDE9013400912B46AE
:10F47000054900F015F800F089F8044BF4E700BFE7
:10F480000C000020670D0208390D02082C0D02083F
:10F49000024B01461868F1F77DBA00BF0C0000204E
:10F4A0000EB403B5014603AB054853F8042B0068BE
:10F4B000019300F0BFFB02B05DF804EB03B07047AE
:10F4C0000C0000200CB430B5174B0C1E1D689DB00D
:10F4D00008DA8B232B604FF0FF301DB0BDE83040C1
:10F4E00002B070474FF40273ADF8143014BF04F14A
:10F4F000FF332346049307934FF6FF730290069061
:10F50000ADF81630209A21AB02A92846019300F0ED
:10F510009FF8431CBCBF8B232B60002CDDD0029BCB
:10F5200000221A70D9E700BF0C0000200EB430B5DD
:10F530009CB01FAC4FF4017254F8045BADF814207A
:10F5400002900690F0F7E4FF0B4B039007900B93AB
:10F550000A48019400230F9314934FF6FF73ADF8FC
:10F5600016302A46234602A9006800F0C5F91CB0EF
:10F57000BDE8304003B07047670701080C00002069
:10F58000014B1868704700BF0C00002008B506202A
:10F5900001F08EF80120FFF7BBFE2DE9F0478E68E1
:10F5A0001F46BE420B6882460C4690462DD8B1F9E4
:10F5B0000C2012F4906F26D06569096905EB4505AA
:10F5C000A3EB010905EBD5757B1C4B446D109D42E7
:10F5D00038BF1D46530527D52946F1F7DBF9064606
:10F5E00060B321694A4601F07FF8A38923F4906350
:10F5F00043F08003A381266165614E44A5EB0905B4
:10F600002660A5603E46BE4200D93E46206832468E
:10F61000414601F00BF8A3689B1BA36023683344A9
:10F6200023600020BDE8F0872A4601F06BF806460B
:10F630000028E0D121695046F1F740F90C23CAF8BF
:10F640000030A38943F04003A3814FF0FF30E9E786
:10F650002DE9F04F98468B891B069DB007460D4655
:10F66000144610D50B6973B94021F1F793F928605E
:10F67000286130B90C233B604FF0FF301DB0BDE86E
:10F68000F08F40236B610023099320238DF82930EC
:10F69000CDF80C803023DFF89C818DF82A304FF0B4
:10F6A000010923469A4613F8012B0AB1252AF9D1FC
:10F6B000BAEB040B0BD05B46224629463846FFF7CF
:10F6C0006CFF013000F0A780099A5A4409929AF819
:10F6D0000030002B00F09F8000234FF0FF32CDE977
:10F6E00005230AF1010A049307938DF853301A9306
:10F6F0005446052214F8011B4E48F0F711FF049AF6
:10F70000D8B9D00644BF20238DF85330110744BF29
:10F710002B238DF853309AF800302A2B15D0079AF6
:10F72000544600204FF00A0C214611F8013B303BB3
:10F73000092B4BD9B0B1079214E0A0EB080309FAEA
:10F7400003F313430493A246D2E7039B191D1B68DE
:10F750000391002BBBBF5B4242F002020793079369
:10F76000B8BF049223782E2B0AD163782A2B32D18A
:10F77000039B1A1D1B68039243EAE373023405934B
:10F78000DFF8C0A0217803225046F0F7C9FE38B157
:10F79000049BA0EB0A0040228240134301340493EF
:10F7A00014F8011B24488DF828100622F0F7B8FE43
:10F7B000002836D0214B1BBB039B073323F00703E4
:10F7C00008330393099B334409936AE70CFB023225
:10F7D0000C460120A8E700230134059319464FF099
:10F7E0000A0C204610F8012B303A092A03D9002BC5
:10F7F000C6D00591C4E70CFB012104460123F0E7C4
:10F8000003AB00932A460E4B04A93846AFF30080A1
:10F81000421C0646D6D1AB895B063FF52DAF099851
:10F820002CE703AB00932A46054B04A9384600F0A9
:10F8300087FBEDE7680D0208720D0208000000006A
:10F840009BF501086E0D020838B54B1C144603D118
:10F850004FF0FF35284638BD938923F0200393816C
:10F860005368526BCDB28AB1A26B9A4208DD23680D
:10F870005A1E226003F8015C636801336360E9E7A4
:10F88000214600F004FE0028F1D0E1E7216922685A
:10F8900041B1914206D212F8011CA94202D1013AAB
:10F8A0002260EAE7C4E90F2304F1440363630323FE
:10F8B000A363234603F8465F23600123DEE710B508
:10F8C0000C46496B69B104F14403994201D0F0F749
:10F8D000F5FF236C63600020606313B1E36B23606A
:10F8E00010BD2369236000236360A38943F02003D4
:10F8F000A3814FF0FF30F3E72DE9F0470C46ADF55B
:10F90000227D0021CDE94411A549A0910DF1040803
:10F91000A449A54FCDF818810646A191009313780C
:10F92000002B00F05881F95C11F0080102F101058B
:10F9300019D06368002B0FDD23681A78BA5C1207B0
:10F9400001D42A46EBE7459A0132459262680133B9
:10F95000013A62602360ECE7A19B2146304698475C
:10F960000028E9D0EDE7252B12D099466368002BDB
:10F9700040F39380226813784B4540F02C816368F4
:10F98000013B6360459B0132013322604593D8E718
:10F990004191439153782A2B02BF1023951C419328
:10F9A0000A22A94619F8011BA1F13003092B1ED91F
:10F9B000DFF8F8A103225046F0F7B2FD38B1419AC2
:10F9C000A0EB0A0001238340134341934D4615F8F1
:10F9D000013B782B06D8572B10D8252BC5D057D8EC
:10F9E000002B65D0032347930A23429378E0439B7F
:10F9F00002FB0311303943914D46D2E7A3F158027F
:10FA0000202AEFD801A151F822F000BFBFFA010867
:10FA1000E5F90108E5F9010819FB0108E5F9010814
:10FA2000E5F90108E5F90108E5F90108E5F901083A
:10FA3000E5F90108E5F901082FFB010815FB0108AC
:10FA400097FA010897FA010897FA0108E5F9010801
:10FA5000D1FA0108E5F90108E5F90108E5F901081D
:10FA6000E5F901083FFB0108D9FA0108B7FA0108D6
:10FA7000E5F90108E5F901083BFB0108E5F9010892
:10FA800015FB0108E5F90108E5F90108BFFA0108CD
:10FA9000453B022BA6D8052321E0A19B21463046F9
:10FAA000984700283FF466AF4498002840F08B80C8
:10FAB0004FF0FF308BE0419A42F020024192419A90
:10FAC00042F40072419210226E2B429202D905E05C
:10FAD00000234293032302E0082342930423479325
:10FAE0006368002B39DD419B590604D423681A78DA
:10FAF000BA5C120738D4479B022B47DC6B46224680
:10FB000041A9304600F03CFB012864D002287FF474
:10FB100018AFC9E70A22D7E72946404600F07EFC25
:10FB2000419B43F04003419305460123D7E7419BA6
:10FB300043F0400341930023D1E70223CFE74198EC
:10FB4000C3063FF5FEAE009B459A191D00911B6848
:10FB5000C0074CBF1A801A60F3E6A19B21463046CD
:10FB600098470028BFD09FE7459A013245926268C6
:10FB7000013A002A626002DD01332360B6E7A19BEF
:10FB80002146304698470028B0D08DE7042B0FDC83
:10FB90006B46224641A9304600F04CFBB4E700BF5B
:10FBA00049F80108BFF80108B70D02086E0D0208F8
:10FBB0000A4B002B3FF4C5AE6B46224641A93046A6
:10FBC000AFF30080A0E7A3895B063FF571AF0DF5A9
:10FBD000227DBDE8F0874498F9E700BF00000000EF
:10FBE0009368013B002B10B4936008DA9469A34238
:10FBF00001DB0A2903D15DF8044B00F082BC1368D5
:10FC0000581C1060197008465DF8044B7047F8B531
:10FC100006460F461446D518AC4201D1002007E035
:10FC200014F8011B3A463046FFF7DAFF431CF3D1C4
:10FC3000F8BD00002DE9F04F0D469DB014469846E2
:10FC4000064618B1036A0BB9F0F746FD6B6ED9078B
:10FC500005D4AB899A0502D4A86DF0F72CFEAB89C8
:10FC60001B0701D52B699BB92946304600F088FC5B
:10FC700070B16B6EDC0704D54FF0FF301DB0BDE8EE
:10FC8000F08FAB899805F7D4A86DF0F715FEF3E770
:10FC90000023099320238DF82930CDF80C803023E0
:10FCA000DFF8AC818DF82A304FF0010923469A46DF
:10FCB00013F8012B0AB1252AF9D1BAEB040B0BD0AA
:10FCC0005B46224629463046FFF7A1FF013000F08F
:10FCD000A780099A5A4409929AF80030002B00F044
:10FCE0009F8000234FF0FF32CDE905230AF1010A7E
:10FCF000049307938DF853301A935446052214F851
:10FD0000011B5348F0F70CFC049AD8B9D10644BF44
:10FD100020238DF85330130744BF2B238DF8533025
:10FD20009AF800302A2B15D0079A544600204FF03D
:10FD30000A0C214611F8013B303B092B4BD9B0B1DD
:10FD4000079214E0A0EB080309FA03F313430493AA
:10FD5000A246D2E7039B191D1B680391002BBBBF72
:10FD60005B4242F0020207930793B8BF04922378E4
:10FD70002E2B0AD163782A2B32D1039B1A1D1B68C4
:10FD8000039243EAE37302340593DFF8D4A02178A9
:10FD900003225046F0F7C4FB38B1049BA0EB0A00E5
:10FDA0004022824013430134049314F8011B294874
:10FDB0008DF828100622F0F7B3FB00283FD0264B21
:10FDC0001BBB039B073323F0070308330393099BF3
:10FDD0003B4409936AE70CFB02320C460120A8E77A
:10FDE00000230134059319464FF00A0C204610F801
:10FDF000012B303A092A03D9002BC6D00591C4E75C
:10FE00000CFB012104460123F0E703AB00932A46D3
:10FE1000124B04A93046AFF300800746781CD6D1B8
:10FE20006B6ED90705D4AB899A0502D4A86DF0F79B
:10FE300043FDAB895B063FF51FAF09981EE703AB97
:10FE400000932A46054B04A9304600F079F8E4E710
:10FE5000680D0208720D0208000000000FFC010886
:10FE60006E0D02082DE9F047164698468A680B6920
:10FE7000DDF820909342B8BF1346336091F84320D9
:10FE800007460C460AB1013333602368990642BF26
:10FE9000336802333360256815F0060506D104F196
:10FEA000190AE36832689B1AAB4226DC94F84330A7
:10FEB0002268003B18BF012392062BD404F14302B1
:10FEC00041463846C84701301ED02368226903F0F6
:10FED0000603042B02BFE5683368ED1AA3680CBF64
:10FEE00025EAE57500259342C4BF9B1AED1800264C
:10FEF0001A34B5421AD1002008E001235246414687
:10FF00003846C847013003D14FF0FF30BDE8F087D5
:10FF10000135C6E7E1185A1C302081F8430022441D
:10FF200094F8451082F843100233C7E701232246B4
:10FF300041463846C8470130E6D00136D9E70000CF
:10FF40002DE9FF470F7E0C9E782F914680460C4688
:10FF50009A4601F1430207D8622F0AD8002F00F019
:10FF6000D280582F00F0B98004F1420684F8427024
:10FF70003AE0A7F16303152BF6D801A151F823F05D
:10FF8000D9FF0108EDFF010869FF010869FF0108B9
:10FF900069FF010869FF0108EDFF010869FF010819
:10FFA00069FF010869FF010869FF0108ED00020807
:10FFB00017000208A700020869FF010869FF01088D
:10FFC0000F01020869FF01081700020869FF010814
:10FFD00069FF0108AF00020833681A1D1B68326010
:10FFE00004F1420684F8423001239DE03368206822
:10FFF000191D3160060601D51D6803E04506FBD5D5
:020000040802F0
:10000000B3F90050002D03DA2D236D4284F84330FC
:1000100059480A2311E021683368080653F8045B45
:1000200002D4490648BFADB26F2F5348336014BFA6
:100030000A230823002184F843106668A660002E76
:10004000A2BF216821F0040121600DB9002E4BD020
:100050001646B5FBF3F103FB1157C75D06F8017DAA
:100060002F46BB420D46F4D9082B0BD12368DF077E
:1000700008D5236961689942DEBF302306F8013C48
:1000800006F1FF36921B2261CDF800A04B4603AA71
:1000900021464046FFF7E6FE01304AD14FF0FF30DF
:1000A00004B0BDE8F087236843F0200323603348A1
:1000B000782784F84570236831681F0651F8045B7F
:1000C00002D45F0648BFADB23160D90744BF43F0E8
:1000D000200323601DB11023ACE72748E9E723681C
:1000E00023F020032360F6E71646BDE73368256852
:1000F0006169181D30602E061B6801D5196002E089
:100100006806FBD51980002323611646BCE73368D7
:100110001A1D32601E68626800213046F0F700FA4E
:1001200008B1801B606063682361002384F843305A
:10013000AAE72369324649464046D0470130ADD050
:1001400023689B0713D4E068039B9842B8BF184606
:10015000A6E70123324649464046D04701309DD0AC
:100160000135E36803995B1AAB42F2DCEBE700254B
:1001700004F11906F5E700BF790D02088A0D02089F
:100180002DE9F84315468A6880460C4632B98A69DB
:10019000002A14BF4FF0FF3201228A602268DFF884
:1001A0009090D1065FBF1A68111D1960166800276C
:1001B000A06988B1012807D12B681A7863699B5C14
:1001C00053B9002F31D022E0022820D12B681B78B0
:1001D00019F803301B071AD42368DA065EBF2B68B0
:1001E0001B7806F8013B2A686B6801322A60A26816
:1001F000013B013A6B600137A26042B1002BD7DCB2
:10020000D4F880312946404698470028D0D023684A
:1002100013F0100305D1E2680132E260A26902B175
:10022000337023693B4423610020BDE8F88300BF9D
:10023000B70D02082DE9F04F9846744B0C468246E4
:10024000164693E8070087B003AB83E80700704BBE
:10025000A169704A032908BF1A46A36801925A1E71
:10026000B2F5AE7F88BF6FF4AE75274682BF03EB51
:10027000050940F25D13A36057F81C3B43F450633B
:1002800098BF4FF0000923603D464FF0000B3168E6
:1002900003AB097853F82B000222F0F741F928B399
:1002A000BBF1010F59D162682AB92268082142F4D2
:1002B000007261602260226822F4A0622260A2685B
:1002C000511EA16092B13268511C3160127805F85C
:1002D000012B7268013A002A726007DCD4F8802191
:1002E000314650469047002840F085800BF1010BC5
:1002F000BBF1030FCBD163680BB90A23636063685A
:1003000045496069C91A00F089F84FF0000BA368ED
:100310002268002B3DD03168606991F800C010F868
:100320000C00002835D0BCF1300F24D1100522D5A7
:100330000BF1010BB9F1000F03D0013309F1FF39C3
:10034000A3607368013B002B73601BDD33680133CE
:100350003360A368013BA360D9E7BBF1020FAED1C4
:10036000226802F4C061B1F5007FBFD11021616045
:1003700042F48072A2E722F4106222600B7805F842
:10038000013BDEE7D4F880313146504698470028DB
:10039000DFD02368D9050DD5BD4209D915F8011C58
:1003A000D4F87C3132465046984705F1FF394D4626
:1003B000BD4228D0226812F0100213D12A7063685F
:1003C000019E39465046B047D8F8003021681A1DC2
:1003D000C8F8002011F0200F1B680FD01860E368E8
:1003E0000133E3602369ED1B5D442B44236100204E
:1003F00007B0BDE8F08F4FF0000BCAE7CA074CBF4B
:1004000018801860EBE70120F2E700BF380C020803
:100410005508020835090208AB0D020870B50B78C3
:1004200004465E2B0BBF4B784A1C8A1C002108BF78
:100430000121013804F1FF0500F8011FA842FBD19A
:100440000BB9501E70BD81F00101E1541046024607
:1004500012F8015B2D2D05D05D2D16D0002DF1D0A9
:100460002B46F2E746785D2EFAD0B342F8DC023034
:100470001A4601329642A154FBDCF21A013A5D1C85
:10048000B342A8BF0022AB18E1E71046DAE72DE936
:10049000F0410C46496B04F1440399421DD14FF4DD
:1004A0008061F0F777FA18B94FF0FF30BDE8F081BE
:1004B0004FF48063A36394F84630606380F8FF33A1
:1004C00094F8453080F8FE3394F8443080F8FD33DA
:1004D00000F2FD3020600020E8E7A66B77003A4686
:1004E00000F010F905460028DED000EB06080146B2
:1004F0003246404600F0F8F8C4E90D57C4F80080D1
:10050000E9E7F8B50E461446054618B1036A0BB97B
:10051000F0F7E2F8A369A360A3891A0701D523695C
:1005200043B92146284600F02BF818B14FF0FF37A9
:100530003846F8BD23682269981A6369F6B2834287
:10054000374605DC21462846F0F734FB0028EDD17C
:10055000A368013BA36023685A1C22601E70626975
:10056000431C9A4204D0A389DB07E1D50A2EDFD1D0
:1005700021462846F0F71EFB0028D9D0D6E7000018
:1005800038B5294B054618680C4618B1036A0BB9F3
:10059000F0F7A2F8B4F90C30190722D4DA0607D420
:1005A00009222A6043F04003A3814FF0FF3033E07B
:1005B000580712D5616B41B104F14403994202D04E
:1005C0002846F0F77BF900236363A38923F0240313
:1005D000A3810023636023692360A38943F0080398
:1005E000A38123694BB9A38903F42073B3F5007F7A
:1005F00003D02146284600F0C5F9B4F90C3013F0B9
:1006000001020AD00022A26062695242A2612269FC
:1006100042B913F08000C5D138BD990758BF62694F
:10062000A260F4E70020F7E70C000020884210B534
:1006300001EB020402D98442234607D8431EA1429B
:1006400008D011F8012B03F8012FF8E70244014606
:100650008A4200D110BD13F8014D02F8014DF7E7B1
:100660001F2938B505460C4604D9162303604FF000
:10067000FF3038BDC26B12B152F821304BB9284659
:1006800000F030F8224601462846BDE8384000F028
:1006900017B8012B0AD0591C03D11623036001207F
:1006A000E7E7002142F82410204698470020E0E7C1
:1006B000024B01461868FFF7D3BF00BF0C000020B3
:1006C00038B5074D00230446084611462B60FEF757
:1006D0000FFE431C02D12B6803B1236038BD00BF5D
:1006E00058030020FEF7FCBD0A44914200F1FF339D
:1006F00000D1704710B511F8014B03F8014F91423A
:10070000F9D110BD2DE9F041804615460C4621B9BE
:10071000BDE8F0411146F0F73DB92AB9F0F7CEF83F
:1007200000242046BDE8F08100F08AF985420646A3
:1007300002D8B5EB500FF4D829464046F0F72AF915
:1007400007460028ECD0B5422A46214628BF32464B
:10075000FFF7CAFF21464046F0F7B0F83C46E0E715
:10076000242B2DE9F0478646904601D8012B06D16F
:10077000FEF706FF162303600020BDE8F08734482B
:100780000D462A4615F8014B065D16F00806F8D10D
:100790002D2C2DD12C780126951C33F0100209D177
:1007A000302C2AD12A7802F0DF02582A25D16C7821
:1007B0001023023506F1004C0CF1FF3C0022BCFB7B
:1007C000F3F9104603FB19CAA4F13007092F1BD80F
:1007D0003C46A34227DD571C07D0814520D301D1D9
:1007E000A2451DDB00FB0340012215F8014BEBE79E
:1007F0002B2C04BF2C78951CCFE7002BDAD1302CA2
:100800000CBF08230A23D5E7A4F14107192F01D80B
:10081000373CDEE7A4F16107192F04D8573CD8E72D
:100820004FF0FF32E1E7531C08D12223CEF800300D
:100830006046B8F1000FA0D0691E06E006B1404244
:10084000B8F1000F99D0002AF6D1C8F8001094E74B
:10085000B70D0208FFF784BF2DE9F043344E8646FA
:100860000D46284615F8014B375D17F00807F8D1FB
:100870002D2C2FD12C780127851C33F0100009D1A5
:10088000302C2CD1287800F0DF00582827D16C7844
:10089000102302354FF0FF380026B8FBF3F803FBB6
:1008A00008F96FEA09093046A4F1300CBCF1090FD0
:1008B0001CD86446A3422ADDB6F1FF3F07D080452D
:1008C00022D301D1A1451FDB00FB0340012615F80F
:1008D000014BE9E72B2C04BF2C78851CCDE7002BBE
:1008E000D8D1302C0CBF08230A23D3E7A4F1410C44
:1008F000BCF1190F01D8373CDCE7A4F1610CBCF165
:10090000190F04D8573CD5E74FF0FF36DFE7731CCB
:1009100006D12223CEF80030304632B9BDE8F0834C
:1009200007B14042002AF9D006B1691E1160F5E70F
:10093000B70D0208FFF790BF70B50C46B1F90E1065
:10094000002996B015461E460DDAA38913F0800FD4
:100950004FF0000114BF40234FF48063002031604A
:100960002B6016B070BD6A4600F048F80028ECDB3A
:10097000019901F47041A1F50053594259414FF4D6
:100980008063EBE78B89F7B59D0706460C4607D5D4
:1009900004F14703236023610123636103B0F0BDC9
:1009A00001AB6A46FFF7C8FF009F0546394630464F
:1009B000EFF7F0FF48B9B4F90C309A05EED423F004
:1009C000030343F00203A381E2E7A389206043F01D
:1009D0008003A381019BC4E904075BB1B4F90E1045
:1009E000304600F01DF828B1A38923F0030343F03B
:1009F0000103A381A3891D43A581CFE738B5074D26
:100A000000230446084611462B60FEF7D1FC431C28
:100A100002D12B6803B1236038BD00BF580300200A
:100A200038B5064D0023044608462B60FEF7D0FC7F
:100A3000431C02D12B6803B1236038BD580300204A
:100A400051F8043C181F002BBCBF0B58C01870474E
:100A5000F8B500BFF8BC08BC9E467047F8B500BFAB
:080A6000F8BC08BC9E4670477B
:100A68006D650000443A2F4E657874436C6F756469
:100A78002F50726F6A656374732F50776E5F446589
:100A8800636B2F53572F53572F436F72652F537232
:100A9800632F6369725F6275662E630062756666AE
:100AA80065722026262073697A6500006362756680
:100AB8000000000063697263756C61725F6275663D
:100AC8005F656D707479286362756629000000009F
:100AD8006D65202626206D652D3E627566666572F9
:100AE800000000006D6520262620646174612026C0
:100AF80026206D652D3E62756666657200000000F1
:100B0800256C64004D61696E204D656E753A0D0A5D
:100B1800536C69646572205B315D3A2022256C69EB
:100B2800220D0A536C69646572205B325D3A20229B
:100B3800256C69220D0A536C69646572205B335D0C
:100B48003A2022256C69220D0A536C69646572206B
:100B58005B345D3A2022256C69220D0A5B535D6186
:100B680076650D0A56657273696F6E3A2025730DA6
:100B78000A456E7465722053656C656374696F6E9F
:100B88003A20000056312E312E310000536C696432
:100B9800657220256C75204D61782056616C7565ED
:100BA8002028302D313030293A2000005341564555
:100BB8004421213121000000534156452046414936
:100BC8004C454421000000001B5B313B306D0000A8
:100BD8001B5B313B33316D001B5B313B33326D00A6
:100BE8001B5B324A1B5B480053544D333220566915
:100BF800727475616C20436F6D506F7274000000E1
:100C080053544D6963726F656C656374726F6E6976
:100C18006373000043444320436F6E6669670000B6
:100C280043444320496E7465726661636500000041
:100C3800AD0D0208B00D0208B30D020861647661BB
:100C48006E63655F686561645F706F696E74657215
:100C58000000000063697263756C61725F6275669B
:100C68005F696E697400000063697263756C617214
:100C78005F6275665F7265736574000063697263AD
:100C8800756C61725F6275665F73697A65000000F2
:100C980063697263756C61725F6275665F7472799D
:100CA8005F7075740000000063697263756C61722F
:100CB8005F6275665F676574000000006369726350
:100CC800756C61725F6275665F656D70747900003E
:100CD80063697263756C61725F6275665F66756C75
:100CE8006C000000010002000400060008000A0071
:100CF8000C001000200040008000000101010103E9
:100D080007010000080402040801010100000000B6
:100D180000000000010203040607080900000000A3
:100D2800010203042C2066756E6374696F6E3A20A5
:100D380000617373657274696F6E202225732220B7
:100D48006661696C65643A2066696C652022257362
:100D5800222C206C696E65202564257325730A0092
:100D6800232D302B2000686C4C006566674546478C
:100D7800003031323334353637383941424344450F
:100D8800460030313233343536373839616263647E
:100D9800656600412D46612D66383930313233346D
:100DA8003536375D002B2D00303000785800002094
:100DB8002020202020202020282828282820202003
:100DC80020202020202020202020202020202088B3
:100DD8001010101010101010101010101010100417
:100DE8000404040404040404041010101010101067
:100DF800414141414141010101010101010101015B
:100E08000101010101010101010110101010101070
:100E1800424242424242020202020202020202022A
:100E28000202020202020202020210101010200046
:100E380000000000000000000000000000000000AA
:100E4800000000000000000000000000000000009A
:100E5800000000000000000000000000000000008A
:100E6800000000000000000000000000000000007A
:100E7800000000000000000000000000000000006A
:100E8800000000000000000000000000000000005A
:100E9800000000000000000000000000000000004A
:100EA800000000000000000000000000000000003A
:080EB80098F3FE7F0100000029
:040EC000050201081E
:040EC400E10101083F
:100EC80000000000030000001C02002010000020A9
:100ED800000000001C02002084020020EC02002018
:100EE80000000000000000000000000000000000FA
:100EF80000000000000000000000000000000000EA
:100F080000000000000000000000000000000000D9
:100F1800000000000000000000000000F535010896
:100F280019360108793601083D360108A13601084D
:100F3800C53601080137010800000000120100024F
:100F4800020200408304405700020102030100002E
:100F5800040309041A030000000000000000000058
:100F68000000000000000000000000000000000079
:100F7800153801083D3801084D38010809390108BC
:100F8800A139010810000000010000000000000065
:100F98000000000000000000000000000100000048
:100FA8000000000000000000000000000024F40021
:100FB8000A06000200000040010000002FEC0108B2
:100FC8002DED0108A1ED01080000000051F0010815
:100FD80031EF0108FBEF01080000000000000000ED
:100FE80000000000C9F00108A9F00108E9F00108B3
:100FF80009F1010809024300020100C03209040096
:10100800000102020100052400100105240100016D
:1010180004240202052406000107058203080010C3
:1010280009040100020A000000070501020002008D
:10103800070581020002000009024300020100C006
:101048003209040000010202010005240010010514
:101058002401000104240202052406000107058278
:101068000308001009040100020A00000007050136
:101078000240000007058102400000000907430004
:10108800020104C032090400000102020100052423
:1010980000100105240100010424020205240600B1
:1010A800010705820308001009040100020A000074
:1010B800000705010240000007058102400000000A
:040000050801F401F9
:00000001FF
